:10000000FCFB0220D101000035340100ED3301007A
:10001000ED330100ED330100ED330100ED3301005C
:10002000ED330100ED330100ED3301003534010003
:1000300035340100ED330100914F0100E151010021
:100040003534010035340100353401003534010008
:1000500035340100353401003534010035340100F8
:1000600035340100353401003534010035340100E8
:1000700035340100353401003534010035340100D8
:1000800035340100353401003534010035340100C8
:1000900035340100353401003534010035340100B8
:1000A000692F01007D2F01006530010089310100B9
:1000B000353401003534010035340100815301002D
:1000C000353401009D55010035340100B957010058
:1000D00035340100B958010035340100412F0100C9
:1000E0003534010035340100353401003534010068
:1000F0003534010035340100353401003534010058
:10010000B92F0100D12F0100E92F010001300100BA
:10011000353401009D4101003534010035340100C2
:100120003534010035340100353401003534010027
:100130003534010035340100353401003534010017
:100140003534010035340100B9590100353401005E
:1001500035340100353401003534010035340100F7
:1001600035340100552F0100912F01003534010075
:1001700035340100353401003534010035340100D7
:1001800035340100253001003534010035340100DB
:100190003534010035340100B95A0100353401000D
:1001A000353401003534010035340100A52F01003C
:1001B0003534010035340100353401003534010097
:1001C0003534010035340100353401003534010087
:1001D000614B4CF220524DF6281010B51A80188051
:1001E00000BF00BF5D4C13F029F94FF03061216072
:1001F0005B4B5C49A3604FF470005B4A5B4BE26071
:1002000008605B4C5B481C6090F800C05FEA0C71B2
:1002100004D590F800E04EF008020270564C574AA0
:10022000574BAA212170574CA34204D252F8040F15
:1002300043F8040BF8E7544954480024814202D2A1
:1002400041F8044BFAE75249524A002352F823007E
:1002500041F823000133742BF8D14F4C4F498023D0
:1002600004F8013B8C42FBD14D4B4E48484A02609A
:10027000A3F5805C8A242421A0221C708CF8011034
:100280008CF800209CF806008207FBD59CF80640FD
:10029000E406FBD4444991F806E00EF00C03082B69
:1002A000F9D142486022027002300478802CFCD1DF
:1002B0003D4B01215D2219715A7198798006FCD558
:1002C00093F806C0384C5FEA4C61F9D5384B394990
:1002D0001960002220205A602070A17901F00C03DF
:1002E0000C2BFAD1344A354C354814600168354C32
:1002F00011F4807303D14FF4A85223600260324995
:10030000324808600023072231484B6041F8042C32
:10031000C1F80C0D62B613F083F92468E20705D525
:100320002C4813F06BF92C4B2C4919602C4A10788F
:10033000430609D5284C294B2168994204D1254808
:1003400013F05CF90022226015F0CEFC13F07CF86B
:1003500012F0ACFFFEE700BF0E20054030800440E5
:10036000823F040088ED00E00100002B002008E03F
:100370000300008502D0074000E00740D4BB010025
:100380003007FF1F3014FF1F3014FF1F5449012096
:100390000002FF1F0000000000E400E064E400E051
:1003A0000050064008ED00E00040064001E0074034
:1003B000448004400000060204800440C01007008E
:1003C00010D0034014D0034014E000E01FBF02002F
:1003D000000020207BBE5B661CE00340A5C3945A4E
:1003E00000F00740FFFFFFFFFFFFFFFFFFFFFFFFE2
:1003F000FFFFFFFFFFFFFFFFFFFFFFFFFFFFFFFF0D
:10040000FFFFFFFFFFFFFFFFFFFFFFFFDEF9FFFF23
:1004100010B5054C237833B9044B13B10448AFF33E
:1004200000800123237010BD3014FF1F0000000066
:10043000D0BB0100084B10B51BB108490848AFF309
:1004400000800848036803B910BD074B002BFBD0A0
:10045000BDE81040184700BF000000003414FF1F23
:10046000D0BB01003014FF1F00000000034B586890
:1004700010B101680A681047704700BFA44301200B
:10048000034B986810B101680A681047704700BFB5
:10049000A4430120034BD86810B101680A681047D3
:1004A000704700BFA4430120034B186910B10168D5
:1004B0000A681047704700BFA4430120034B5869E6
:1004C00010B101680A681047704700BFA4430120BB
:1004D000034B986910B101680A681047704700BF64
:1004E000A4430120034BD86910B101680A68104782
:1004F000704700BFA4430120034B186A10B1016884
:100500000A681047704700BFA4430120034B586A94
:1005100010B101680A681047704700BFA44301206A
:10052000034B986A10B101680A681047704700BF12
:10053000A4430120034BD86A10B101680A68104730
:10054000704700BFA4430120034B186B10B1016832
:100550000A681047704700BFA4430120034B586B43
:1005600010B101680A681047704700BFA44301201A
:10057000034B986B10B101680A681047704700BFC1
:10058000A4430120034BD86B10B101680A681047DF
:10059000704700BFA4430120034B186C10B10168E1
:1005A0000A681047704700BFA4430120034B586CF2
:1005B00010B101680A681047704700BFA4430120CA
:1005C000034B986C10B101680A681047704700BF70
:1005D000A4430120034BD86C10B101680A6810478E
:1005E000704700BFA4430120034B186D10B1016890
:1005F0000A681047704700BFA4430120034B586DA1
:1006000010B101680A681047704700BFA443012079
:10061000034B986D10B101680A681047704700BF1E
:10062000A4430120034BD86D10B101680A6810473C
:10063000704700BFA4430120034B186E10B101683E
:100640000A681047704700BFA4430120034B586E4F
:1006500010B101680A681047704700BFA443012029
:10066000034B986E10B101680A681047704700BFCD
:10067000A4430120034BD86E10B101680A681047EB
:10068000704700BFA4430120034B186F10B10168ED
:100690000A681047704700BFA4430120034B586FFE
:1006A00010B101680A681047704700BFA4430120D9
:1006B000034B986F10B101680A681047704700BF7C
:1006C000A4430120034BD86F10B101680A6810479A
:1006D000704700BFA4430120034BD3F8800010B142
:1006E00001680A6810477047A4430120034BD3F800
:1006F000840010B101680A6810477047A4430120C4
:10070000034BD3F8880010B101680A68104770479E
:10071000A4430120034BD3F88C0010B101680A6890
:1007200010477047A4430120034BD3F8900010B149
:1007300001680A6810477047A4430120034BD3F8AF
:10074000940010B101680A6810477047A443012063
:10075000034BD3F8980010B101680A68104770473E
:10076000A4430120034BD3F89C0010B101680A6830
:1007700010477047A4430120034BD3F8A00010B1E9
:1007800001680A6810477047A4430120034BD3F85F
:10079000A40010B101680A6810477047A443012003
:1007A000034BD3F8A80010B101680A6810477047DE
:1007B000A4430120034BD3F8AC0010B101680A68D0
:1007C00010477047A4430120034BD3F8B00010B189
:1007D00001680A6810477047A4430120034BD3F80F
:1007E000B40010B101680A6810477047A4430120A3
:1007F000034BD3F8B80010B101680A68104770477E
:10080000A4430120034BD3F8BC0010B101680A686F
:1008100010477047A4430120034BD3F8C00010B128
:1008200001680A6810477047A4430120034BD3F8BE
:10083000C40010B101680A6810477047A443012042
:10084000034BD3F8C80010B101680A68104770471D
:10085000A4430120034BD3F8CC0010B101680A680F
:1008600010477047A4430120034BD3F8D00010B1C8
:1008700001680A6810477047A4430120034BD3F86E
:10088000D40010B101680A6810477047A4430120E2
:10089000034BD3F8D80010B101680A6810477047BD
:1008A000A4430120034BD3F8DC0010B101680A68AF
:1008B00010477047A4430120034BD3F8E00010B168
:1008C00001680A6810477047A4430120034BD3F81E
:1008D000E40010B101680A6810477047A443012082
:1008E000034BD3F8E80010B101680A68104770475D
:1008F000A4430120034BD3F8EC0010B101680A684F
:1009000010477047A4430120704700BF704700BFE5
:10091000F8B5D0F8C832064600F53F7500EB830005
:10092000002490F88C722A6847FA04F128469368EC
:1009300001F0010101349847042C05F10805F2D1BA
:10094000377D1549B06906EB870C4D26DCF80C2085
:10095000046806FB071E5509AB009EF8427003F1C0
:10096000604101F5614C02F01F0607F01F010122F2
:1009700044F0400402FA06F51F290460CCF8005048
:1009800009D03B064ABFC368102323F0100341F08F
:100990004007C3600760F8BD74B20100F8B50646B1
:1009A000044690F8587000252DE0042B00F0C0801C
:1009B000022B00F0B1800834A069013540B1227FDC
:1009C000032A00F09D80042A00F08F80022A7CD048
:1009D000206A6A1C38B194F82430032B69D0042BA8
:1009E0005CD0022B4CD0A06AAA1C38B194F82C1011
:1009F00003293AD004292DD0022917D00335082D18
:100A000004F1180425D0A0690028D4D0237F032B3B
:100A1000CBD147FA05F1CB07CDD496F858202A411F
:100A2000D107C8D5036819688847C4E747FA02FCAC
:100A30005FEACC71E2D596F8583043FA02F2D30758
:100A4000DCD40368196888470335082D04F11804BD
:100A5000D9D1F8BD96F85810794041FA02F3DB0776
:100A6000CCD5036819688847EEE747FA02F1C90751
:100A7000C4D496F858C04CFA02F2D207BED5E0E7CB
:100A800047FA02F1C907AED596F858C04CFA02F2FF
:100A9000D307A8D401680B689847A4E796F85830A4
:100AA0007B4043FA02F1CB079DD501680B6898475C
:100AB00099E747FA02FC5FEACC7194D496F8583073
:100AC00043FA02F2D2078ED5E4E747FA05FC5FEA63
:100AD000CC727FF57DAF96F858302B41DB073FF5A0
:100AE00077AF01680A68904772E796F85810794026
:100AF0002941C9077FF56CAF01680A68904767E72D
:100B000047FA05F2D2073FF563AF96F858302B410C
:100B1000DB077FF55DAFE4E747FA05F1CA077FF52C
:100B20004AAF96F858202A41D3073FF544AF79E7FA
:100B300096F858307B402B41D9077FF53CAF0368CE
:100B40001968884737E700BF30B48369164C027FC5
:100B500093F858302568016982B01341019503F07C
:100B60000103019A81B14468551AA54209D3A3B97A
:100B7000826895424FF0010334BF00250125457579
:100B8000037502B030BC7047002BFAD12468009482
:100B9000009D056102B030BC704700210161017504
:100BA000417502B030BC7047EC44012040680368D6
:100BB0009A68104730B44468057A69B1837A012B8A
:100BC0000DD094F85920012101FA05F022EA000520
:100BD00084F8595030BC7047437A012BF1D194F816
:100BE0005910AB400B43DDB284F8595030BC70470C
:100BF000C368DA0706D55B1041688268C858825816
:100C0000C81810474168826801EB6300104700BFB5
:100C1000C368DA0706D55B1041688268C8588258F5
:100C2000C81810474168826801EB6300104700BF95
:100C30004368074AD8B211F0FF0F52F830304FF036
:100C4000010014BF83F8800083F80001704700BFE3
:100C5000D8B6010008B5007913F030F908BD00BF1F
:100C6000C9B2007913F038B9F8B5414C2368DB07F5
:100C7000064666D53F4D404F2879012113F02CF9E7
:100C800039783C48FFF7D4FFD6F8C8423B78B569BD
:100C900006EB840283F00101D2F88C3228693970A6
:100CA0000134364F42F6AC0506EB430C0E2C795955
:100CB000ACF8CC0288BF0024C6F8C84200240A78E9
:100CC0000C704A784C70D6F8C82206EB820306F501
:100CD0003F7593F88C72286847FA04FE82680EF01C
:100CE0000101284601349047042C05F10805F2D192
:100CF000D6F8C8422249214F083451F82430002B3D
:100D00002DDB42F6AC0204330431BF5831F8131026
:100D100039801C4B357D4D2000FB053C9CF8424042
:100D200004F01F071F2F0BD0B66914F0800F16BFF9
:100D3000F068102020F0100047F04002F0603260B0
:100D4000F8BD204612F098FB0A4D002893D00E48BB
:100D5000286023212046696012F094FB8BE742F65D
:100D6000AC0500207C592278207062786070D0E752
:100D70004C14FF1F5014FF1F5814FF1F94D5002060
:100D800038FE002074B201001CA801000279034B58
:100D900053F83200012180F880107047D8B6010066
:100DA0000279034B53F83200012180F8001170479B
:100DB000D8B60100F8B54FF4FA62044600210C30B1
:100DC00014F0BAFF4FF47A72002104F2DC7014F0D0
:100DD000B3FF04F5DB50202200210C3014F0ACFFEF
:100DE0004FF4FA62002104F6C83014F0A5FF04F5B0
:100DF0009C504FF4FA620021183014F09DFF41F628
:100E0000693341F66831002201264FF0FF30632537
:100E10009FED467A6254F6EE007AE25422606260F8
:100E200084F8C42B84F8C72BA06084F8C65B84F8D0
:100E3000DC6784F8C56B84F8C36B04F10A03941C67
:100E4000551D03EE904A05EE105AD41D571CD11CB7
:100E5000101D961D06EE104A04EE101A04EE900ABC
:100E600006EE907AB8EEC52A03EE102A05EE906AD7
:100E7000B8EEC66AB0EE675AB8EEE30AF8EEE60AD4
:100E8000F8EEC32AB8EEC41AF8EEE41AF8EEE55A02
:100E9000A2EE075A0832B2F57A7FB0EE672AA6EEC4
:100EA000072AB0EE673AF0EE673AB0EE674AF0EE26
:100EB000674AF0EE676AB0EE676AA0EE073AE0EEC6
:100EC000873AA1EE074AE1EE874AE5EE876AA2EE8D
:100ED000876AFCEEC35AFCEEE32ABCEEC43AFCEE91
:100EE000E43ABCEEC54ABCEEE60AFCEEC24AFCEEB1
:100EF000C60A15EE90CA12EE90EA13EE107A13EEBF
:100F0000906A14EE105A10EE104A14EE901A10EE79
:100F1000900AA3F806C0A3F804E01F815E819D81BA
:100F2000DC81588023F8101F89D1F8BD82338342B9
:100F3000314B1B682BB193F87010C27811B9162A87
:100F40003ED0704793F8711011B9162A3CD0704703
:100F500002F1FF3C0179BCF1160FF2D801A050F864
:100F60002CF000BFEB0F0000DD0F0000430F00006E
:100F7000430F0000430F0000430F0000430F000029
:100F8000430F0000430F0000430F0000430F000019
:100F9000430F0000430F0000430F0000430F000009
:100FA000430F0000430F0000430F0000430F0000F9
:100FB000430F0000430F0000C90F0000D50F0000D1
:100FC00093F871100029C3D1012183F8701083F8C0
:100FD00071107047002083F87100704700229967F4
:100FE00083F8722083F8732070470020596783F8D4
:100FF000720083F87300704760D5002038B5437BDA
:1010000085689C1E012CEA78A97902D90223EB702D
:1010100038BD5FFA82FC5FEACC642AD45FEA4C6395
:101020002DD4CBB213F0500F044612D0A87940F063
:101030005002AA71A568A97901F0DF03AB71A0681D
:101040000222C27025690DB1606DA8470221A56812
:101050006173636D3F2B04D8581C606523442A7963
:101060001A75A97941F05003AB71A4680225E570A7
:1010700038BD1022EA705FEA4C621CD585680021F9
:101080004165816595F806C04CF02003AB7184681A
:10109000C025A57081680A79530880F85C308C7986
:1010A00044F050058D7181684222CA708468032320
:1010B000A279437338BD8568A97941F05002AA71BD
:1010C00080680224C47038BDF8B504464FF4FA6253
:1010D00000210C3004F2DC7514F02EFE4FF47A720D
:1010E0000021284614F028FE04F5DB5020220021C0
:1010F0000C3014F021FE4FF4FA62002104F6C830DF
:1011000014F01AFE04F59C504FF4FA6200211830D6
:1011100014F012FE41F6683141F6693300220126CF
:101120004FF0FF30632762549446E254114684F82E
:10113000DC672260626084F8C42B84F8C52B84F8D5
:10114000C72BA06084F8C67B04F10A0304F6C636F8
:10115000B3F802E0BEF1000F18BF8C46A6F802C03B
:1011600098884A1C002818BF9446A6F804C0DF8857
:10117000881C002F18BF8446A6F806C0B3F808E004
:10118000CA1CBEF1000F18BF9446A6F808C05F89BC
:10119000081D002F18BF8446A6F80AC0B3F80CE05B
:1011A0004A1DBEF1000F18BF9446A6F80CC0DF8997
:1011B000881D002F18BF8446A6F80EC033F810EF24
:1011C000CA1D0831BEF1000F18BF9446B1F57A7FF1
:1011D00026F810CFBCD104F5DB5440F2E73C0834CC
:1011E000614635F8023C002B18BF8C4624F802CC2F
:1011F00035F8046C4F1E002E18BFBC4624F804CCF2
:1012000035F8060CA1F1020E002818BFF44624F8A8
:1012100006CC35F8083CCA1E002B18BF944624F8AB
:1012200008CC35F80A6C0F1F002E18BFBC4624F8F6
:101230000ACC35F80C0C4B1F002818BF9C4624F82C
:101240000CCC35F80E6CA1F1060E002E18BFF4463A
:1012500024F80ECC35F8107DCA1F0839002F18BFAE
:1012600094464A1C24F810CDBBD1F8BD2DE9F04FAF
:101270004FF49673ADF5057D03FB00F3794F0193B1
:10128000DFF824A2DFF8F4B1774E02910133039224
:101290000093B946DAF80080744D12F059FE044606
:1012A00004E012F055FE031BAB42F3D83068C307CD
:1012B000F7D46F4A6F49C2F80080516012F048FEBF
:1012C0006A4C054604E012F043FE411BA142E1D8FE
:1012D0003868694B0340002BF5D0D9F80010CBF8E3
:1012E0000010C9F80010DBF80020634D6349154079
:1012F000012DCFD1624C2068C005CBD500230B60F7
:101300006049614C614A0E78257004AD15603EBBA2
:10131000009F7802564A5E4D5E4B5F4E5F4F1060F5
:101320004FF48131296016631F6012F011FE4F4E99
:10133000054604E012F00CFE411BB14212D82078A1
:101340000028F7D1DBF80020534B1340022B09D1C2
:10135000049F7B1C13D001200DF5057DBDE8F08FA7
:101360000098D7E74FF4F47231214D4811F054FE44
:101370000028EDD106200DF5057DBDE8F08FDFF8E2
:10138000E480394FDAF80090384E12F0E1FD05465E
:1013900004E012F0DDFD401BB042F3D83868C2070C
:1013A000F7D4334A334BC2F80090536012F0D0FDAB
:1013B0002E4D064604E012F0CBFD821BAA42E1D876
:1013C000D8F800102C4808400028F4D0254B254AB6
:1013D0001E68CBF800601660DBF8005026482749ED
:1013E00028400128CED1264B1E68F305CAD500221D
:1013F0000A602449254D019A0F78207003982860CF
:10140000023207B95202029B194D264821492A602F
:101410005E0A013637041E4E204A47F400731E4F01
:10142000336007600A6012F093FD104E054604E039
:1014300012F08EFD431BB3420AD820780028F7D162
:10144000DBF8004014492140022901D1002083E744
:101450004FF4F4723121124811F0DEFD002889D0DA
:10146000F4E700BF30100B4024100B4040420F0047
:1014700008100B4000001A0D01000F00D04401209D
:1014800010100B40C4440120D444012000100B4034
:1014900004100B400C100B4002007F1137003A1271
:1014A0004CFF002038100B40D84401202DE9F04FAC
:1014B0004FF49673ADF5057D03FB00F3794F03926E
:1014C0001A464FF0FF340132DFF81CA2DFF8ECB10E
:1014D000754E0193029100920494B946DAF80080A7
:1014E000724D12F035FD044604E012F031FD031B8D
:1014F000AB42F3D83168CB07F7D46D486D4BC0F8D9
:101500000080436012F024FD684C054604E012F0B0
:101510001FFD411BA142E1D83A68674911400029EB
:10152000F5D0D9F80030CBF80030C9F80030DBF83E
:101530000000614D614C0540012DCFD1604A11681A
:10154000C805CBD5002323605E4C5F4F5F482678EB
:101550003D7004AD0560002E40F08C80009A500272
:10156000534D5B495B4B5C4A5C4E28604FF48134C1
:101570000C602E631A6012F0EBFC4C4D044604E044
:1015800012F0E6FC061BAE4276D838780028F7D178
:10159000DBF80010514B0B40022B6DD1DFF80481BA
:1015A000414EDAF80090414D12F0D2FC044604E0BE
:1015B00012F0CEFC001BA842F3D83268D207F7D451
:1015C0003B493C48C1F80090486012F0C1FC374CE0
:1015D000054604E012F0BCFC421BA242E1D8D8F858
:1015E0000020354B1340002BF4D02E482D4D0168C0
:1015F000CBF800102960DBF800402F4A2F4822402A
:10160000012ACED12E4B1968CB05CAD5002404601F
:101610002E4D2C483A70039A2A600678019A0232BD
:1016200006B95202029B224C294D2D482260590ACC
:1016300001310E042749284A46F40073274E2B60D7
:1016400006600A6012F084FC184D044604E012F0B3
:101650007FFC031BAB421CD838780028F7D1DBF89D
:1016600000701E493940022913D100200DF5057D77
:10167000BDE8F08F009873E74FF4027233211948E8
:1016800011F0CAFC002889D106200DF5057DBDE8C2
:10169000F08F4FF402723321124811F0BDFC002884
:1016A000F2D0E2E730100B4024100B4040420F0014
:1016B00008100B4000001A0D01000F00D04401205B
:1016C00010100B40C4440120D444012000100B40F2
:1016D00004100B400C100B4027003A1902007F1138
:1016E00038100B404CFF0020D8440120234B10B48D
:1016F0005A6811685068097892F809C00478137A1A
:1017000014EA0C0F01EA03011DD0947A04F00300DF
:1017100009B140F0040040F00803991003F1FF3CC8
:101720009172BCF10D0F0BD8DFE80CF021071B07FD
:101730000A152121150A071B0721D1684B1ED3600A
:101740005DF8044B7047907A00F003030029E4D061
:1017500043F00403E1E7D3689C1ED4605DF8044BBA
:101760007047D0685DF8044B0230D0607047D46891
:101770000134D4605DF8044B704700BF9C420120E7
:10178000234B10B49A6811685068097892F809C020
:101790000478137A14EA0C0F01EA03011DD0947A3D
:1017A00004F0030009B140F0040040F00803991070
:1017B00003F1FF3C9172BCF10D0F0BD8DFE80CF088
:1017C00021071B070A152121150A071B0721D168CC
:1017D0004B1ED3605DF8044B7047907A00F0030312
:1017E0000029E4D043F00403E1E7D3689C1ED460F1
:1017F0005DF8044B7047D0685DF8044B0230D06050
:101800007047D4680134D4605DF8044B704700BF62
:101810009C420120234B10B4DA68116850680978A3
:1018200092F809C00478137A14EA0C0F01EA030154
:101830001DD0947A04F0030009B140F0040040F098
:101840000803991003F1FF3C9172BCF10D0F0BD806
:10185000DFE80CF021071B070A152121150A071BD9
:101860000721D1684B1ED3605DF8044B7047907A16
:1018700000F003030029E4D043F00403E1E7D36858
:101880009C1ED4605DF8044B7047D0685DF8044B33
:101890000230D0607047D4680134D4605DF8044BE6
:1018A000704700BF9C4201202DE9F04F002A9DF8AF
:1018B000244070DB002B6EDBFF286CDC3F296ADCE8
:1018C000FF2AA8BFFF2220EAE07E3F2BA8BF3F23CC
:1018D000724521EAE17998465DDB5F1CC9EB0700A0
:1018E000DFF8B8C002F1010A07024FEA092BC84528
:1018F0004BDB0EEB0B024FF48073A7F58071BB42FC
:101900000CF80240C1F3022562443ED01DB3012D04
:101910001CD0022D17D0032D12D0042D0DD0052D73
:1019200008D0062D1CBF4FF4007382F80041D45438
:1019300003F58073D45403F58073D45403F5807396
:10194000D45403F58073D45403F58073D45403F551
:101950008073BB4219D003F5807103F5007603F55F
:101960004075D45403F580605454945503F5A06138
:10197000545503F5C06603F5E06503F50063BB420B
:101980001454545494555455E5D10EF1010ED645D6
:10199000ADD1BDE8F08FBDE8F08F00BF9802012007
:1019A0002DE9F04F002A9DF8244071DB002B6FDBFE
:1019B000FF286DDC3F296BDCFF2AA8BFFF2220EA4D
:1019C000E0773F2BA8BF3F23BA42944621EAE17E4D
:1019D0005EDBCEEB0306700801302E4A46024FEA6A
:1019E0000E2873454FDB07EB08004FF40071A6F596
:1019F00000758E421454C5F34225104443D01DB3E4
:101A0000012D1CD0022D17D0032D12D0042D0DD086
:101A1000052D08D0062D1CBF4FF4806180F80042D0
:101A2000445401F50071445401F50071445401F52A
:101A30000071445401F50071445401F5007144549F
:101A400001F500718E421ED001F5007501F5806B25
:101A500001F5C06A445401F50069445500F80B4093
:101A600001F5206500F80A4001F5406B01F5606A58
:101A700001F580518E4200F80940445500F80B40B2
:101A800000F80A40E0D10237BC45AADABDE8F08F81
:101A9000BDE8F08F98020120F6EE007A30EE270ABA
:101AA00070EEA70ABDEEC07A70B417EE103AFF2BA5
:101AB00031EE271A71EEA71ABDEEE06A04D816EED1
:101AC000102A3F2A40F24B82BDEEC12AFDEEE12AE8
:101AD00012EE104AFF2C12EE901A02D83F2940F263
:101AE000388231EE403A71EEE03AF0EEC36AF0EE41
:101AF000E35AF4EEE56AF1EE10FAC0F21781DFED79
:101B0000894AF4EEE46AF1EE10FA00F10881B4EECD
:101B1000C10AF1EE10FA00F32782F0EE432A1A46CA
:101B2000944283EEA23A40F3FA80D1432144FF2A43
:101B300001F007037C4E08D8FDEEE03A13EE905A10
:101B40003F2D9CBF06EB0525A8540132A24270EE42
:101B5000830A00F0E480002B6FD0012B5DD0022BB4
:101B60004DD0032B3DD0042B2DD0052B1DD0062BA3
:101B70000DD0FF2A08D8FDEEE06A16EE901A3F2934
:101B80009CBF06EB0121885470EE830A0132FF2AC4
:101B900008D8FDEEE05A15EE903A3F2B9CBF06EBBD
:101BA0000323985470EE830A0132FF2A08D8BDEE51
:101BB000E04A14EE105A3F2D9CBF06EB0525A854B1
:101BC00070EE830A0132FF2A08D8BDEEE05A15EE06
:101BD000101A3F299CBF06EB0121885470EE830A3E
:101BE0000132FF2A08D8FDEEE07A17EE903A3F2B3B
:101BF0009CBF06EB0323985470EE830A0132FF2A40
:101C000008D8BDEEE07A17EE105A3F2D9CBF06EBC8
:101C10000525A85470EE830A0132FF2A08D8BDEECC
:101C2000E01A11EE101A3F299CBF06EB01218854DF
:101C30000132A24270EE830A71D0FF2A08D8FDEE6D
:101C4000E01A11EE903A3F2B9CBF06EB0323985409
:101C50000132FF2A70EE830A08D8BDEEE06A16EE64
:101C6000105A3F2D9CBF06EB0525A854511CFF2997
:101C700030EE832A08D8BDEEC20A10EE103A3F2B90
:101C80009CBF06EB03235854911CFF2972EE034AB4
:101C900008D8FDEEE42A12EE905A3F2D9CBF06EBC9
:101CA00005256854D31CFF2B74EE833A08D8FDEE4B
:101CB000E36A16EE901A3F299CBF06EB0121C85437
:101CC000131DFF2B73EE835A08D8BDEEE54A14EEC0
:101CD000105A3F2D9CBF06EB0525E854511DFF29E6
:101CE00035EE835A08D8FDEEC57A17EE903A3F2BB1
:101CF0009CBF06EB03235854911DFF2935EE037A50
:101D000008D8BDEEC71A11EE105A3F2D9CBF06EB46
:101D1000052568540732A24277EE030A8DD170BCC4
:101D2000704700BFACC5273798020120F4EEE10AE6
:101D3000F1EE10FA00F3038116EE103AB0EE434ACA
:101D40008B42C4EE234AEADADD430D4405F0070274
:101D50008A4CBDEEC05A15EE105AFF2D04D83F2B09
:101D60009CBF04EB0326705501338B4230EE240AEE
:101D7000D5D0002A70D0012A5DD0022A4DD0032A86
:101D80003DD0042A2DD0052A1DD0062A0DD0FDEE07
:101D9000C07A17EE906AFF2E04D83F2B9CBF04EB4D
:101DA0000325A85530EE240A0133FDEEC00A10EEDB
:101DB000902AFF2A04D83F2B9CBF04EB0325A8548C
:101DC00030EE240A0133BDEEC07A17EE106AFF2E02
:101DD00004D83F2B9CBF04EB0325A85530EE240A02
:101DE0000133BDEEC01A11EE102AFF2A04D83F2B92
:101DF0009CBF04EB0325A85430EE240A0133FDEE0A
:101E0000C01A11EE906AFF2E04D83F2B9CBF04EB42
:101E10000325A85530EE240A0133BDEEC06A16EE44
:101E2000102AFF2A04D83F2B9CBF04EB0325A8549B
:101E300030EE240A0133BDEEC02A12EE106AFF2EE6
:101E400004D83F2B9CBF04EB0325A85501338B42DC
:101E500030EE240A3FF463AFFDEEC02A12EE902A62
:101E6000FF2A04D83F2B9CBF04EB0325A85430EE77
:101E7000240A0133BDEEC03A13EE106AFF2E04D8D7
:101E80003F2B9CBF04EB0325A85570EE243A5D1C44
:101E9000FDEEE36A16EE902AFF2A04D83F2D9CBF80
:101EA00004EB0525A85473EEA45A9E1CBDEEE54A2A
:101EB00014EE105AFF2D04D83F2E9CBF04EB0626CB
:101EC000705535EEA45ADE1CFDEEC57A17EE902A49
:101ED000FF2A04D83F2E9CBF04EB0626B05475EEB3
:101EE000240A1D1DBDEEE07A17EE106AFF2E04D8FD
:101EF0003F2D9CBF04EB0525A85530EEA41A5D1DAF
:101F0000FDEEC11A11EE902AFF2A04D83F2D9CBF86
:101F100004EB0525A85431EE246A9D1DBDEEC62AAA
:101F200012EE106AFF2E04D83F2D9CBF04EB05254E
:101F3000A85507338B4236EE240A8DD1EFE630EEFA
:101F4000414A0B4670EEE13AB0EE410A16EE101A25
:101F5000F6E60A4A02EB012C0CF80400C1E5074C36
:101F600004EB0225E854AFE570EEE13A224670EE4C
:101F7000412A1C46F0EE610AD2E500BF980201201A
:101F80002DE9F04F854B854ADD6A196854689BB08E
:101F9000002D1191064640F38181032D57DC304618
:101FA00013F06EFF3278002A5AD000284FF0000E4E
:101FB000ACBF07466FF00047F44606F1FF3801203A
:101FC00018F8013F33B99FB918F8013F4FF0FF37B8
:101FD000002BF8D00A2B04D01F2BF1D90EF1060EDE
:101FE000EEE7F445B8BFF44601304FF0000EE7E7E6
:101FF0006A4FB96A083100FB01F06849F44505FBF6
:1020000000F7C8686346B8BF734605FB03F30128B1
:1020100016932CD0022800F04481604B19690129E5
:1020200030D0022908BFE41B5C4BDFF870B1D3F855
:1020300018E0196A119B01EB0E0843459C4603DA30
:1020400016998C44E64522DB1BB0BDE8F08F53485F
:102050000325C562304613F013FF3278002AA4D15D
:102060004E491692C86801284FEAC507D2D1169981
:10207000119B01EBD179A3EB6901484B11911969CF
:102080000129CED107EBD77AA4EB6A04CCE7DBF8C1
:102090001CE0DBF8243073449C42D5DA2744BE456B
:1020A000D2DA002AD0D00996CDF864B00A2A099F66
:1020B00000F0DB853E461346002102E00A2B00F0CB
:1020C000A0831F2B16F8013F88BF0131002BF5D1EB
:1020D00001EB410E4FEA4E01179605FB01FE2F4E14
:1020E000B76A083705FB07F90128A9EBC50600F018
:1020F0009283022800F0B185119806902749087D47
:10210000002840F0D38009EB04032644022D0E93EF
:10211000109600F08A83032D40F0FF80002A00F023
:10212000AE810A2A00F0AB811C4E109D1B4C316A17
:10213000776AD6F81890D6F81CB0207A0290203A28
:102140002E02D3B2A81C09EB010A01350BEB0701E3
:102150006B2B06F1020703910A970C900B9500F286
:1021600026830F4E56F823703E78069C0A990D4D33
:10217000059701EB04080022A11C631CDDF830E088
:10218000DDF82CC0109F0492A844079308910846DC
:10219000224607994446002335E000BF64D500205D
:1021A00018AC010098020120814500F3738182453B
:1021B00040F37081894540F34782BB4505DC039DB0
:1021C000BD42C4BF9DF808502570E34506DC039D61
:1021D000654503DD9DF8085084F80051F34506DCA1
:1021E000039D754503DD9DF8085084F800520133C6
:1021F000062B02F1030204F1030401F1030100F1D3
:10220000030000F0678146FA03F5ED07EFD591452D
:10221000CADC824500F37381814540F3968189458C
:1022200000F37281924540F30582BB4500F3898239
:10223000039DBD4240F385829DF8085004F8025C7E
:102240008A4506DD9DF8085004F8015C924540F38C
:10225000E381E34500F3E081039D654540F3DC81C4
:102260009DF8085084F8FE508A4540F3AE829DF8F0
:10227000085084F8FF50924540F32481F345B6DCC2
:10228000039D7545B3DD9DF8085084F8FE518A45DD
:10229000ADDD9DF8085084F8FF51A8E70125D5620F
:1022A0007DE6119B16995B1A1193B6E6199A517D3A
:1022B0009069D2F81CA0136A576A0091069909EB3D
:1022C00004028946F14400EB030E0E920EF1FF3832
:1022D00009F1FF3242450AEB070B0E9FA8BF4246A9
:1022E0008842B8BF08460BF1FF3307F1FF3CA24517
:1022F0005146B8BF21466345A8BF6346FFF7D4FAED
:102300003019099E1090022D327800F08E82032D34
:102310003FF404AF002A00F0B2800A2A00F0AF8038
:10232000B94DB94FD5F81CB0387A6B6A109FA969BE
:102330002E6A069D07905B44380205350E440593CE
:1023400006900837A2F1200A5FFA8AF36B2B96BF3A
:10235000AE4AAF4C52F82340069AAE4B0395501943
:10236000013C05F1FF3E109ACDF810E01844A5F1AC
:10237000050AA5F10409A5F10308A5F1020C0294D0
:10238000029D15F8013F0295DC070FD551450DDC84
:1023900056450BDD934509DC059C944206DD039D03
:1023A000441B9DF81C5004F80A50A6469D070FD503
:1023B00049450DDC4E450BDD934509DC059C9442F7
:1023C00006DD039D441B9DF81C5004F80950A646E9
:1023D0005C070FD541450DDC46450BDD934509DC17
:1023E000059C944206DD039D441B9DF81C5004F897
:1023F0000850A6461D070FD58C450DDBB4450BDAFA
:10240000934509DC059C944206DD039D441B9DF821
:102410001C5004F80C50A646DC0611D5049DA942B8
:102420002C460DDCAE420BDD934509DC059C944245
:1024300006DD039C041BA6469DF81C400EF80540D3
:102440009B060CD5039B994209DC9E4207DD934510
:1024500005DC059D9542C4BF9DF81C5005700132F6
:10246000974200F580708BD1099B039D13F8012FD3
:10247000099322B10A2A05F106057FF463AF179E7E
:102480000E9C3278002A3FF4DFAD5F490996CD6A91
:10249000C8680BE689453FF7AAAE8A457FF7A7AE25
:1024A000BB4506DC039DBD4203DD9DF8085004F8E2
:1024B000015CE34506DC039D654503DD9DF808509E
:1024C00084F8FF50F3453FF792AE039D75453FF703
:1024D000E0AE8CE6049E0336182E049608F540788C
:1024E0000EF1030E07F103070CF1030C00F04D8110
:1024F0000598069A10F8016F0590089849E68145FD
:1025000051DD4945BFF68EAE92457FF770AEBB45B3
:1025100006DC039DBD4203DD9DF8085004F8025C13
:10252000E34506DC039D654503DD9DF8085084F80E
:10253000FE50F3453FF75BAE039D75457FF757AE01
:102540009DF8085084F8FE5151E68945DCDC92453F
:1025500040F34281BB4500F34A81039DBD4240F3F5
:1025600046819DF8085004F8025C8A4506DD9DF816
:10257000085004F8015C924540F31C81E34500F3E8
:102580001981039D654540F315819DF8085084F835
:10259000FE508A4540F32E819DF8085084F8FF5084
:1025A00092458FDD6AE68A457ADC924540F3D98010
:1025B000BB450CDC039DBD4209DD9DF8085004F8C5
:1025C000025C9DF808502570924540F3D080E345A9
:1025D0000DDC039D65450ADD9DF8085084F8FE502A
:1025E0009DF8085084F8005192457FF7F7ADF34508
:1025F0003FF7FDAD039D75457FF7F9AD9DF8085098
:1026000084F8FE51EFE500BF64D5002018AC01004E
:10261000DCAD0100980201208A4507DDE3453FF764
:102620002AAE039D65457FF726AE20E692457FF7EB
:10263000DEAD23E68A45F9DDBB453FF707AE039DD6
:10264000BD427FF703AEFDE58A457EDDBB450BDC71
:10265000039DBD4208DD9DF8085004F8015C9DF81B
:10266000085025708A4575DDE3450DDC039D654501
:102670000ADD9DF8085084F8FF509DF8085084F852
:1026800000518A457FF7AAADF3453FF7B0AD039DF2
:1026900075457FF7ACAD9DF8085084F8FF51A2E571
:1026A000924542DDBB4540DC039DBD423DDD9DF8CA
:1026B000085004F8025C89453EDD039DBD4202DD01
:1026C0009DF80850257092451FDDE3451DDC039DF4
:1026D00065451ADD9DF8085084F8FE5089451BDDDC
:1026E000039D654503DD9DF8085084F8005192452F
:1026F00017DDF34515DC039D754512DD9DF8085087
:1027000084F8FE518945C6DD6AE5894537DCE34535
:10271000EDDC039D6545EADD9DF8085084F8FF5027
:10272000E1E789453FF75AADAEE789452ADCBB456D
:10273000C9DC039DBD42C6DD9DF8085004F8015C6C
:10274000BEE78A453FF778AF83E5BB4502DC039DD2
:10275000BD4284DCE3453FF741AD039D65458CDC1C
:102760003CE5BB4503DC039DBD423FF72AAFE34593
:102770003FF734AD039D65453FF732AF2EE5E345A6
:10278000B5DCADE7BB459EDC97E70999069B11F8E0
:10279000012F099112330693002A3FF470AE0A2AE2
:1027A0003FF46DAE203AD3B26B2B7FF6DAAC9B4F81
:1027B0000026DAE48A457FF739AFE3453FF7F0AE0C
:1027C000039D65457FF7ECAEE6E692453FF756ADD3
:1027D0008A453FF777AE0AE58A457FF727AFBB45C5
:1027E0003FF7C9AE039DBD427FF7C5AEBFE68A4540
:1027F000F5DCC3E692453FF741AD8A457FF7F7AC7C
:1028000060E601EB41077B00179605FB03FE3746A8
:102810000137179763E41698119BCEEB000A0AEB79
:10282000DA7B03EB6B07069768E4002A3FF427AED8
:102830000A2A3FF424AE7A4F069B796AFE693D6A04
:10284000BC69774898465F1C06EB010A0B3341468A
:10285000093104EB050B0F934546434690F8089069
:102860000C910A35591D4046083003970D95DF1D20
:102870009D1D0691203A109904900B97181DDF1C9E
:102880000A95C8469D1C9946D3B201316B2B08901E
:1028900007970595189100F24281624850F823701D
:1028A0003978109A189B029700208CE0CD0711D53B
:1028B000039DA542C0F29F81A14580F2E3815D4561
:1028C00008DAB34206DB534504DA574F07EB032C13
:1028D0000CF805808D0713D5079D059FAC4200F3CA
:1028E0007581BC4240F3C881079DAB4508DD9E421F
:1028F00006DC9A4504DD4C4F07EB032C0CF80580F1
:102900004F0713D5069D089FAC4200F30B81BC42D4
:1029100040F3BB81069DAB4508DD9E4206DC9A452F
:1029200004DD414F07EB032C0CF805800D0713D590
:102930000B9D0A9FA542C0F20A81BC4240F3A981C7
:102940000B9D5D4508DA9E4206DC9A4504DD364F54
:1029500007EB032C0CF80580CF0613D50C9D049FC4
:10296000AC4200F30981BC4240F397810C9DAB451A
:1029700008DD9E4206DC9A4504DD2B4F07EB032C55
:102980000CF805808D0613D50F990D9DA142C0F25C
:102990000881AC4240F36D810F9F5F4508DA9E428B
:1029A00006DC9A4504DD204901EB032505F8078084
:1029B0000130082802F1020203F102037DD0029FD8
:1029C00017F8011F029796423FF770AF924513DC4C
:1029D000CF077FF57FAF039DA542C0F22A81A145B5
:1029E00080F24D815D45BFF675AF9E423FF772AFF5
:1029F0009A457FF76FAF68E70B4DDDF80CC0CDF857
:102A0000509005EB0227084D129705EB032513950F
:102A1000CE460027029D159222E000BFDCAD0100EA
:102A200064D5002018AC010098020120DE4502DACE
:102A3000129A02F80E8064451BDDDE4509DA9E42DB
:102A400004DC9A45C4BF139A02F80E80644540F333
:102A5000EC800137062F0CF1020C0EF1020E21D092
:102A600041FA07F919F0010FF3D0A645DEDA644503
:102A7000EFDCE34540F3D380129AA64502F80C80C0
:102A800080F2D0809E42E4DC9A45C8BF139A07F1D9
:102A90000107C8BF02F80C80062F0CF1020C0EF1E2
:102AA000020EDDD1159ADDF850900295013008280C
:102AB00002F1020203F1020381D1099810F8012FFB
:102AC000099009F10C09002A3FF4D9AC039B0F9936
:102AD0000D9D0C9F04980C3303930B9B0C310C350C
:102AE0000C370C300C330F910D950A99069D0C97FD
:102AF0000490089F07980B93059B0C310C350C37FD
:102B00000C300C330A2A0A91069508970790059312
:102B10003FF4B5AC203AD3B26B2B7FF6BEAE614F1B
:102B20000021BEE6BC423FF701AFBB457FF7FEAEDA
:102B30009E4207DC9A4505DD5B4D089F05EB032CA3
:102B40000CF80780069DAC423FF7F0AEE2E6BC42CF
:102B50003FF702AFBB457FF7FFAE9E4207DC9A45C9
:102B600005DD514D0A9F05EB032C0CF807800B9DEA
:102B7000A542FFF6F1AEE3E6BC423FF703AFBB452B
:102B80007FF700AF9E4207DC9A4505DD464D049F66
:102B900005EB032C0CF807800C9DAC423FF7F2AE1E
:102BA000E4E6AC423FF704AFAB457FF701AF9E428E
:102BB00007DC9A4505DD3C4F0D9907EB032C0CF81B
:102BC00001800F9DA542FFF6F3AEE5E6BC423FF75C
:102BD00097AEBB457FF794AE9E4207DC9A4505DD74
:102BE000314D059F05EB032C0CF80780079DAC4287
:102BF0003FF786AE78E6A145FFF66CAED945BFF645
:102C000069AE9E4206DC9A4504DD274F07EB032C94
:102C10000CF80980039DA542FFF65CAE4FE6A64581
:102C2000FFF617AFDE45FFF60AAFE3453FF72AAFE1
:102C30000FE7A145FFF64EAED945BFF64BAE9E421B
:102C400006DC9A4504DD184D05EB032707F80980DB
:102C5000039DA542FFF63EAEC4E6169B1199CEEB4E
:102C600003070F440697FFF749BA17974FF0000E76
:102C7000CEE5AB459BDC8FE6BB45ADDC34E6D94504
:102C8000DDDBAFE6D945BCDB19E6BB453FF750AF0E
:102C900040E6BB453FF761AF52E6BB453FF772AF39
:102CA00064E600BFDCAD01009802012091420B46B2
:102CB000A8BF1346002BC0F2C981531A002BB8BF1E
:102CC0005B42012B40F3D48191422DE9F04700F3A0
:102CD000A1810029C0F2A481B2F57A7F00EB410501
:102CE00001F1010680F2BB81AF8990F8C5AB07EE18
:102CF000907AF8EE676ABAF1000F00F0A18100EB5C
:102D00004208541AB8F80C9007EE109A01EE104AD7
:102D1000F8EEC70AB8EEC16A70EEE61AB24281EE6A
:102D2000860A40F3A38100EB4603F54306F1010C4C
:102D30000A331544624505F0070676EE806AB6EE62
:102D4000002A76EE822ABCEEE23A13EE107A23F8DD
:102D5000027F40F3B380002E61D0012E51D0022EAD
:102D600043D0032E35D0042E27D0052E19D0062EA1
:102D70000BD076EE806A0CF1010C76EE823ABCEE56
:102D8000E34A14EE101A23F8021F76EE806A0CF163
:102D9000010C76EE824ABCEEE45A15EE104A23F896
:102DA000024F76EE806A0CF1010C76EE825AFCEE50
:102DB000E57A17EE905A23F8025F76EE806A0CF1FE
:102DC000010C36EE827AFCEEC70A10EE906A23F808
:102DD000026F76EE806A0CF1010C36EE821ABCEEC0
:102DE000C16A16EE107A23F8027F76EE806A0CF143
:102DF000010C76EE821AFCEEE12A12EE908A23F89C
:102E0000028F76EE806A0CF1010C36EE823A624552
:102E1000FCEEC33A13EE909A23F8029F4EDD36EE95
:102E2000804A0CF1080C74EE004A74EE027A74EEDB
:102E3000805A34EE827A35EE805A75EE820A35EE8B
:102E4000001A35EE026A71EE001A71EE022A31EEB6
:102E5000803A31EE824A73EE006A73EE023A76EE01
:102E6000824AFCEEE35ABCEEE45ABCEEC41AFCEE15
:102E7000E21ABCEEC66AFCEEE00ABCEEC77AFCEED3
:102E8000E77A15EE90EA15EE108A11EE107A11EE3F
:102E9000906A16EE105A10EE904A17EE101A17EEBE
:102EA000909A6245A3F80EE09F815E811D81DC80CF
:102EB0009980A3F8029023F8108FB0DCBAF1000FCC
:102EC00040F0D48000231E4600F10A0E00F6C63AF8
:102ED000BEF80220002A18BF3346AAF80230BEF816
:102EE0000470751C002F18BF2B46AAF80430BEF8DA
:102EF0000640B11C002C0CBF1F460F46AAF80670F6
:102F0000BEF80850F21C002D0CBF3C461446AAF82F
:102F10000840BEF80AC0331DBCF1000F0CBF2146AB
:102F20001946AAF80A10BEF80C70751D002F0CBFC8
:102F30000C462C46AAF80C40BEF80E80B21DB8F123
:102F4000000F0CBF27461746AAF80E703EF8109FD8
:102F5000F31D0836B9F1000F08BF3B46B6F57A7F7E
:102F60002AF8103FB4D100F5DB5640F2E7390836B5
:102F700000F2DC7A4D463AF8020C002818BFA94648
:102F800026F8029C3AF8041C6C1E00290CBFCC46A3
:102F9000A44626F804CC3AF8062CA5F1020E002A25
:102FA0000CBF6746774626F8067C3AF8083CE81ED0
:102FB000002B0CBFB846804626F8088C3AF80A9CCD
:102FC000291FB9F1000F0CBF44460C4626F80A4CE5
:102FD0003AF80CCC6A1FBCF1000F0CBF274617460D
:102FE00026F80C7C3AF80E0CAB1F00280CBF3C46B0
:102FF0001C4626F80E4C3AF8108DA5F10709083D3D
:10300000B8F1000F08BFA1466A1C26F8109DB2D186
:10301000BDE8F0870C46114600292246BFF65CAE9B
:1030200000EB420190F8C5AB8F89878107EE907A5B
:1030300001260021F8EE676ABAF1000F7FF45FAE57
:10304000B2427FF73FAF9FED0B0A6CE691428C4690
:10305000B8BF9446BCF57A7FFFF62FAE7047AA89B9
:10306000A0F8DA27AF8940F2E7323EE6BDE8F08704
:10307000704700BF00000000F0B40B4640F2E73795
:1030800006E095F8DC570DB1012E13D1994211D00D
:103090009B1812D4B3F57A7F17DB00231E46012458
:1030A0000546044494F8DC47002CEAD195F8DC6727
:1030B000002EEBD01846F0BC704740F2E733C5183D
:1030C00095F8DC67002EE1D0F4E733B1C518BB42B8
:1030D00095F8DB67EAD05C1CE3E701241E46054651
:1030E000DFE700BFD0ED017A9FEDBD6ADFEDBD6A7D
:1030F000B8EEE77AB6EE000AA7EE060A2DE9F04729
:10310000FDEEC00A0668B8EEE01A831961EE261AD1
:1031100000EB4605BDEEE12A012212EE104A06F24E
:10312000DC7116F0070783F8DC2700EB0103324659
:10313000AC814DD0721E00F19684B2F57A7F80F298
:10314000BA8413F8015D002D40F09280012F3FD02A
:10315000022F34D0032F29D0042F1ED0052F13D0D7
:10316000062F08D0013AB2F57A7F80F2A48413F8D2
:10317000014D002C7CD1013AB2F57A7F80F29B841C
:1031800013F8017D002F73D1013AB2F57A7F80F2F6
:10319000928413F8015D002D6AD1013AB2F57A7F6D
:1031A00080F2898413F8014D002C61D1013AB2F507
:1031B0007A7F80F2808413F8017D002F58D1013A84
:1031C000B2F57A7F80F2778413F8015D002D4FD13C
:1031D000013A002A9046C0F24684B2F57A7F80F226
:1031E0006A8413F8014C03F1FF39002C40D1013AF5
:1031F000B2F57A7F80F25F8419F8017CC7BBA8F131
:103200000202B2F57A7F80F2568413F8035C7DBB2C
:10321000A8F10302B2F57A7F80F24D8413F8043CE2
:1032200033BBA8F10402B2F57A7F80F2448419F826
:10323000044CECB9A8F10502B2F57A7F80F23B8428
:1032400019F8057CA7B9A8F10602B2F57A7F80F2D9
:10325000328419F8065C5DB9A8F10702B2F57A7FED
:1032600080F2298419F8074CA9F10703002CAFD08C
:10327000C6F579750335431815F0070137463FD079
:10328000771C00F1F383B7F57A7F80F2188413F886
:10329000014F002C65D1012932D002292AD00329FF
:1032A00021D0042918D005290FD0062906D00137CE
:1032B00000F1DC8313F8015F002D52D1013700F1DA
:1032C000D58313F8011F00294BD1013700F1CE83BC
:1032D00013F8014F002C44D1013700F1C78313F8D4
:1032E000015F002D3DD1013700F1C08313F8011FAC
:1032F000002936D1013700F1B98313F8014F84BB9F
:103300000137002F3946C0F2B183B7F57A7F80F2DA
:10331000D6835D785C1C25BB013700F1A7836578F7
:10332000FDB98F1C00F1A283DD78D5B9CF1C00F167
:103330009D831B79ABB90F1D00F19883257985B961
:103340004F1D00F1938363795BB98F1D00F18E836C
:10335000A57935B9CF1D00F18983E179E31D0029F5
:10336000CED096423446A8BF1446002CC0F28783C4
:10337000B51A85EAE571A1EBE573012B40F3A9814C
:103380009642AABF154635463246002DC0F2BB8391
:10339000B2F57A7F00EB450C05F1010880F29B83C2
:1033A000BCF80C4090F8C59B02EE904AB8EE623A29
:1033B000B9F1000F00F0A18300EB4203551B99897E
:1033C00003EE901A04EE905AB8EEE34AB8EEE45ACF
:1033D00074EE435A4245C5EE857A40F37A8103E0A4
:1033E000FA007A3CEC11834200EB48036FEA080CC8
:1033F0000A3308F10108944442450CF0070573EEC6
:10340000276AB6EE007A36EE876ABCEEC60A10EE80
:10341000104A23F8024F40F3B380002D61D0012DF4
:1034200051D0022D43D0032D35D0042D27D0052DAA
:1034300019D0062D0BD076EEA76A08F1010876EEBA
:10344000870ABCEEE01A11EE10AA23F802AF76EE5E
:10345000A76A08F1010876EE871ABCEEE12A12EE9F
:10346000101A23F8021F76EEA76A08F1010876EE1B
:10347000872ABCEEE23A13EE105A23F8025F76EE8A
:10348000A76A08F1010876EE873ABCEEE34A14EE2B
:10349000104A23F8024F76EEA76A08F1010876EE8B
:1034A000874ABCEEE45A15EE10CA23F802CF76EE36
:1034B000A76A08F1010876EE875ABCEEE56A16EEB7
:1034C00010AA23F802AF76EEA76A08F1010836EEDB
:1034D000870A4245FCEEC00A10EE901A23F8021F3C
:1034E0004EDD36EEA71A08F1080871EE271A31EE04
:1034F000072A71EEA72A31EE873A32EEA74A72EE1A
:10350000874A74EE273A34EE076A73EEA75A33EE11
:10351000870A35EEA75A75EE870A75EE276A35EEEB
:10352000071A76EE871AFCEEC12AFCEEE03A12EE9C
:10353000901A13EE904ABCEEE14AFCEEC05ABCEE83
:10354000C66AFCEEE44ABCEEC33ABCEEC22AD9819C
:103550009C8114EE10AA15EE90CA16EE10EA14EE35
:10356000905A13EE101A12EE104A4245A3F80AC000
:10357000A3F808E0DD8099805C8023F810AFB0DC10
:10358000B9F1000F40F0A5800023194600F10A08A8
:1035900000F6C639B8F802E0BEF1000F18BF0B46BE
:1035A000A9F80230B8F804504A1C002D18BF134681
:1035B000A9F80430B8F806408D1C002C18BF2B4623
:1035C000A9F80630B8F80840CA1C002C18BF1346EA
:1035D000A9F80830B8F80A500C1D002D18BF234672
:1035E000A9F80A30B8F80C504A1D002D18BF134630
:1035F000A9F80C30B8F80E408D1D002C18BF2B46D2
:10360000A9F80E3038F8104FCA1D0831002C18BF29
:103610001346B1F57A7F29F8103FBBD100F5DB5A8C
:1036200040F2E7330AF1080C9E4600F2DC7838F8E5
:10363000021C002918BF73462CF8023C38F8045CC1
:103640000EF1FF34002D18BF23462CF8043C38F847
:10365000062CAEF10201002A0CBF1D460D462CF8C7
:10366000065C38F8089CAEF10304B9F1000F0CBFFA
:103670002A4622462CF8082C38F80AACAEF104038E
:10368000BAF1000F0CBF114619462CF80A1C38F885
:103690000C5CAEF10504002D0CBF8946A1462CF848
:1036A0000C9C38F80E2CAEF1060A002A0CBF4D46D1
:1036B00055462CF80E5C38F8101DAEF10703AEF13C
:1036C000080E002908BF2B46BEF1FF3F2CF8103D25
:1036D000ADD1BE423446A8BF3C46002CC0F2DE81CC
:1036E000BA1B82EAE275A5EBE271012940F39981E8
:1036F000BE4240F39B81002FC0F29E81B6F57A7FD7
:1037000000EB470907F1010A80F2DC81B9F80C30BF
:1037100090F8C59B07EE903AF8EE676AB9F1000F92
:1037200000F09B8100EB4604F21BA58907EE105ABE
:1037300000EE902AB8EEC75AB8EEE01A75EE661A97
:10374000564581EE810A40F36C8100EB4A030A334F
:103750006FEA0A010AF1010C3144664501F00707DE
:1037600076EE806AB6EE002A76EE822ABCEEE24A57
:1037700014EE104A23F8024F40F3B380002F61D0BB
:10378000012F51D0022F43D0032F35D0042F27D043
:10379000052F19D0062F0BD076EE806A0CF1010CA4
:1037A00076EE823AFCEEE35A15EE908A23F8028F09
:1037B00076EE806A0CF1010C36EE826AFCEEC64AA7
:1037C00014EE90AA23F802AF76EE806A0CF1010C99
:1037D00036EE823AFCEEC37A17EE902A23F8022FD7
:1037E00076EE806A0CF1010C36EE827ABCEEC75A96
:1037F00015EE105A23F8025F76EE806A0CF1010C88
:1038000076EE820ABCEEE01A11EE101A23F8021FBF
:1038100076EE806A0CF1010C76EE821AFCEEE12A5B
:1038200012EE907A23F8027F76EE806A0CF1010C9A
:1038300036EE824A6645FCEEC43A13EE904A23F80F
:10384000024F4EDD76EE805A0CF1080C35EE806AA0
:1038500075EE827A76EE004A36EE027A34EE803ADF
:1038600074EE820A33EE001A33EE025A71EE001A39
:1038700071EE022A71EE803A31EE824A73EE806A6E
:1038800073EE825A36EE826AFCEEE54ABCEEC63A28
:10389000BCEEC41AFCEEE21ABCEEC55AFCEEE00A1D
:1038A000BCEEC77AFCEEE77A14EE90EA13EE108ACB
:1038B00011EE107A11EE905A15EE104A10EE901A91
:1038C00017EE102A17EE90AA6645A3F80EE09F8126
:1038D0005D811C81D9809A80A3F802A023F8108F03
:1038E000B0DCB9F1000F40F09C8000231F4600F1CE
:1038F0000A0C00F6C639BCF80260002E18BF3B4621
:10390000A9F80230BCF804507C1C002D18BF2346D7
:10391000A9F80430BCF80610BA1C002918BF1346D9
:10392000A9F80630BCF80880FE1CB8F1000F18BFDB
:103930003346A9F80830BCF80A503C1D002D18BFCA
:103940002346A9F80A30BCF80C107A1D002918BFCC
:103950001346A9F80C30BCF80EA0BE1DBAF1000F3A
:1039600018BF3346A9F80E303CF8105FFC1D08372D
:10397000002D18BF2346B7F57A7F29F8103FBAD13A
:1039800000F5DB5740F2E7330837194600F2DC7CDC
:103990003CF8029CB9F1000F18BF0B4627F8023C17
:1039A0003CF8048C4A1EB8F1000F18BF134627F8E4
:1039B000043C3CF806AC8E1EBAF1000F18BF33462B
:1039C00027F8063C3CF8085CCC1E002D18BF2346A7
:1039D00027F8083C3CF80A9CA1F10408B9F1000F53
:1039E00018BF434627F80A3C3CF80CAC4A1FBAF112
:1039F000000F18BF134627F80C3C3CF80E6C8D1FC7
:103A0000002E18BF2B4627F80E3C3CF8104DA1F1B4
:103A100007090839002C18BF4B464A1C27F8103DEF
:103A2000B6D1012780F8C47BBDE8F087B846374699
:103A3000002F4646BFF662AE00EB460790F8C59BE6
:103A4000BB89838107EE903A4FF0010A0027F8EE18
:103A5000676AB9F1000F7FF465AE56457FF745AF51
:103A60009FED2D0A71E64FF0FF3201E49642344695
:103A7000A8BF1446002C4FF0FF37BFF679AC964232
:103A8000B246B8BF9246BAF57A7FFFF671ACBE4235
:103A90003446A8BF3C46002CBFF622AEBE42B44618
:103AA000B8BFBC46BCF57A7FFFF61AAE012780F896
:103AB000C47BBDE8F0874FF47A72FFF7D9BB4FF4AF
:103AC0007A774EE4B9F80C60A0F8DA67B9F80C30F0
:103AD00040F2E7361CE6BCF80C90A0F8DA97BCF888
:103AE0000C4090F8C59B02EE904A40F2E732B8EEE7
:103AF000623AB9F1000F7FF45FAC42457FF744AD05
:103B0000DFED057A70E400EB420A4FF00108BAF8E5
:103B10000C408481002545E400000000F8B540F227
:103B2000E63384689942D4BF21EAE17540F2E73573
:103B3000002C0560C0F29880174606464FF4FA62E2
:103B400007F10C010C300FF0B7FB07F2DC714FF4FA
:103B50007A7206F2DC700FF0AFFBA54202DA204663
:103B60002C46054604F2DC72291BB4F57A7F3244F8
:103B700001F007074FF0000077DB631CAB4202F156
:103B800001026EDCCFB3012F2DD0022F25D0032FE1
:103B90001DD0042F15D0052F0DD0062F05D0B3F55D
:103BA0007A7FB8BF107001330132B3F57A7FB8BFA6
:103BB000107001330132B3F57A7FB8BF1070013352
:103BC0000132B3F57A7FB8BF107001330132B3F51B
:103BD0007A7FB8BF107001330132B3F57A7FB8BF76
:103BE000107001330132B3F57A7F03F10103B8BFDE
:103BF0001070AB4202F1010233DCB3F57A7F03F1BE
:103C00000103B8BF1070B3F57A7F02F1010400DA46
:103C100050705A1CB2F57A7F03F1020103F10307D9
:103C2000B8BF6070B1F57A7F03F10402B8BFA0702D
:103C3000B7F57A7F03F10501B8BFE070B2F57A7F7E
:103C400003F10607B8BF2071B1F57A7FB8BF607184
:103C50000733B7F57A7FB8BFA071AB4204F1070212
:103C6000CBDD3046FFF73EFAF8BD107085E700BFA8
:103C70002DE9F04F2DED028B0546FF2485B048223B
:103C8000002112F059F805F5A84A85F8244085F876
:103C9000254005F148004822002105F5F83912F0C9
:103CA0004BF80AF1640A85F86C4085F86D4009F517
:103CB000CC790027AAF5A540AAF59548AAF55D5646
:103CC000A0F12404A8F15408043E4FF4FA62002144
:103CD000204612F031F84FF47A720021404612F07B
:103CE0002BF820220021304612F026F84FF4FA6219
:103CF000002104F6BC3012F01FF804F59C504FF47C
:103D0000FA6200210C3012F017F801214FF0FF3257
:103D100063234FF0000C84F8D01744F8042C84F887
:103D2000BA3B44F80C7C44F8087C84F8B87B84F8EF
:103D3000B97B84F8BB7B634606F8047C06F8037CF9
:103D4000A11E04F6BA32B1F802B0BBF1000F14BFE5
:103D5000184660465080B1F804C003F1010EBCF172
:103D6000000F18BF70469080B1F806B003F1020C46
:103D7000BBF1000F18BF6046D080B1F808B003F166
:103D8000030EBBF1000F18BF70461081B1F80AC0D6
:103D900003F1040BBCF1000F18BF58465081B1F875
:103DA0000CE003F1050CBEF1000F18BF60469081D6
:103DB000B1F80EE003F1060BBEF1000F14BFDC46B4
:103DC0008446A2F80EC031F810EFD81D0833BEF1BA
:103DD000000F18BF8446B3F57A7F22F810CFB2D116
:103DE00004F5DA5040F2E7331C301946C3463BF87D
:103DF000022C002A18BF0B4620F8023C3BF804ECCA
:103E000001F1FF3CBEF1000F18BF634620F8043CEF
:103E10003BF806EC8A1EBEF1000F18BF134620F8CF
:103E2000063C3BF808CCA1F1030EBCF1000F18BF13
:103E3000734620F8083C3BF80ACC0A1FBCF1000F7F
:103E400018BF134620F80A3C3BF80CECA1F1050C16
:103E5000BEF1000F18BF634620F80C3C3BF80EEC97
:103E60008A1FBEF1000F18BF134620F80E3C3BF826
:103E700010CDA1F1070E0839BCF1000F18BF734631
:103E80004A1C20F8103DB2D104F5DC540C3408F57E
:103E9000DC5806F5DC56A24508F10C0806F10C06C4
:103EA0007FF413AF0AF5A54A0AF1240AD1457FF43D
:103EB00001AF05F5D13909F5807B5846FDF704F9C6
:103EC00005F5DF3005F5E03CDFEDC87AC84EC0ED02
:103ED0002E7A00244FF07E534FF07C57C0ED377A96
:103EE000C0ED407AC0ED497AC0F8B040C0F8BC409F
:103EF000C0F8C040C0F8B430C0F8C830C0F8CC300A
:103F0000C0F8C470C0F8D060C0F8D440C0F8D83051
:103F1000C0F8E040C0F8E870C0F8E440C0F8EC3009
:103F2000C0F8F030C0F8F460C0F8F840C0F8FC30D9
:103F3000C0F80441C0F80C71C0F80841C0F8103155
:103F4000C0F81431C0F81861C0F81C41C0F8203125
:103F5000C0F82841C0F830710021C0F82C41A54AB2
:103F6000C0ED527AC0ED5B7AC0ED647AC0F83431AE
:103F7000C0F83831C0F83C61C0F84041C0F8443165
:103F8000C0F84C41C0F85471C0F85041C0F85831E5
:103F9000C0F85C31C0F86061C0F86441C0F86831B5
:103FA000C0F87041C0F87871C0F87441C0F87C3135
:103FB000C0F88031C0F88461C0F88841C0F88C3105
:103FC000C0F89441C0F89C71C0F89841C0F8A03185
:103FD000C0F8A431C0F8A861C0F8AC41C0F8B03155
:103FE000C0ED6D7AC0ED767AC0ED7F7AC0F8B84149
:103FF000C0F8C071C0F8BC41C0F8C431C0F8C831C5
:10400000C0F8CC61C0F8D041C0F8D431C0F8DC4170
:10401000C0F8E471C0F8E041C0F8E831C0F8EC3114
:10402000C0F8F061C0F8F441C0F8F831C0F80042BF
:10403000C0F80872C0F80442C0F80C32C0F8103260
:10404000C0F81462CCF81840CCED087ACCF82440C3
:10405000CCF82C70CCF82840CCF81C30CCF83030A0
:10406000CCF834302846CCF83860CCF83C40CCED65
:10407000117ACCF84840CCF85070CCF84C40CCF8D1
:104080005C60CCF86040CCED1A7ACCF86C40CCF88F
:104090007470CCF87040CCF88060CCF88440CCEDE3
:1040A000237ACCF89040CCF89870CCF89440CCF8B7
:1040B000A460CCF8A840CCED2C7ACCF8B440CCF875
:1040C000BC70CCF84030CCF85430CCF85830CCF838
:1040D0006430CCF87830CCF87C30CCF88830CCF830
:1040E0009C30CCF8A030CCF8AC30CCF8B840CCF850
:1040F000C860CCF8C030CCF8C43011F01DFE0027E9
:1041000001225846C5F89470C5F8987085F8A170DA
:10411000C5F89C20FCF7D8FF3749C5F818410E6850
:1041200003964FF0030903989FED348A85F8AA900F
:104130004FF00F0A05F5CF38052485F8907085F803
:10414000917085F81471C5F81071C5F80C0185F8E7
:10415000A9A008F1E4082E46A946009501944FF461
:10416000FA62002106F5E07011F0E6FD4FF47A7274
:10417000002106F5196011F0DFFD2022002106F56F
:10418000E95011F0D9FD4FF4FA62002106F67C5097
:1041900011F0D2FD06F5AA504FF4FA62002106F59F
:1041A000E85B0C3011F0C8FD012263234FF0FF31B2
:1041B00086F87A3DC6F8B471C6F8B87186F8787D8D
:1041C00086F87B7D86F8902986F8792DC6F8BC1193
:1041D00006F5DF738BF81C708BF81D704FF0000A2A
:1041E000B6EE000A86F8772D0AE000BF0AD7233C16
:1041F000CDCCCC3DF4C00100EC440120823383429D
:104200000AF102040AF1010006EE904A0AF10601E1
:104210000AF103020AF1040E0AF1050B07EE100A77
:1042200005EE901A0AF1070004EE102A04EE90EA57
:1042300005EE10BAF8EEE60A06EE100A03EE90AAB2
:10424000F8EEE58AF0EE406AB8EEC71AF8EEC67AE4
:10425000B8EEE33AE0EE886A0AF1080ABAF57A7F26
:10426000F8EEC41AB8EEE42AF8EEC52AB0EE407AA9
:10427000A8EE887AF0EE403AB0EE404AF0EE404ABE
:10428000B0EE405AB0EE406AF0EE408AE1EE083AF5
:10429000A1EE884AE2EE084AA7EE886AE3EE088AB1
:1042A000A2EE885AFCEEE67ABCEEE33A17EE90CA2C
:1042B000FCEEC46AFCEEE40AFCEEC53ABCEEC74A6A
:1042C000BCEEC61AFCEEE84AA3F806C013EE102AAC
:1042D00016EE90BA10EE90EA13EE904A14EE100A21
:1042E00011EE10CA14EE901A9A80A3F808B0A3F841
:1042F0000AE09C81D881598023F810CF80D106F53F
:10430000145406F5EA504FF4FA6200211C340C30C4
:1043100011F012FD52460021204611F00DFD06F568
:104320006250202200212C3011F006FD06F52450A9
:104330004FF4FA620021083011F0FEFC06F54350FC
:1043400006F5EA5A4FF4FA620021183011F0F4FC35
:1043500006F5245ED446012323707246CAF8007025
:10436000CAF80470D34606F562534FF0FF3ACCF812
:1043700008A006327146283306F5625C4FF0630AE6
:1043800000208EF804708EF805700BF10A0B82F88D
:1043900000A0CF7182461F708CF82970BBF8021004
:1043A000002918BF50465080BBF804C00AF1010E26
:1043B000BCF1000F18BF70469080BBF806C00AF130
:1043C0000201BCF1000F18BF0846D080BBF808E01E
:1043D0000AF1030CBEF1000F18BF60461081BBF854
:1043E0000AE00AF10401BEF1000F18BF084650812F
:1043F000BBF80CC00AF1050EBCF1000F18BF7046E7
:104400009081BBF80EC00AF10601BCF1000F18BF85
:104410000846D0813BF810EF0AF1070C0AF1080AB0
:10442000BEF1000F18BF6046BAF57A7F22F8100F70
:10443000B4D140F2E732924634F8020C002818BF9B
:10444000524623F8022C34F804BC0AF1FF31BBF1C8
:10445000000F18BF0A4623F8042C34F806ECAAF122
:104460000200BEF1000F18BF024623F8062C34F8F4
:1044700008CCAAF1030BBCF1000F18BF5A4623F871
:10448000082C34F80AECAAF10401BEF1000F18BFA1
:104490000A4623F80A2C34F80C0CAAF1050C002863
:1044A00018BF624623F80C2C34F80EBCAAF1060E95
:1044B000BBF1000F18BF724623F80E2C34F8100D14
:1044C000AAF10701AAF1080A002818BF0A46BAF1A2
:1044D000FF3F23F8102DAFD106F5814406F5635058
:1044E0004FF4FA6200212834183011F025FC4FF403
:1044F0007A720021204611F01FFC06F5A840202208
:104500000021383011F018FC06F589404FF4FA62AA
:104510000021143011F010FC06F598404FF4FA62B7
:104520000021643011F008FC06F56352944606F54C
:1045300089409346012121700346D760CCF8107062
:1045400006F5A84CCBF814A000F1120E02460CF1AF
:10455000340C06F5A84B077406F5635A5F746320A4
:1045600000238EF800000AF1160AD77418468CF85A
:1045700000708BF83570BAF80210002918BF034696
:10458000AEF80230BAF804B0421CBBF1000F18BFFD
:104590001346AEF80430BAF80610821C002918BF82
:1045A0001346AEF80630BAF808B0C11CBBF1000FD4
:1045B00018BF0B46AEF80830BAF80AB0021DBBF1BE
:1045C000000F18BF1346AEF80A30BAF80C10421D9F
:1045D000002918BF1346AEF80C30BAF80EB0811D92
:1045E000BBF1000F18BF0B46AEF80E303AF810BF03
:1045F000C21D0830BBF1000F18BF1346B0F57A7F1B
:104600002EF8103FB7D140F2E7339E4634F8020C43
:10461000002818BF73462CF8023C34F804AC0EF1A5
:10462000FF31BAF1000F18BF0B462CF8043C34F8E8
:10463000060CAEF1020B002818BF5B462CF8063CB6
:1046400034F808ACAEF10302BAF1000F18BF1346FC
:104650002CF8083C34F80A1CAEF10400002918BFFD
:1046600003462CF80A3C34F80CBCAEF1050ABBF149
:10467000000F18BF53462CF80C3C34F80E1CAEF15A
:104680000602002918BF13462CF80E3C34F8100D12
:10469000AEF10701AEF1080E002818BF0B46BEF1BF
:1046A000FF3F2CF8103DB1D100982F4BC0F8C4301B
:1046B0002E4A9FED2F0A2F4CDFF8BCB0DFF8BCA0CC
:1046C000DFF8BCC0DFF8BCE0022348F8043FC0F8C4
:1046D0001C2109F5DF3309F5E03200210430C3F86D
:1046E000CC40C3F88041C3F8B010C3F8BC10C3F885
:1046F000C010C3F86411C3F87011C3F87411C3F883
:10470000B4B0C3F868B1C3F8B8A0C3F86CA1C3F8DB
:10471000C4C0C3F878C1C3F8C8E0C3F87CE183ED36
:10472000340A83ED610A00905463C2F81CB09161B1
:10473000C2F820A051629162C2F82CC0C2F830E0E9
:1047400082ED0E0A019906F5A5464C1E06F12406D7
:1047500009F1240901947FF402AD284605B0BDECAF
:10476000028BBDE8F08F00BFF1D8FFFF0AD7233DD1
:10477000507EAA46C000C03800FF7F470000FA43C1
:104780008FC2753CC1FB813FFE2843D0431E03F01E
:10479000FE01FE2922D0D12922DCA92922DC872989
:1047A00022DC692922DC512922DC3D2922DC2B294B
:1047B00022DC1F2922DC152922DC0D2922DC092913
:1047C00022DC052922DC032922DC0129D4BF0021B7
:1047D0000121C2074CBF481CC84370470F21F8E7AE
:1047E0000E21F6E70D21F4E70C21F2E70B21F0E7AB
:1047F0000A21EEE70921ECE70821EAE70721E8E7CB
:104800000621E6E70521E4E70421E2E70321E0E7EA
:104810000221DEE76FF00F00704700BFD0F8942050
:104820008A4200F082812DE9F04F2DED028B90F845
:10483000A130D0F8985085B0002B40F0248145F28B
:10484000A42404FB05F641F68C3707FB026880447C
:1048500008F5DA7C074600F5D130C7F8941041F628
:104860008C3101FB02F201929FEDB08A029000F5BB
:10487000867203924FF0000945F2A42BB8460BFB59
:1048800005F441F68C3606FB094A0BFB05F1DCF812
:10489000006041F68C3C0AF5D8770CFB091A08EB4E
:1048A0000A0240F2E630D2F8BC418642D4BF26EA82
:1048B000E67640F2E7364744002C07F10403C2F8DD
:1048C000B461C0F2A88002F5E070039900934FF440
:1048D000FA620EF0F1FC029908EB0A0303F5196085
:1048E0004FF47A7201F6DC010EF0E6FCA642009B62
:1048F00002DA3046264604460BFB05FC0CF5196A25
:1049000041F68C3202FB09ACA444311BB4F57A7F2A
:1049100008EB0C0E01F007014FF0000001DA08F877
:104920000C000134B4420EF101026FDCD1B3012955
:104930002ED0022926D003291ED0042916D00529FD
:104940000ED0062906D0B4F57A7FB8BF8EF80100E4
:1049500001340132B4F57A7FB8BF107001340132EE
:10496000B4F57A7FB8BF107001340132B4F57A7FA4
:10497000B8BF107001340132B4F57A7FB8BF10703F
:1049800001340132B4F57A7FB8BF107001340132BE
:10499000B4F57A7F04F10104B8BF1070B44202F19B
:1049A000010233DCB4F57A7F04F10104B8BF107062
:1049B000B4F57A7F02F1010100DA5070621CB2F5A1
:1049C0007A7F04F10202B8BF4870B2F57A7F04F131
:1049D0000302B8BF8870B2F57A7F04F10402B8BF51
:1049E000C870B2F57A7F04F10502B8BF0871B2F55C
:1049F0007A7F04F10602B8BF48710734B2F57A7FB6
:104A0000B8BF8871B44201F10702CBDD18460093AC
:104A1000FEF768FB009B97ED017AB8EEC70AC0EE7F
:104A2000087A67EE880AF5EEC00AF1EE10FA72D93C
:104A3000F4EEC80AF1EE10FA3ADB0BFB05F041F692
:104A40008C3A0AFB090CC444BCF88E490BFB05F5F3
:104A500041F68C3606FB09504044C0F8B8419C68CA
:104A6000002C02DB1846FEF73DFB09F10109B9F104
:104A7000030F4BD0D8F89850019B0BFB053AC2446A
:104A80000AF5DA7CFBE645F2A42404FB05F441F6C2
:104A90008C3909FB024A82440AF5DA7B4FF0000C9C
:104AA0004FF0FF3680F8A1C0DC46CBF80860D1E6B5
:104AB000BDEEE01A42F6521606FB05F440F6C6506B
:104AC00011EE10CA00FB094AE24408EB4A01F8EE75
:104AD000C11AB1F8C071B1F8C26106EE907A06EE63
:104AE000106AB8EE662AF8EE462A30EEE13A72EE27
:104AF000C23AB6EE004AA3EE232A72EE044ABCEE96
:104B0000E45A8DED005ABDF800409FE705B0BDECBA
:104B1000028BBDE8F08F0BFB05F241F68C3101FBF7
:104B200009274744B7F8C04190E7704700C079446F
:104B30002DE9F04FD0F89890D0F894A0436FC26A56
:104B400045F2A42606FB09F541F68C3101FB0A5714
:104B500007F5D87606440446371D981A03B283B089
:104B6000D7F804B0002B00F04B8183EAE37CACEB78
:104B7000E372022A984615DD03EB430585EAE578E2
:104B8000A8EBE572102AA8460CDD002D40F38182C7
:104B90004FF00108083A510008FB01F888EAE87074
:104BA000A0EBE872082A09DDB8F1000F40F3848217
:104BB0004FF00108131F5D0008FB05F894F85C1026
:104BC0007068002900F01882012584F8A350642140
:104BD00001FB08F8404440F2E6329042D8BF20EA98
:104BE000E07845F2A42000FB09FC41F68C3303FB7E
:104BF0000AC104EB0102C8BF40F2E738D2F8BC5149
:104C0000C2F8B481002DC0F2A78004F5D13C019117
:104C100002F5E0700CF586714FF4FA62CDF800C031
:104C20000EF04AFB01980099221802F5196001F66E
:104C3000DC014FF47A720EF03FFBA84502DAC6465B
:104C4000A846754641F68C3C0CFB0AF045F2A423BD
:104C500003FB090202F51963C5EB08012B44B5F506
:104C60007A7F01F0070023444FF00001C0F2078271
:104C70000135454503F101036BDCC8B301282DD094
:104C8000022825D003281DD0042815D005280DD0D2
:104C9000062805D0B5F57A7FB8BF19700135013304
:104CA000B5F57A7FB8BF197001350133B5F57A7F54
:104CB000B8BF197001350133B5F57A7FB8BF1970E7
:104CC00001350133B5F57A7FB8BF1970013501336D
:104CD000B5F57A7FB8BF197001350133B5F57A7F24
:104CE00005F10105B8BF1970454503F1010330DC3A
:104CF000B5F57A7F05F10105B8BF1970B5F57A7F72
:104D000003F1010200DA59706B1CB3F57A7F05F1EB
:104D1000020005F10303B8BF5170B0F57A7FB8BF48
:104D20009170281DB3F57A7FB8BFD1706B1DB0F5B7
:104D30007A7FB8BF1171A81DB3F57A7FB8BF5171E2
:104D40000735B0F57A7FB8BF9171454502F1070389
:104D5000CEDD3846FEF7C6F9D6ED017ADFEDD26A30
:104D6000B8EEE77A87EE260A60EE260AF5EEC00A6C
:104D7000F1EE10FA40F2A681F4EEE60AF1EE10FA36
:104D800080F27181BDEEE06A42F6521505FB09F131
:104D900040F6C65216EE10CA02FB0A18E04404EBB5
:104DA0004800B8EEC62AB0F8C051B0F8C21101EE02
:104DB000105A01EE901AF8EE412AB8EE613A70EE00
:104DC000C23A33EE624AF6EE004AE4EE232A32EEAD
:104DD000A45AFCEEC55ACDED005ABDF8000045F2CC
:104DE000A42505FB09F141F68C3808FB0A1CA444F4
:104DF000CCF8B801BB68002B02DB3846FEF772F92D
:104E0000A06F226B851A2BB2002B71D083EAE37E50
:104E1000AEEBE371302904DD5B0083EAE371A1EBC3
:104E2000E371022914DD03EB430383EAE370A0EB93
:104E3000E37110290CDD002B40F326810122A1F142
:104E400008035B0002FB03F383EAE375A5EBE37160
:104E5000082907DD002B40F322810122081F4300AF
:104E600002FB03F394F85E50002D00F0D080012087
:104E700084F8A400652505FB03F303EB8318C34402
:104E8000ABF165014FF6357C614515D806EE90BA59
:104E90009FED860ADFED860AF8EEE67AB6EE007A36
:104EA000A7EE807ABDEEC71AF8EEC11A21EEA02A4D
:104EB000FDEEC22A12EE90BA45F2A42E0EFB09F0C6
:104EC00041F68C324FF6FE7302FB0A059B452544E2
:104ED000D4BF2BEAEB734FF6FF73C5F8B831B9684E
:104EE000002902DB3846FEF7FDF83846FEF7FAF8EF
:104EF00094F864301BBB207F08B394F8A120002AEB
:104F000000F0BF80D4F89850D4F8940084F8A13011
:104F100045F2A42303FB05F541F68C3101FB005C4F
:104F2000A4444FF0FF32CCF8BC21002800F0EA8006
:104F3000471E012F40F2D18103B0BDE8F08F94F8F5
:104F400060509DB9227E8AB194F8A100002840F0FB
:104F5000C580D4F89420012A00F0F88232F00203D0
:104F6000EAD120460121FFF759FCE5E794F86230C9
:104F700073B394F85C00002854D1257D002D51D0E6
:104F800094F8A330002B4DD194F8A100002800F034
:104F9000A981D4F89860D4F8940084F8A13045F23F
:104FA000A42303FB06F341F68C3202FB003B04F51D
:104FB000D138A34408F580714FF0FF358F42CBF80C
:104FC000BC51B9D0384603B0BDE8F04F0EF074B90B
:104FD000A17E0029CDD094F8A120002A40F049817B
:104FE000D4F89400022800F0BD820128A4D82046FD
:104FF0000221FFF713FC9FE794F85D20002A7FF45D
:10500000E3AD94F8A330002B3FF4E4ADDFE594F872
:105010005F1000297FF42BAF94F8A420002A3FF4FE
:105020002CAF27E794F85E60002E85D1A27D002A80
:1050300082D094F8A40000287FF47EAF94F8A110E9
:10504000002940F0368104F5D13808F58070874298
:1050500004D041F68C3239460EF02EF90121384643
:1050600084F8A110DEE045F2A42202FB09F541F626
:105070008C3808FB0A5CA444BCF88E09AFE61970B2
:10508000F6E5D4F8940050E714BF4FF0FF32002249
:10509000D5E614BF4FF0FF384FF000087AE514BF93
:1050A0004FF0FF320022D9E600C07944FA007A3C82
:1050B000EC11834200C0794414BF4FF0FF384FF029
:1050C000000877E545F2A42341F68C3003FB09F193
:1050D00000FB0A122244B2F8C00180E6D4F898100E
:1050E000D4F8942084F8A15045F2A42303FB01F1E5
:1050F00041F68C3505FB021BA3444FF0FF30CBF883
:10510000BC0128E74FF0FF30BD68B86045F2A4232A
:1051100003FB09F1D6F804B041F68C3202FB0A1009
:105120002044594640F2E73808E0431893F89029A4
:1051300012B1BEF1010F16D18B4514D04A1C00F1FB
:105140008380B2F57A7FC0F288804FF0000E7146FE
:105150000123034493F89029002AE6D1431893F8D9
:105160009029002AE8D004F5D13808F58072384635
:10517000FEF7D4FC96ED013A5FED323AB8EEC34A41
:10518000C4EE234A24EEA35AB5EEC05AF1EE10FA4B
:1051900040F2D081B4EEE35AF1EE10FA7DDAFDEE82
:1051A000C55A42F6521606FB09F140F6C65015EEF6
:1051B00090BA00FB0A1CDC4404EB4C08B8EEE50A8C
:1051C000B8F8C031B8F8C22107EE903A06EE902A3E
:1051D000F8EE670AB8EE667A35EE401A77EE601A96
:1051E000B6EE006AE1EE210AC64630EE862AFCEEF3
:1051F000C22ACDED002ABDF8006045F2A42101FBD2
:1052000009F041F68C3C0CFB0A0BA344CBF8B861C7
:10521000BE68002E02DB3846FDF764FF002DFFF666
:105220008BAE384645F2A42505FB09F741F68C39CB
:1052300009FB0A7A5444FDF755FFD4F8B431C4F899
:10524000BC3103B0BDE8F08F40F2E731431893F86A
:105250009029002A3FF470AF85E7002A00F0C5814D
:105260004318424593F890E900F083818B1C114666
:105270006FE7D4F89810D4F8940084F8A13045F280
:10528000A42303FB01F141F68C3505FB001CA4446B
:105290004FF0FF32CCF8BC21A4E645F2A42101FB7B
:1052A00009F041F68C3C0CFB0A0BA344BBF88E6959
:1052B000A3E7D4F89870D4F8945084F8A10045F28C
:1052C000A42303FB07F341F68C3606FB05394C4457
:1052D0004FF0FF32C4F8BC212EE620460021FFF734
:1052E0009DFA29E641F68C3C45F2A42B0CFB0AFE04
:1052F0000BFB09F50EEB05032344D3F8B421B2F5FB
:105300007A7F80F0E58002F68F11134471442944BE
:10531000013183F8900912F0070004EB01031146F4
:105320002BD013F8018D511EB8F1000F53D1012875
:1053300023D002281DD0032817D0042811D0052817
:105340000BD0062804D013F8010D0139002842D1F2
:1053500013F8010D013900283DD113F8010D013971
:10536000C8BB13F8010D0139A8BB13F8010D0139B1
:1053700088BB13F8010D013968BB934601394A1CFB
:10538000884627D013F8012C03F1FF3C12BB1CF810
:10539000010C0139F0B913F8032CA8F10201CAB9C4
:1053A00013F8040CA8F10301A0B913F8052CA8F117
:1053B00004017AB913F8060CA8F1050150B913F8E5
:1053C000072CA8F106012AB913F8080DA8F1070166
:1053D0000028D3D05A4602F691139E44AE44C2F53B
:1053E000797503350EF1FF3B15F00700A34428D073
:1053F0001BF8013F0132002B4AD1012821D002289D
:105400001BD0032815D004280FD0052809D0062862
:1054100003D01BF8015F0132D5BB1BF8010F01322D
:10542000B0BB1BF8013F013293BB1BF8015F013297
:1054300075BB1BF8010F013250BB1BF8013F013255
:1054400033BB0132B2F57A7F104621D09BF8015070
:105450000BF10108E5B998F801300132C3B99BF8A6
:105460000350821CA5B99BF80430C21C83B99BF879
:105470000550021D65B99BF80630421D43B99BF8E3
:105480000750821D25B91BF8083FC21D002BD8D03C
:105490003846FDF70BFC45F2A42101FB09FC41F65F
:1054A0008C3202FB0ACBA34442F6521000FB09F3F4
:1054B000DBF8B45140F6C65808FB0A310D4404EB42
:1054C000450C0120BCF8C021CBF8B8218BF8780D31
:1054D00096ED013ADFED473AB8EEC34AC4EE234AEF
:1054E00024EEA35AB5EEC05AF1EE10FA71D9B4EE1B
:1054F000E35AF1EE10FA3EDB45F2A42505FB09F173
:1055000041F68C3B0BFB0A132344B3F88E6945F23A
:10551000A42505FB09F141F68C3909FB0A1A54440C
:10552000C4F8B861BC68002CFFF606AD3846FDF73C
:10553000D9FD01E545F2A42808FB09FE41F68C33AC
:1055400003FB0AE22244B2F8C06156E64FF0FF3195
:10555000BD68B96071683846FDF78EFD04F5D13835
:10556000014602E64FF0FF31BD68B9607168012263
:10557000F1E74146F2E5FDEEC55A42F6521606FB4A
:1055800009F540F6C65B15EE908A0BFB0A534344BF
:1055900004EB4301B8EEE50AB1F8C001B1F8C2214D
:1055A00007EE900A06EE902AF8EE670AB8EE667AE1
:1055B00035EE401A77EE601AB6EE006AE1EE210A87
:1055C00030EE862AFCEEC22ACDED002ABDF800603E
:1055D0009DE745F2A42000FB09F841F68C3202FB5E
:1055E0000A8CA444BCF8C06191E711469646012399
:1055F000AFE500BF00C079442DE9F041064600F157
:1056000047050024012741F68C3815F8013F3BBBC4
:1056100015F8480C20B396F8A6300BBBD6F89820A6
:10562000A24222D096F8A11096F890C086F891C0B8
:1056300086F8907071B1D6F8941086F8A13045F2D2
:10564000A42000FB02F208FB012EB6444FF0FF330A
:10565000CEF8BC3100213046FFF7E0F8C6F898409C
:105660000134052CD1D1BDE8F08196F89020002AB4
:10567000F6D096F8A10086F8912086F8903070B1A7
:10568000D6F8941086F8A13045F2A42C0CFB04FE49
:1056900008FB01E333444FF0FF32C3F8BC21002183
:1056A00030460134FFF7BAF8052CAED1DBE700BF76
:1056B00090F89020012A30B403462ED093F8485039
:1056C00015B11978002970D193F8491019B15C7897
:1056D000002C40F0BC8093F84A201AB1987800283A
:1056E00040F0C88093F84B401CB1DA78002A40F0B3
:1056F000C68093F84C0030B993F8F80008B993F8D5
:10570000FA0030BC70471C79002CF5D00424002D21
:1057100040F09F80002954D050E0817EC9B190F8BC
:105720006000B0B1187E0028C8D193F8A11083F8AA
:10573000A220F9B90222C3F8F0200121002501209E
:10574000C3F8F41083F8F85083F8FA5083F8F9009E
:10575000D7E7187E0028B1D093F86240002CADD076
:105760000029ABD193F8A15093F86010012283F87F
:10577000A2209DB1D3F89850D3F8942045F2A424E8
:1057800004FB05F441F68C3C0CFB02421A44002554
:105790004FF0FF3483F8A150C2F8BC41002973D107
:1057A0000120C3F8F0000221C8E793F85240002C12
:1057B00040F09F8093F8494034B100245D78012186
:1057C000E5B1022C00F0A48093F84A5015B19A7804
:1057D00002219AB1032C00F0918093F84B5015B13F
:1057E000DA78032152B1042C53D093F84C50002D99
:1057F00082D01A79002A7FF47FAF042193F8A15058
:105800004FF0010C83F8A2C09DB1D3F89850D3F8A3
:10581000942045F2A42000FB05F041F68C3C0CFBE3
:1058200002021A4400254FF0FF3083F8A150C2F85D
:10583000BC014FF0000C0120C3F8F040C3F8F41095
:1058400083F8F80083F8FAC083F8F9C059E7012417
:1058500025B11D78DDB1012C7FF45CAF93F85310B6
:1058600011B1DA7A0124EAB193F84A000124002840
:10587000ADD1B2E70224002D3FF44CAFE9E7032499
:10588000002D3FF447AFE4E7002889D152E72946CD
:10589000B4E793F8561000293FF42EAF987B002808
:1058A0007FF42AAF93F8A120012183F8A2109AB1C6
:1058B000D3F89850D3F8942045F2A42101FB05F1C8
:1058C00041F68C3000FB021C9C4400254FF0FF3257
:1058D00083F8A150CCF8BC2100200121C3F8F0408E
:1058E000C3F8F44083F8F80083F8F90083F8FA105D
:1058F00005E79C7A002C7FF45DAFD3E793F8551051
:1059000000293FF472AF587B00287FF46EAFC9E7DF
:1059100093F8541011B11A7B002AC3D093F84B00AE
:1059200000287FF45DAF60E72DE9F04F2DED028B8D
:1059300090F85C308BB00546002B40F04E8490F818
:105940005D40002C00F06C8495F852700FB995F80A
:10595000577095F8533013B995F858303B4395F884
:10596000540010B995F85900184395F8551011B91D
:1059700095F85A10014395F856402CB995F85B20DC
:1059800012B909B985F8A51095F96C0000287EDBDD
:1059900042F6041847F6A83749F234764BF2C02491
:1059A0004CF64C6205F5DF3B44F2904C46F21C0E7F
:1059B00000238BF8AF304EF6D81185F8783D05F509
:1059C000823A05F8083005F5903905F80C3005F5F0
:1059D0009E3805F80E30EB55AB5505F5AC372B5519
:1059E00005F5B936AB5405F5C73495F8A1206B54CD
:1059F0008AF8643189F8F03088F87C303B7286F898
:105A0000943184F8203192B1D5F89810D5F89420CB
:105A100085F8A13045F2A42303FB01F141F68C3C4B
:105A20000CFB021EAE444FF0FF31CEF8BC1105F561
:105A3000D872E749FBF73AFD48BB8BF8AF0042F656
:105A4000041246F21C0144F2904B85F8780D47F69B
:105A5000A833A85449F2347C05F80B004CF64C6E80
:105A600068544EF6D8124BF2C021E85405F80C00E9
:105A7000685405F80E00A8548AF8640189F8F0000B
:105A800088F87C00387286F8940184F8200195F932
:105A90006D000028C0F2868395F8A170A7B1D5F8F3
:105AA0009860D5F8944045F2A42303FB06F341F631
:105AB0008C3A0AFB0439A9444FF000084FF0FF313B
:105AC00085F8A180C9F8BC1105F5D13B0BF58070B4
:105AD000FBF7FAFA47F6A83705F5DF3C49F23476CA
:105AE0004BF2C0244EF6D81105F5823005F5903200
:105AF00042F6041A44F2904846F21C0E4CF64C69E9
:105B000000230090019205F59E3295F96D000292F6
:105B10008CF8AF3095F8A12085F8783D05F80A306B
:105B200005F8083005F80E30EB55AB552B5505F848
:105B300009306B540099CDF80CC081F8643101999B
:105B400005F5AC3781F8F03005F5B93605F5C73401
:105B50000299049781F87C3005963B72069486F88A
:105B6000943184F82031002A40F0468305F5D8723C
:105B70009749FBF77BFB002800F0D68205F5814AA8
:105B800005F5A84E05F5145705209FED928A079557
:105B90002C460AF128080EF134091C370026054668
:105BA0004FF4FA62002104F5E07010F0C5F84FF4EC
:105BB0007A72002104F5196010F0BEF8202200214D
:105BC00004F5E95010F0B8F84FF4FA62002104F639
:105BD0007C5010F0B1F804F5AA5004F5E85B4FF4DE
:105BE000FA6200210C3010F0A7F859464FF0010C72
:105BF0004FF0FF336322C4F8B461C4F8B86184F88D
:105C0000786D84F87B6D84F890C984F879CDC4F8F8
:105C1000BC3184F87A2DF6EE007A8BF81C604FF0D8
:105C2000000A4E7704F5DF7B84F877CD0AF1020E87
:105C30000AF104030AF1010006EE10EA04EE103A3C
:105C40000AF1050C0AF1030107EE100A04EE90CAEE
:105C50000AF106020AF1070005EE90AA03EE901A77
:105C6000B8EEC60A05EE102A06EE900AF8EEC41A3F
:105C7000B8EEE42AB8EEE53AF8EEC70AF0EE675A55
:105C8000B0EE677AF8EEC52AF8EEE68AE0EE085A3A
:105C90000AF1080ABAF57A7FB8EEE31AA1EE887A1B
:105CA000B0EE674AA2EE084AB0EE676AF0EE673AD5
:105CB000F0EE674AB0EE675AB0EE672AA0EE886A47
:105CC000E1EE083AE2EE884AA8EE885AA3EE082AE6
:105CD000FCEEE56ABCEEC73A16EE903AFCEEC62A38
:105CE000FCEEE38A13EE102AFCEEC45ABCEEE46A22
:105CF000FCEEC53ABCEEC20AABF80630ABF80A209F
:105D000012EE90EA18EE90CA15EE901A16EE100AEE
:105D100013EE903A10EE102AABF804E0ABF808C08E
:105D2000ABF80C10ABF80E00ABF802202BF8103FCC
:105D30007FF47CAF04F5EA504FF4FA6200210C3096
:105D40000FF0FAFF5246002138460FF0F5FF04F538
:105D50006250202200212C300FF0EEFF04F5245079
:105D60004FF4FA62002108300FF0E6FF04F54350CB
:105D700004F5EA5A4FF4FA62002118300FF0DCFF04
:105D800004F5245ED44601233B707246CAF80060D5
:105D9000CAF80460D34604F562534FF0FF3ACCF8DA
:105DA00008A071460632283304F5625C4FF0630A9E
:105DB00000208EF804608EF8056082F800A00BF1D8
:105DC0000A0ECE7182461E708CF8296004E000BF76
:105DD0004C9D010082338342BEF80210002918BF97
:105DE00050465080BEF804C00AF10101BCF1000F1A
:105DF00008BF01469180BEF806000AF1020B002898
:105E00000CBF8C46DC46A2F806C0BEF808100AF1AA
:105E10000300002908BF60461081BEF80AB00AF1ED
:105E2000040CBBF1000F18BF60465081BEF80CB0E7
:105E30000AF10501BBF1000F0CBF84468C46A2F8A5
:105E40000CC0BEF80E000AF1060B002808BFE3469E
:105E5000A2F80EB03EF8101F0AF107000AF1080A76
:105E6000002908BF5846BAF57A7F22F8100FB3D13F
:105E700040F2E7329246BC463CF802ECBEF1000F1D
:105E800018BF524623F8022C3CF804BC0AF1FF313B
:105E9000BBF1000F18BF0A4623F8042C3CF8061C7F
:105EA000AAF1020000290CBF9346834623F806BCE2
:105EB0003CF8082CAAF1030E002A0CBF5946714683
:105EC00023F8081C3CF80A0CAAF1040B00280CBFAC
:105ED0000846584623F80A0C3CF80CECAAF10502D7
:105EE000BEF1000F0CBF8346934623F80CBC3CF870
:105EF0000E1CAAF1060000290CBFDE46864623F8D8
:105F00000EEC3CF8101DAAF10702AAF1080A0029BC
:105F100008BF7246BAF1FF3F23F8102DACD104F54B
:105F200063504FF4FA62002118300FF005FF4FF470
:105F30007A72002140460FF0FFFE04F5A8402022AF
:105F4000002138300FF0F8FE04F589404FF4FA6272
:105F5000002114300FF0F0FE04F598404FF4FA627F
:105F6000643000210FF0E8FE04F5635C04F589401D
:105F7000E646E346012388F8003004F5A842CCF851
:105F80000C60034600F1120CCBF81060CEF814A0A0
:105F9000067446744FF0630E04F5635A00208CF8C3
:105FA00000E0DE74864689F800600AF1160382F884
:105FB00035605988002918BF7046ACF80200B3F864
:105FC00004B00EF10102BBF1000F18BF1046ACF88F
:105FD0000400B3F806A00EF10201BAF1000F18BFD9
:105FE0000846ACF80600B3F808B00EF10302BBF1A6
:105FF000000F18BF1046ACF80800B3F80AA00EF165
:106000000401BAF1000F18BF0846ACF80A00B3F853
:106010000CB00EF10502BBF1000F18BF1046ACF832
:106020000C00B3F80EA00EF10601BAF1000F18BF74
:106030000846ACF80E0033F810BF0EF107020EF15F
:10604000080EBBF1000F18BF1046BEF57A7F2CF882
:10605000100FAED140F2E73086464B46C4463CF8BE
:10606000021C002918BF704623F8020C3CF804AC4F
:106070000EF1FF3BBAF1000F18BF584623F8040C8D
:106080003CF8061CAEF10202002918BF104623F8A6
:10609000060C3CF808ACAEF10301BAF1000F18BFD2
:1060A000084623F8080C3CF80ABCAEF10402BBF128
:1060B000000F18BF104623F80A0C3CF80CACAEF1E8
:1060C0000501BAF1000F18BF084623F80C0C3CF884
:1060D0000EBCAEF10602BBF1000F18BF104623F84C
:1060E0000E0C3CF810ADAEF10701AEF1080EBAF19E
:1060F000000F18BF0846BEF1FF3F23F8100DAED1C8
:1061000004F5A54408F5A54809F5A54907F5A547EF
:10611000013D04F1240408F1240809F1240907F1E0
:1061200024077FF43DAD079D434E30680990099ADE
:106130003368039A089344F2904747F6A83642F62C
:10614000041C46F21C0B002482F8AF404BF2C02026
:1061500085F8784D4CF64C6105F80C404EF6D81396
:10616000EC5549F2347A05F80B40AC55009E05F821
:106170000A4001272C546C540198EC54029985F87C
:10618000A270049B86F86441059F069E089A80F8D9
:10619000F04081F87C401C7287F8944186F82041D9
:1061A000C5F8002195F85F4094B1EA7D82B995F871
:1061B0005C0068B995F8A31051B995F8A4303BB9C3
:1061C00095F8A77027B9012685F8A26085F8A76021
:1061D0000BB0BDEC028BBDE8F08F90F85E0000289C
:1061E0007FF4B2AB95F85D1000297FF4ADAB0026CB
:1061F00085F8A460FFF7A8BBD5F89870D5F894602F
:1062000085F8A13045F2A42303FB07F741F68C344F
:1062100004FB067CAC444FF0FF32CCF8BC21A5E473
:1062200090F85E2080F8A340002A7FF48DAB002612
:1062300085F8A460FFF788BBEC4401202DE9F04FFE
:106240002DED028B8146D0F80401DE4A8DB00D465B
:1062500010B913680893089811680991099C9FED7B
:10626000DA7A0294261A08EE106AF8EE487AC9F82B
:10627000044167EE878A09F1480421464822C9EDA6
:10628000428A48460DF018F82046482229460DF06B
:1062900013F899ED470ADFEDCD0AB4EEE00AF1EE0E
:1062A00010FA0ADD30EE681AB4EEE01AF1EE10FAD8
:1062B00048BFB0EE601A89ED471AD9ED481A9FED34
:1062C000C32AF4EEC21AF1EE10FA0ADD71EEE82AE2
:1062D000F4EEC22AF1EE10FA48BFF0EE422AC9ED00
:1062E000482A99ED493ADFEDB93AB4EEE33AF1EED6
:1062F00010FA0ADD33EE684AB4EEE34AF1EE10FA22
:1063000048BFB0EE634A89ED494AD9ED4A4A9FED4C
:10631000AF5AF4EEC54AF1EE10FA0ADD74EEE85A0F
:10632000F4EEC55AF1EE10FA48BFF0EE455AC9ED49
:106330004A5A99ED4B6ADFEDA56AB4EEE66AF1EED2
:1063400010FA0ADD36EE687AB4EEE67AF1EE10FA6B
:1063500048BFB0EE667A89ED4B7A99ED2B8A9FEDB6
:106360009B0AB4EEC08AF1EE10FA0ADD78EE687A84
:10637000F4EEC07AF1EE10FA48BFF0EE407AC9EDC3
:106380002B7AD9ED2C0A9FED911AF4EEC10AF1EEA9
:1063900010FA0ADD70EEE81AF4EEC11AF1EE10FA06
:1063A00048BFF0EE411AC9ED2C1A99ED2D2ADFED08
:1063B000872AB4EEE22AF1EE10FA0ADD72EE688A5C
:1063C000F4EEE28AF1EE10FA48BFF0EE628AC9ED0F
:1063D0002D8A7F4A7F4F92F806807D48CDF80C8049
:1063E000C17907EB880A6329DAF80060C9F81861F7
:1063F00040F21482784F0491A1F1640B07EB8B0CEF
:10640000DCF8003099F8008099F8051099F80FA091
:1064100099F8016099F80B2099F8060099F80CC0DA
:106420000A9409F5DF3B09F5E03ECBF8C430CBF820
:106430007831CEF82C30CBF8E830CBF89C31CEF860
:106440005030CBF80C31CBF8C031CEF87430CBF8EB
:106450003031CBF8E431CEF89830CBF85431CEF867
:106460000830CEF8BC3099F80A3099F807E0CDF83A
:106470002C9048EA0307394341EA0A01314399F86D
:10648000036099F81030019641EA020699F80280FB
:106490000093064399F8117099F80DA099F84800F7
:1064A00099F8081099F812200346A07A1843009B27
:1064B000334343EA080663791843E37B46EA0C0852
:1064C000667894F812C01843E37A3043A6791843EB
:1064D000304348EA0E03267C99F809E01F43A3786D
:1064E0003043267B1843019B3043E6791F43637C8E
:1064F0003043034347EA0A00E778667B99F819A01E
:106500003B43277A334301433B4399F80400267900
:1065100043EA0C070A4399F80E3099F81C1002431D
:1065200037431A4399F8136099F81D0099F8183009
:1065300042EA0E02324399F81A60009642EA0106D6
:1065400099F81B8099F814C099F815E099F816107D
:1065500099F817200643A07B33433843677A009E9F
:1065600043EA0A0AE37C38431843237F4AEA0607D2
:10657000667F184347EA0803277E94F81680304365
:10658000667E384343EA0C07A37E3043E67E184319
:10659000237D30430343607DE67D47EA0E070343D6
:1065A000394343EA08040A4344EA060752EA070C5F
:1065B00040F03A8199F8A23089F8A6C073B189F801
:1065C000A2C00BE0EC4401206F12833A00000000EF
:1065D0005C14FF1F8CA90100B4A90100B2484179E5
:1065E00007914E1EF4B2042C40F22B8199F816E06C
:1065F00099F814A02E7DA87D95F81E8099F81E406C
:1066000099F81F30E97F95F800C0CDF818E077467B
:106610008AEA0606784099F800E06A78304388EA0A
:106620000407074399F8014095F8028099F8026041
:10663000E878594039438CEA0E0341EA030C624082
:1066400099F8033095F804E099F80410AF7A4CEA11
:10665000020288EA06041443584099F80A2095F883
:106660000BC099F80B302E7B99F81880CDF8148068
:1066700020438EEA010101437A4099F80C0099F811
:106680000D7095F80DE099F81A4000940A438CEAD1
:106690000303134399F81C20019246408EEA070C2D
:1066A000AA7B99F80E70D9F82C00D9F830101E4347
:1066B0007A4046EA0C061643AB7E009A2F7E534082
:1066C0001E432A7F019B88EA070446EA040783EAFF
:1066D0000206EC6A2A6B6B6B374384420CBFB846E8
:1066E00047F00108D9F83460AC6BEF6B8A4218BFF1
:1066F00048F00108D9F83820B34218BF48F0010823
:10670000944218BF48F00108D9F83C402E6CD9F8E3
:106710004030A74218BF48F001089E420CBF4746D0
:1067200048F00107002F40F0A2806D6CD9F844209A
:10673000954240F09C8099F8A350A5B999F8A420FF
:106740008AB999F85D6076B199F815305BB999F816
:106750005E7047B999F86A30002B00F0E387012793
:1067600089F8A87092E09BF8AE50002D40F0A6800A
:1067700099F89080B8F1000F07D199F8624024B1E0
:1067800099F86020002A40F0DE8399F8F860002E26
:1067900040F01E8399F8FA70002F40F0C88099F8F5
:1067A000F930002B40F0B98499F8FB50002D40F0EF
:1067B0003B8309F151029FED3D3ACDF80880284610
:1067C00009F1560B494609F1C40E09F1BC0709F15C
:1067D0007C0509F1340409F10F0C09F10A0AC846D5
:1067E00091461BF8012F002A00F03B819CF80060C5
:1067F000002E40F00B8398F8A530002B40F0AD83BD
:106800003E7886F001033B700126294BCEF800301C
:10681000019688ED2B3AC8F8B80023E12248254BB1
:106820006922C2710492EDE599F8A220002A3FF492
:10683000D5AE4846FFF778F80DB0BDEC028BBDE849
:10684000F08F99F81471002F7FF4D0AE1A4A029994
:10685000D9F80C3152F82400CE1AB042B4BF012648
:10686000002689F81461B8BFC9F81011BEE699F87E
:10687000A760029BC9F80C3166B199F81461002534
:1068800089F8A75016B1002489F81441012089F82D
:10689000A200CEE799F81471002FF4D199F8A35013
:1068A000002D7FF460AF49E75C14FF1FCDCCCC3ED8
:1068B000F1D8FFFFD2AB413DC8AD010099F860604F
:1068C00016B9059D002D55D199F8627017B9009B36
:1068D000002B4FD199F8642012B9019E002E49D1A6
:1068E00099F85C50002D3DD0BAF1000F3AD199F8DB
:1068F000AA20013202F0030689F8AA60D9F8745080
:10690000D9F87870281A791A03B20AB2002B00F06D
:1069100020831344002B99F8AA6040F38E83032E42
:1069200087D8DFE816F0C703B703D6039903D9ED7C
:106930003B0A89F8F960F5EEC00AF1EE10FA40F36F
:106940001B8399ED421A70EEC11AF5EEC01AF1EEF2
:1069500010FAC9ED3B1A3FF66CAF89F8FA6089F876
:10696000FC6066E799F85E70002FC7D0069B002B8D
:10697000C4D1BCE75F4F604CDFF898A15F4E97E849
:106980000F004FF001084FF0000E89F8A2808BF83D
:10699000AEE089F8A08084E80F00594FDFF89CB181
:1069A000DBF80080574D0DF0D3FA044604E00DF0FB
:1069B000CFFA031BAB42F3D83068C107F7D4524972
:1069C000524BC1F800804B600DF0C2FA4D4C0546A9
:1069D00004E00DF0BDFA401BA042E1D83A684C48F3
:1069E00010400028F5D0464B454D1968CAF80010F4
:1069F0002960DAF80040464B46492340012BCFD1AD
:106A0000454A1068C205CBD5444C454F23703E4ED5
:106A1000444D454A454800230B6045493960336081
:106A20004FF481362E60434D1060FD600DF090FAFA
:106A3000344E074604E00DF08BFAC21BB24209D86F
:106A40002378002BF7D1DAF8004038492140022999
:106A50003FF4EFAE4FF40272332137480CF0DCFA0A
:106A6000E7E6019219F8016F002E69D19AF80060EB
:106A700006B35AB99CF8003043B12A682668931BC4
:106A80001DD098F8A520002A65D061E098F8A530BF
:106A900083B94FF0010681F8786D3B78002B00F048
:106AA000228491F97A6D002E40F0C0854FF0630387
:106AB00081F87A3D26682B689B1B40F04082019A42
:106AC000002A69D03B78002B40F0498291F97B6D18
:106AD0003344632B00F31F83002B40F31983322BC5
:106AE00000F017831A46B342CEF8002054D081F844
:106AF0007B3D4DE05C14FF1F8CFF002024100B40F9
:106B000030100B4040420F0008100B4000001A0DDF
:106B100001000F00D044012010100B40D44401208C
:106B200000100B4004100B4038100B4002007F1186
:106B300080FF002027003A194CFF0020D844012094
:106B40002A682368D31ABAD04FF0010688F8A560E6
:106B500003EB83035B003A78002A00F05A81112B83
:106B600091F97A6D40F3F38212233344622B00F3E0
:106B7000DA8113F1620FC0F2F6815AB281F87A2DF0
:106B8000002B40F0D781A64BCEF80030B24203D0A4
:106B90004FF0010681F8786D013001F5A541052817
:106BA00001F124010EF1040E07F1010705F10405BE
:106BB00004F104040CF1010C0AF1010A45F2A423CA
:106BC0007FF40FAEC146DDF8088099F8A2000028D6
:106BD0007FF42FAEB8F1010F00F02884B8F1000F58
:106BE0007FF427AE4846FEF763FD00287FF421AE10
:106BF00099F8481039B999F8004024B199F8A6508D
:106C0000002D01F0328099F849703FB999F80120C0
:106C100022B199F8A660002E01F0618099F84A30FF
:106C20003BB999F8020020B199F8A610002901F0AB
:106C3000658099F84B403CB999F8035025B199F813
:106C4000A670002F01F05C8099F84C2042B999F8A9
:106C500004602EB199F8A6300424002B01F00680C0
:106C600099F8A240002C7FF4E4AD99F84850E5B1C2
:106C700099F86070002F40F0828799F86220A2B1E5
:106C800099F81A308BB945F2344B44F2904119F817
:106C90000B406448012784F0010509F80B5009F8FE
:106CA000017089F8A670C9F8B00099F8496006B378
:106CB00099F8602022B199F81830002B00F07B87FA
:106CC00099F86210A9B199F81A4094B94AF2D865B6
:106CD00049F2347719F8056052484FF0010E86F0FA
:106CE000010C09F805C009F807E089F8A6E0C9F821
:106CF000B00099F84A50FDB199F8607027B199F841
:106D00001860002E00F06F8799F86200A0B199F822
:106D10001A1089B94FF67C154EF6D81C19F80520C3
:106D2000404C012382F0010E09F805E009F80C300F
:106D300089F8A630C9F8B04099F84B20002A00F035
:106D4000678799F8603023B199F81870002F00F028
:106D5000738799F86260002E00F05A8799F81A102C
:106D6000002940F0558709F5A63A09F59E3B9AF8A7
:106D700020502C4C4FF0010C85F001028AF82020A5
:106D80008BF87CC099F84C0089F8A6C0C9F8B040CF
:106D900000283FF44EAD99F86000002800F0B58758
:106DA00099F81840002C40F0B08709F5C13B09F56F
:106DB000B93C9BF838511B4C012085F001028BF83F
:106DC00038218CF8940189F8A600C9F8B44030E560
:106DD00099ED3B2AB5EEC02A0027F1EE10FA89F8AA
:106DE000FA7089F8F97040F3C781D9ED422A72EE42
:106DF000628AF5EEC08AF1EE10FAC9ED3B8A3FF6E1
:106E000018AD89F8F87089F8FC7012E50023019339
:106E100028E6112B91F97B6D40F3A880122357E6E9
:106E2000F1D8FFFFCDCC4C3ED9F874301E1A002E9D
:106E300040F30E8102270126D9F87820551A002D3B
:106E400040F3AE81D9F8984009EB840B0BF5CF3CA9
:106E5000DCF8E830F918012940F3D88302218B428D
:106E60000FD045F2A42606FB049E0027BB4DCBF8AD
:106E700030714FF00108CCF8E810CBF81C518EF8B7
:106E8000788D99F8482022B199F80000002800F088
:106E9000D48499F8494024B199F80130002B00F0CE
:106EA000CC8499F84A1021B199F80260002E00F0C4
:106EB000C48499F84B7027B199F80350002D00F065
:106EC000BC8499F84C4024B199F80420B2FA82F0BD
:106ED000440999F860301BB90599002940F00481F4
:106EE00099F862601EB9009F002F40F0FD8099F86C
:106EF00064501DB9019A002A40F0F68099F85C00B0
:106F000018B9BAF1000F40F0EF8099F85E301BB964
:106F10000699002940F0E880002C3FF48AAC002458
:106F200089F8FB4085E4632212F1630F81F87A2D22
:106F30003FF429AE632A3FF426AE134624E6002A26
:106F40007FF402AE9DE5012289F8A2208BF8AE20E5
:106F50006FE4002A7FF4DDAC6BE4019682E591F9E1
:106F60007A6D002301E66FF06202DDE713F1110F85
:106F7000B8BF6FF01103ABE599F85C3089F8FC609D
:106F80001BB9BAF1000F40F0FF8099F860401CB9BE
:106F9000059E002E40F0F48499F862501DB9009FC0
:106FA000002F40F0B58599F8640018B9019A002ABD
:106FB00040F0CE8599F85E1000297FF43AAC069B2C
:106FC000002B3FF436ACD9F8F46045F2A42404FB5E
:106FD000069A10250AF5EA5089F8FC50FAF774F879
:106FE000D9F8F47004FB07F709EB070B42F6041815
:106FF00001260BF563500C300BF80860FAF764F8C3
:10700000D9F8F40004FB00F009EB000144F29042CF
:1070100001F5DA708E54F9F7CDFED9F8F45004FB7F
:10702000059484F8786D99F8FC70002F3FF401AC5A
:107030004B4BC9F8EC30FFF7FCBB14BF4FF0FF34EB
:107040000024032E3FF6F5ABDFE806F058565A074A
:1070500040F09E800127EFE6012442480079FDF7C9
:1070600093FB031940F0F18284EAE472A2EBE47628
:10707000751E002E40F035860121002C03DC013105
:10708000FE29A8BFFE21CBB2364989F8A9300B7181
:10709000FFF7CFBB4FF0010B049858446C28034610
:1070A00000F3D1826428B8BF6423D9B22D4CE171BA
:1070B000FFF7BFBB4FF0010C039A2A4D6244082A28
:1070C0001646DABF22EAE276F6B20926AE71FFF77B
:1070D000B0BB079C052C00F29782234F17F8245071
:1070E000204F7D71FFF7A5BB002689F8FB60002CBF
:1070F0003FF4CCABFFF79DBBA346CDE7A446DBE74F
:10710000079C052C00F28082184E16F82450E7E701
:107110000023174AE7E46423FBE799ED3B8AB5EEC9
:10712000C08AF1EE10FA40F39A8099ED420A78EEA7
:10713000407AF5EEC07AF1EE10FAC9ED3B7A3FF6EF
:1071400078AB89F8F97089F8FC70FFF772BB13F11E
:10715000110FB8BF6FF0110307E500BF0AD7233C3A
:10716000CDCC4C3E5C14FF1FDCA9010000AC01003B
:10717000F1D8FFFF00C0794499F85C6089F8FC7091
:10718000B6B9BAF1000F13D0012789F8FC704FE7A8
:10719000D9F87800451A002D3FF773AE4FF0FF364F
:1071A000002D0CBF3746771E002F3FF46AAE49E62C
:1071B00099F8601031BB059D25B3D9F8F440D9F892
:1071C000F05045F2A42B0BFB049C0BFB05980CF52F
:1071D000EA5008F5EA510227884289F8FC7007D086
:1071E00041F68C320CF068F8D9F8F44099F8FC704C
:1071F00045F2A42E0EFB049A42F6041101200AF86F
:10720000010012E799F86220002A77D1009800283F
:1072100074D0D9F8F440D9F8F05045F2A42101FB1C
:10722000049A01FB059707F563510AF563500C308A
:107230000C310427884289F8FC7007D041F68C3263
:107240000CF03AF8D9F8F44099F8FC7045F2A42013
:1072500000FB049344F2904201269E54E5E699F81F
:107260005C5089F8FC7015B9BAF1000F8CD199F80F
:107270005E70002F7FF4DDAA069A002A3FF4D9AA97
:10728000D9F89800D9F8F410D9F8F03045F2A424D0
:1072900004FB00F041F68C3A0AFB010B0AFB030CDD
:1072A000CC4409EB0B0E0CF5DA710EF5DA701026F2
:1072B000884289F8FC6000F0B28452460BF0FCFF73
:1072C000D9F89870D9F8F40099F8FC2004FB07F479
:1072D0000AFB0048C844012188F8781D002A7FF481
:1072E000A7AEFFF7A6BA91F97B6D002E40F0928110
:1072F0004FF0320381F87B3DFFF7DCBB99F8644027
:107300002CBB019B1BB3D9F8F420D9F8F04045F20F
:10731000A42303FB029B03FB049C0BF5DA700CF522
:10732000DA710827884289F8FC7007D041F68C3260
:107330000BF0C2FFD9F8F42099F8FC7045F2A426AE
:1073400006FB02984FF0010E88F878ED6DE699F88B
:107350005E70002F7FF46DAA069E002E3FF469AA8E
:10736000D9F8F420D9F8F03045F2A42B0BFB029C9D
:107370000BFB03980CF5EA5008F5EA5110258842FA
:1073800089F8FC5007D041F68C320BF095FFD9F804
:10739000F420D9F8F03045F2A42E0EFB02FA09EBE6
:1073A0000A000EFB039101F5635100F56350CA44D6
:1073B00042F604140C310C30012788420AF804709C
:1073C00007D041F68C320BF077FFD9F8F420D9F8CA
:1073D000F03045F2A42606FB02F509EB050C06FB8E
:1073E000039B44F290470BF5DA710CF5DA70012437
:1073F00088420CF8074007D041F68C320BF05CFF56
:10740000D9F8F420D9F8F03003F5CF463A3645F2F2
:10741000A42E02F5CF410EFB029A3A3159F82650BC
:1074200001208AF8780D49F82150FCE5D9F89870C8
:10743000D9F8946003FB07F341F68C3101FB063861
:1074400008F5D8734B44191D002E00F06281C9F86D
:107450009C605D685FEDB93AAF4C9FEDB04A04EEB9
:10746000905AB8EEE45A45F2A422C5EE235A02FB24
:1074700007F741F68C3000FB067A09EB450BDA443E
:10748000BB44BAF8C071BBF8C061009A40F2E73360
:1074900003FB07F384FB030C06EE106AF8EE466A62
:1074A0009C44DD1726EE847AC5EBEC34C9F8A44180
:1074B00089ED6A7AC9ED6B5A002A40F0CD80059FAC
:1074C000002F40F0C38199F84800002800F0708236
:1074D00099F86020002A00F0D18243F6A80799F8B5
:1074E000494019F807508E4AC9F8B42042F60416EC
:1074F000012385F0010E09F807E009F8063089F844
:10750000A630002C00F0D38248F64C3799F84A4058
:1075100019F80750824AC9F8B42047F6A836012363
:1075200085F0010A09F807A009F8063089F8A630A5
:10753000002C00F05F824DF6F05A99F84B6019F874
:107540000A30774FC9F8B4704CF64C604FF0010B1D
:1075500083F0010509F80A5009F800B089F8A6B0CF
:10756000002E00F0C68209F5983A09F5903B9AF88A
:1075700094206B4F012482F001008AF894008BF86C
:10758000F04099F84C3089F8A640C9F8B4708BB136
:1075900009F5C13E09F5B9369EF83821604D012044
:1075A00082F001078EF8387186F8940189F8A600F8
:1075B000C9F8B45099F8A640002C7FF43AA999F87C
:1075C0006130002B40F0788399F86360002E40F022
:1075D000738399F86520002A00F06E8399F81D5096
:1075E000002D40F0698399F8A1704FF0010A89F8E5
:1075F000A2A027B14FF0FF3089F8A1508860012187
:1076000089F8FB10FFF715B9002569E50CBF0121CA
:10761000002124E4322E00F01381642E00F09182C8
:107620004FF0000381F87B3DFFF744BA632E00F072
:10763000878116F1630300F0F8824FF0000381F8B0
:107640007A3DFFF737BA6D2130E50F2BC8BF102404
:1076500040F34E83FF2110E505980028AAD199F840
:107660004870002F00F0718199F86060002E00F0E2
:107670006C8143F6A80E99F8494019F80E70284A13
:10768000C9F8B42042F60410012387F0010609F876
:107690000E6009F8003089F8A630002C00F05D81FA
:1076A00048F64C3799F84A4019F807801C4AC9F83F
:1076B000B42047F6A836012388F0010A09F807A08C
:1076C00009F8063089F8A630002C00F04E814DF6FE
:1076D000F05799F84B4019F807B0114AC9F8B4208F
:1076E0004CF64C6601238BF0010C09F807C009F831
:1076F000063089F8A630002C7FF435AF99F84C504D
:10770000002D3FF457AF99F8600000287FF440AF98
:1077100050E7D9F89C609CE60180008080008037AB
:10772000CDCC4C3E46F21C0647F6A83549F23474DF
:107730004BF2C02042F6041C44F2904E8BF8AF305E
:107740004CF64C6289F8783D4EF6D81109F80C30A9
:1077500009F5823A09F80E3009F5903809F8063033
:1077600009F59E3709F8053009F5AC3609F80430FB
:1077700009F5B93509F8003009F5C73499F8A100C1
:1077800009F8023009F801308AF8643188F8F030DD
:1077900087F87C30337285F8943184F8203190B1C9
:1077A000D9F89810D9F8942089F8A13045F2A4238B
:1077B00003FB01F341F68C3000FB023CCC444FF05C
:1077C000FF31CCF8BC1109F5D872CF491E20F9F76A
:1077D0006DFE00287FF45AA88BF8AF0042F6041E15
:1077E00046F21C0244F2904B89F8780D47F6A83314
:1077F00009F80E0049F2347109F80B004BF2C02C65
:1078000009F802004CF64C6E4EF6D81209F8030047
:1078100009F8010009F80C0009F80E0009F8020047
:107820008AF8640188F8F00087F87C00307285F8E7
:10783000940184F82001FFF729B80124FFF749BB20
:107840004FF0640681F87B6DFFF734B999F8486012
:10785000002E00F0F98099F86220002A00F0F480F0
:1078600045F2344E99F8497019F80E50A748C9F8F6
:10787000B00044F290484FF0010A85F0010609F883
:107880000E6009F808A089F8A6A0002F00F0E48097
:107890004AF2D86B99F84A0019F80B309B4DC9F899
:1078A000B05049F2347C012683F0010709F80B70CF
:1078B00009F80C6089F8A660002800F0D5804FF622
:1078C0007C1E99F84B5019F80EA0904BC9F8B030B7
:1078D0004EF6D81801278AF0010009F80E0009F8C1
:1078E000087089F8A670002D00F0A38009F5A63B6A
:1078F00009F59E3C9BF82060844A012486F0010330
:107900008BF820308CF87C4099F84C5089F8A640D0
:10791000C9F8B020002D3FF44DAE09F5CF3C09F574
:10792000C73E9CF8C430794F012583F001068CF8DE
:10793000C4608EF8205189F8A650C9F8B07039E6B5
:107940009D2681F87A6DFFF7B5B899F8493023B1D3
:1079500099F86050002D7FF4A3AE99F84A5025B1F4
:1079600099F8600000287FF4B2AE99F84B50002DD2
:107970003FF4C4AE99F8600000283FF41BAEF2E576
:10798000D9F8F41045F2A42505FB019E02220EF55C
:10799000EA5089F8FC20F9F797FBD9F8F40042F691
:1079A000041405FB009A01230AF80430FFF73BBBDF
:1079B00099F84970002F7AD099F86060002E7FF412
:1079C000A3AD99F862708FB14AF2D86249F2347C63
:1079D00019F802604D4C012386F0010509F80250A8
:1079E00009F80C3089F8A630C9F8B04099F84A0077
:1079F000002867D199F84B0000287AD099F8607078
:107A0000002F7FF4B0AD99F8627097B109F5A63BED
:107A100009F59E3C9BF820603C4D4FF0010E86F02E
:107A200001028BF820208CF87CE089F8A6E0C9F8E8
:107A3000B05099F84C40002C3FF4BCAD99F862006E
:107A400000283FF4B7AD68E799F8494024B199F8A8
:107A50006230002B7FF41CAF99F84A2022B199F8CC
:107A60006240002C7FF42BAF99F84B20002AE0D025
:107A700099F86240002C3FF49DAD37E799F86270A9
:107A80008FB145F2344844F2904419F808A01F4DD4
:107A900001238AF0010B09F808B009F8043089F8CD
:107AA000A630C9F8B05099F8490000288BD199F850
:107AB0004A0000289ED099F86070002F7FF43BADFB
:107AC00099F862708FB14FF67C124EF6D81819F8FB
:107AD00002600E4D012386F0010409F8024009F806
:107AE000083089F8A630C9F8B05099F84B00002842
:107AF0008BD199F84C20002A3FF45CAD99F8604096
:107B0000002C7FF445AD99E74C9D0100CDCC4C3E57
:107B1000D9F8F42045F2A42505FB029C0CF563502E
:107B20004FF004080C3089F8FC80F9F7CDFAD9F849
:107B3000F43044F2904405FB039701263E55FFF7CD
:107B400072BADEF80030804EB3427FF46BAD67E569
:107B5000D9F8F47045F2A42606FB079E08210EF51D
:107B6000DA7089F8FC10F9F725F9D9F8F40006FB6A
:107B7000009A4FF0010B8AF878BDFFF754BA99F8D4
:107B80001860002E7FF479A843F6A80899F84940B8
:107B900019F808A06D4AC9F8B42042F6041101236F
:107BA0008AF0010B09F808B009F8013089F8A6300D
:107BB000002C3FF49EA848F64C3799F84A0019F873
:107BC0000710624DC9F8B45047F6A8364FF00108C7
:107BD00081F0010409F8074009F8068089F8A680B9
:107BE00000283FF4A9A84DF6F05799F84B1019F862
:107BF0000780564BC9F8B4304CF64C66012488F027
:107C0000010509F8075009F8064089F8A64099B916
:107C100099F84C20002A3EF40CAEFFF7BCB8CB44D8
:107C200001258BF8785DFFF703BADEF80030464E89
:107C3000B3427FF404AD00E509F5983A09F5903BAD
:107C40009AF89470414E012187F001038AF894302C
:107C50008BF8F01099F84C5089F8A610C9F8B46068
:107C6000002D7FF49DA8FEF7E4BD444699F8A100DD
:107C700099F8901089F89110012589F8905098B1E1
:107C8000D9F89870D9F8946045F2A42202FB07F263
:107C900041F68C3303FB062ACA4400204FF0FF3123
:107CA00089F8A100CAF8BC1100214846FCF7B6FDCE
:107CB000C9F89840FEF7D4BF4846FDF7F9FC002804
:107CC0007EF4B7AD4846FCF733FF99F8A240002C8C
:107CD0007EF4AFAD4846FDF78FFCFEF7AABD012448
:107CE000C4E71B4F57F8250040F00101FFF7C5B965
:107CF00013F10F0F06DA6FF00F04ABE40224B5E7BF
:107D00000324B3E71C46FFF7AFB999F86220002AB5
:107D10003EF48FAD99F81A0000287EF48AAD09F57B
:107D2000CF3E09F5C7389EF8C470084E012187F090
:107D300001038EF8C43088F8201189F8A610C9F81C
:107D4000B060FEF776BD00BFF1D8FFFFCDCC4C3E52
:107D5000F4A90100F0B400230B604B608B60CB6092
:107D60000B614B61D0F8982084B0002A00F0298282
:107D700090F84840DFEDB36A9FEDB37A00F5E03547
:107D8000D5ED337A8C7227EEA60AB4EEC70AF1EE6F
:107D900010FA0CD5B5EEC00AF1EE10FA40F33082BD
:107DA000FCEEC00ACDED010A9DF8046000E0FF265C
:107DB0000E7095ED381ADFEDA31A9FEDA32A61EE40
:107DC000212AF4EEC22AF1EE10FA15D5F5EEC02AFA
:107DD000F1EE10FA40F30682BCEEE23A8DED013A84
:107DE0009DF804704F71D0F89830012B0AD190F8AB
:107DF0009020012A06D107E0FF274F71D0F8983074
:107E0000012BF4D090F84920CA72D5ED343A9FED99
:107E10008D4ADFED8D4A23EE845AB4EEE45AF1EE3A
:107E200010FA0CD5B5EEC05AF1EE10FA40F3DC8131
:107E3000FCEEC55ACDED015A9DF8044000E0FF2448
:107E40004C7095ED396ADFED7F7ADFED7F6A26EEC3
:107E5000277AB4EEE67AF1EE10FA15D5B5EEC07ACF
:107E6000F1EE10FA40F3C281BCEEC70A8DED010AB3
:107E70009DF804608E71D0F89870022F0AD190F8A6
:107E80009030012B06D107E0FF268E71D0F8987054
:107E9000022FF4D090F84A300B73D5ED350A9FEDE0
:107EA000691ADFED691A20EE812AB4EEE12AF1EEBB
:107EB00010FA0CD5B5EEC02AF1EE10FA40F390811D
:107EC000FCEEC22ACDED012A9DF8042000E0FF223D
:107ED0008A7095ED3A3ADFED5B3A9FED5B4A63EECF
:107EE000234AF4EEC44AF1EE10FA15D5F5EEC04A75
:107EF000F1EE10FA40F37281BCEEE45A8DED015AB6
:107F00009DF80440CC71D0F89860032E0AD190F807
:107F10009070012F06D107E0FF24CC71D0F8986053
:107F2000032EF4D090F84B704F73D5ED365A9FED79
:107F3000456ADFED456A65EE867AF4EEE67AF1EEA3
:107F400010FA0CD5F5EEC07AF1EE10FA40F352813A
:107F5000BCEEE77A8DED017A9DF8043000E0FF2356
:107F6000CB7095ED3B0ADFED370A9FED371A60EED7
:107F7000201AF4EEC11AF1EE10FA15D5F5EEC01A7A
:107F8000F1EE10FA40F33881BCEEE12A8DED012AC2
:107F90009DF804200A72D0F89840042C0AD190F879
:107FA0009060012E06D107E0FF220A72D0F89840B7
:107FB000042CF4D090F84C608E73D5ED372A9FEDE9
:107FC000213ADFED213A22EE834AB4EEE34AF1EEA4
:107FD00010FA0CD5B5EEC04AF1EE10FA40F3088164
:107FE000FCEEC44ACDED014A9DF8047000E0FF2785
:107FF0000F7195ED3C5ADFED135A9FED136A65EE54
:10800000256AF4EEC66AF1EE10FA1FD5F5EEC06AE5
:10801000F1EE10FA40F3F280FCEEE67ACDED017A53
:108020009DF804504D7290F89020012A14D1D0F898
:108030009460002E40F0CB804A740027012E0F740C
:108040000DD10DE000807F4300007F43FF254D727E
:1080500090F89020012AEAD000234B740B7400267C
:1080600090ED2C0ACE73B5EEC00AF1EE10FA0CDDDD
:10807000B2EE0E7A60EE070ABDEEE01A11EE105A6B
:1080800005F0010282F001030B74D0ED2D1AF5EE1C
:10809000C01AF1EE10FA0CDDB2EE0E2A61EE822A61
:1080A000BDEEE23A13EE106A06F0010484F0010717
:1080B000CF7300F5DF3C9CF8AF50002D40D142F665
:1080C000041244F29046875C90F8783D825D46F257
:1080D0001C0447F6A835045D455D3B4349F23477FF
:1080E00013434BF2C026C25D865D23434CF64C64BD
:1080F0002B434EF6D8151343025D455D00F58237DC
:10810000334300F5903613432B4397F8642196F8D8
:10811000F07000F5AC3500F59E36134396F87C20E0
:108120002E7A00F5B9353B4300F5C737134395F870
:10813000942197F82071334313433B438CF8AF30BD
:10814000304B90F86A601C680394039AC2F30805E8
:108150001EB390F86B3053BB8B7490F8A9404C75EC
:1081600090F8A020002580F8A9501AB101270F75BA
:1081700080F8A05090F8A86090F86B30CB7536B1BD
:1081800083F001044FF0000CCC7580F8A8C090F883
:10819000A700887504B0F0BC70479CF8AF7027B199
:1081A000B5F5807F94BF002701278F74D5E79CF831
:1081B000AF60002ED0D0B5F5807F8CBF00230123A7
:1081C000CAE790F89040012C7FF4D2ADD2E50024AC
:1081D000022E4C747FF431AF0A7440E700249CE611
:1081E000002275E6002708E6002429E600264CE672
:1081F0000027FDE60023B3E60022D6E6002526E7A9
:108200000026D5E5EC4401202DE9F04F2DED048B3F
:1082100085B000F5E03E531EDFEDEE5ADFEDEE3A9D
:108220009FEDEE4A9FEDEE5A9FEDEE3ADFEDEE2A1E
:108230009FEDEE2A029306320EF1CC0C04460EF1AD
:10824000E00E00F5C079054607460026B7EE006A45
:1082500001920A8807EE902A07F5DF33F8EE670AE5
:10826000D3ED306A93ED347A70EEE64A04F5CF38F8
:10827000F0EEE41AF4EEC71AF1EE10FA03F1C00AB8
:10828000D8F8E88000F3908136EEE01A93ED338A57
:10829000D3ED318AB0EEC19AF0EE469AE9EE089A33
:1082A00003F1BC0B69EEA80AF4EE460AF1EE10FAEF
:1082B000C8BFF0EE460AE0EEA46ACAED006A93ED8C
:1082C0002F1A93ED2E7A71EE471AF4EEE16AF1EE71
:1082D00010FA40F15D8136EE871A83ED2F1AD3ED47
:1082E0002C6A93ED328AD3ED2D0A77EE268AF0EED2
:1082F000669A31EE689AE9EE089AF4EEE09AF1EEA9
:1083000010FA08D5F4EEE96AF1EE10FA54BFF0EE77
:10831000660AF0EE690A4A8993ED5D7AD3ED616AE7
:1083200001EE102AB8EE418A60EEA54A78EE471AAF
:1083300003F5BA7AF0EEE18AF4EEE68AF1EE10FA8D
:1083400000F3138137EE489AB0EE478AD3ED609A76
:10835000D3ED5E7AB0EEC91AF0EE460AE1EE290AD4
:1083600003F5B87B60EEA76AF4EE466AF1EE10FA08
:10837000C8BFF0EE466AA6EEA18A8AED008AD3ED68
:108380005C8A93ED5B9A78EEC91AB4EEE18AF1EE5D
:1083900010FA40F1F18078EE098AC3ED5C8AD3EDE2
:1083A000590A93ED5F1AD3ED5A6A79EE207AB0EE4E
:1083B000607A38EEE78AA8EE017AB4EEE67AF1EE5A
:1083C00010FA08D5F4EEC70AF1EE10FA54BFF0EE39
:1083D000606AF0EE476A8B8A09EE103A07F5E032E0
:1083E000F8EE499AD2ED0A7AD2ED0E1A39EEE71A72
:1083F00066EEA56AF0EEC10AF4EEE10AF1EE10FABB
:1084000002F1280A00F3AA8037EEE98AF0EE679AB3
:1084100092ED0D7AD2ED0B8AB0EEC89AF0EE467A64
:10842000E9EE077A02F1240B67EEA80AF4EE460A99
:10843000F1EE10FAC8BFF0EE460AE0EE819ACAEDFE
:10844000009A92ED098A92ED087A38EE471AF4EE16
:10845000C19AF1EE10FA40F1B08039EE878A82EDD0
:10846000098A92ED069AD2ED0C0AD2ED071A77EE40
:10847000097A78EE679AB0EE498AA9EEA08AB4EE3E
:10848000E18AF1EE10FA08D5B4EEC89AF1EE10FACE
:1084900054BFF0EE491AF0EE481A95F97B3D95F974
:1084A0007A2D01EE103A08EE902AB8EEC19AF8EE55
:1084B000E80A61EEA59A69EE237A20EE848AE9EE55
:1084C000887AF4EEC67AF1EE10FA00F19B80B8F1EA
:1084D000000F00F04E83F7EE007AB8F1010F00F0C4
:1084E000C882B8F1020F00F0E781019BDFED3F4A3F
:1084F0001B88D4ED4C7AF5EE407AF1EE10FA07D0F5
:1085000024EEA71AB5EEC01AF1EE10FA40F2368347
:108510004FF00008029A02F8018FC4F88831019BDD
:10852000C4ED4C4A013605F5A5450233052E0292ED
:1085300005F1240501F1020104F1040407F1240707
:1085400009F1010901930CF1040C0EF1040E7FF402
:1085500080AE05B0BDEC048BBDE8F08F39EEE91AB2
:10856000C2ED0A9AB0EE418A52E778EE481A83EDDE
:108570005D8AB0EE619AE9E678EE899AB4EEE98A0E
:10858000F1EE10FAC4BF78EE498ACBED008A06E717
:1085900071EE074AF4EEE46AF1EE10FAC4BF36EE6B
:1085A000C71A8BED001A9AE670EEE04AF0EE606AA8
:1085B000B0EE641AC3ED300A68E678EE078AF4EE8E
:1085C000E89AF1EE10FAC4BF39EEC78A8BED008A43
:1085D00047E700BF800080370AD7233CB57E253CA3
:1085E00000C079446F12833A80FF7F47000000008B
:1085F000AAD71F395F7089306666663F0534833AB3
:1086000000247449F5EEC07AF1EE10FA40F382834B
:10861000B8F1000F7FF461AF77EEA77AB0EE001AE1
:1086200031EE677AB4EE467AF1EE10FAF4EE467A5D
:10863000C8BFB0EE467AF1EE10FAC8BFF0EE467A47
:10864000D0F898208CED007A24EE871A66EEA71AEF
:10865000B242CEED007A04BF80ED681AC0ED671A11
:10866000D4ED519A31EE698AB5EEC08AF1EE10FA76
:1086700040F3A882F7EE004A4FF0010869EE857AD0
:10868000F5EEC07AF1EE10FA40F29082F4EEC57A7F
:10869000F1EE10FA28DB45F2A42202FB06F241F6C5
:1086A0008C3B0BFB08220244B2F88EA9D4ED478A1A
:1086B000F5EEC08AF1EE10FA4ADD5FED2F6A60EE4A
:1086C000268AB0EEC89AB4EEE89AF1EE10FA40F2BB
:1086D000B280B5EEC08AF1EE10FA40F37B83B7EEBC
:1086E000008AE8EE889AA8E0FDEEE76A42F6521B9F
:1086F0000BFB06F240F6C65A16EE90BA0AFB0823A8
:108700005B4400EB4302F8EEE68AB2F8C031B2F8FF
:10871000C22107EE103A09EE102AF8EE476AB8EEC9
:10872000497A77EEE88A37EE669AF6EE000AE9EEC5
:10873000286AD4ED478A76EEA06AF5EEC08ABCEED0
:10874000E67AF1EE10FA8DED037ABDF80CA0B4DCF8
:1087500045F2A42202FB06F241F68C3B0BFB0828F3
:10876000804408F5E8531C331A78002AA5D109EE95
:1087700010AA1FED617A5FED610A5FED5F8AF8EE86
:10878000C96AE6EE870AC6EE206AB0EEE69AB4EE53
:10879000E89AF1EE10FA92DDFDEEE79AF5EEC04AA6
:1087A00019EE902AF1EE10FA40F2E6334CBF4FF08A
:1087B000020A4FF0010A9A4221EE058A2FDCFDEEF3
:1087C000C86A22EAE27216EE90BA9B452FDD40F2AB
:1087D000E73B42F65213BAF1010F03FB062800F003
:1087E000BC8208F50952083200EB420A5FED7E0AAE
:1087F000BAF804201FED7F7A9345B8BF934608EE80
:1088000090BAB8EEE89A79EE209A69EE879AF5EE7A
:10881000C09AF1EE10FAB8BFF0EE429A0DE0FDEE0C
:10882000C87A17EE90BA9B4505DC40F2E7322BEA96
:10883000EB7B9345CDD1F0EE419A31EE691A61EEB2
:10884000850AF0EEC17AF4EEC37AF1EE10FAC8BFF1
:108850000122F5EEC00AC4ED519AC8BF89F8002084
:10886000F1EE10FA40F29D81F4EEC50AF1EE10FA35
:10887000C0F2D480B5F88E8906EE908AF8EEE68ACA
:108880004FF6FE7328EEA59AF4EEC99AF1EE10FAAF
:10889000D8BFF0EE499A69EEA29ABDEEE98A18EEC9
:1088A000102A9A4200F3B68022EAE2731FFA83FB91
:1088B000019AA2F800B01CE676EEE41AD0F89820EF
:1088C000E1EEA74AB24236EE671A64EE858A8CED75
:1088D000001AF5EEC08ACEED007A04BFC0ED684AFA
:1088E000C0ED674AF1EE10FA40F27982F4EEC58AE3
:1088F000F1EE10FA80F24F82BDEEE89A42F652187D
:1089000019EE103A08FB063200EB420AB8EEC98AAB
:10891000BAF8C031BAF8C22100EE903A09EE902AB6
:10892000B8EE607AF8EE696A78EEC84A76EEC71A51
:10893000F6EE007AA4EEA17A37EE271AFCEEC18A91
:10894000CDED038ABDF80C8009EE108AF8EEC90A55
:1089500094ED517A60EEA51A71EEC79AF5EEC09AC1
:10896000F1EE10FA40F35283F7EE004A4FF0010B9C
:1089700067EE057AF5EEC07AF1EE10FA40F23A832E
:10898000F4EEC57AF1EE10FAC0F2808245F2A42A24
:1089900041F68C380AFB06F208FB0B230344B3F8BC
:1089A0008E89D4ED476AF5EEC06AF1EE10FA40F315
:1089B000A2825FEDED8A20EE281AF0EEE90AB4EE0D
:1089C000E01AF1EE10FA80F20C83F5EEC09AF1EEA7
:1089D00010FA40F37683B7EE008AA1EE087A67EECC
:1089E000229AFDEEE97A17EE902A71EEC71A4FF639
:1089F000FE73F0EEE18AF4EEC38AF1EE10FAC8BF1E
:108A00004FF0010884ED517AC8BF89F800809A427E
:108A10007FF74AAF4FF6FF739B4649E7BDEEE07A1A
:108A200042F6521B17EE102A0BFB062A00EB4A08EF
:108A3000F8EEC78AB8F8C0B1B8F8C22101EE90BA12
:108A400006EE902AB8EE619AB8EE668A70EEE87A81
:108A500038EE491AF6EE000AA7EE819A39EE207A2E
:108A6000FCEEC71ACDED031ABDF80CA006EE90AAD5
:108A700004E736EEE41AD0F89820E1EE274AB24235
:108A800076EE670AF0EE641ACCED000ACEED007ABD
:108A900004BFC0ED684AC0ED674AD4ED517A74EE68
:108AA000E79AF5EEC09AF1EE10FA40F3D981F7EEAD
:108AB000004A4FF0010827EE857AB5EEC07AF1EE54
:108AC00010FA40F2C181B4EEC57AF1EE10FA7EDB05
:108AD00045F2A42202FB06F241F68C3B0BFB082276
:108AE0000244B2F88EA9D4ED476AF5EEC06AF1EE01
:108AF00010FA40F3A180DFEDDF6A20EE261AF0EED7
:108B0000E90AB4EEE01AF1EE10FA80F25E81F5EEB9
:108B1000C09AF1EE10FA40F3C782B7EE008AE1EE98
:108B2000087A67EE859A71EEE71AC4ED517AF0EE95
:108B3000E17AF4EEC37AF1EE10FAC8BF0122F5EE45
:108B4000C09AC8BF89F80020F1EE10FA40F2778190
:108B5000F4EEC59AF1EE10FAC0F24681B5F88E89AE
:108B600009EE108AF8EEC98A4FF6FE7368EEA59AF0
:108B700091E69FEDC57AF7EE007A61E599F80080FD
:108B8000B8F1000F09D0D4ED470AF5EEC00AF1EEB6
:108B900010FA40F2C9804FF00008002289F8002046
:108BA000B8E4B5F8C03106EE903A67E645F2A42A7B
:108BB0000AFB06F241F68C3303FB08220244B2F8AA
:108BC000C0A173E500F1EC80DFEDAF4A54E5BDEEE6
:108BD000C78A42F6521B0BFB06F240F6C65A18EE45
:108BE00010BA0AFB08235B4400EB4302B8EEC81A34
:108BF000B2F8C031B2F8C22106EE903A09EE102A5E
:108C0000F8EE660AF8EE496A37EE418A36EEE09AE7
:108C1000F6EE008AE8EE090AD4ED476A30EEA81AAB
:108C2000F5EEC06AFCEEC10AF1EE10FACDED030AD2
:108C3000BDF80CA03FF75FAF45F2A42202FB06F29D
:108C400041F68C3B0BFB0828804408F5E8531C33A5
:108C50001A78002A7FF44FAF08EE10AADFED838A5E
:108C60009FED831ADFED830AB8EEC89AA9EE281AA1
:108C7000C6EE016AB0EEE68AB4EEE08AF1EE10FAD2
:108C80007FF73BAFFDEEC77AF5EEC04A17EE902AAC
:108C9000F1EE10FA40F2E6334CBF4FF0020A4FF00B
:108CA000010A9A4200F3818061EE856A22EAE2724B
:108CB000BDEEE69A19EE10BA9B4540F3818040F272
:108CC000E73B42F65213BAF1010F03FB062800F00E
:108CD000A18108F50952083200EB420ADFED668AED
:108CE000BAF804209FED671A9345B8BF934600EE8B
:108CF00090BAB8EEE08A78EE289A69EE817AF5EEBD
:108D0000C07AF1EE10FABFF60CAFDFED5F9AF0EE2D
:108D1000697A08E7DFED5C7AB7EE007AB8F1000F08
:108D20003FF48EACFFF7D9BB94ED517AD4ED5B1ACA
:108D3000D0ED466A77EE618AB0EEE89AB4EEE69A34
:108D4000F1EE10FA3FF527AF002284ED5B7A4FF089
:108D5000010889F80020FFF7DDBB08F5C3530A338B
:108D600000EB43089FED468AB8F80420DFED456A22
:108D70009345A8BF934607EE90BAF8EEE70A30EEA7
:108D8000887A67EE269AF4EEC69AF1EE10FA58BF8A
:108D9000F0EE469A51E5B5F88EA909EE10AAD5E590
:108DA000FFEE004A4FF0020868E461EE859ABDEEDE
:108DB000E97A17EE10BA9B4500F34D8140F2E73295
:108DC0002BEAEB7B5A457FF47CAF61EE859AF0EE9F
:108DD000617AA8E600F16C819FED2B8A81E4B5F8F9
:108DE000C0B109EE10BAB1E5BDEEE97A42F6521B08
:108DF00017EE102A0BFB062A00EB4A08B8EEC71A3A
:108E0000B8F8C0B1B8F8C22109EE10BA08EE902A3D
:108E1000F8EE496AF8EE680A79EEC19A30EEE68A11
:108E2000F6EE001AE9EE886A76EEA17ABCEEE77AF1
:108E30008DED037ABDF80CA009EE10AA92E6B5F804
:108E4000C03109EE103A8DE645F2A42A0AFB06F27B
:108E500041F68C3303FB08220244B2F8C0A142E67B
:108E600000F11D81DFED084A23E600BFAAD71F39B4
:108E70005F708930002474496666663F00C079449B
:108E8000CDCCCC3D0534833A00000000BDEEE78A2E
:108E900042F6521303FB06F240F6C65818EE10AA2B
:108EA00008FB0B23534400EB4302B8EEC89AB2F818
:108EB000C031B2F8C22106EE903A08EE902AF8EEE0
:108EC000660AF8EE686A37EEC98A76EEE08AB6EE90
:108ED000001AE8EE280AD4ED476A30EE819AF5EEE2
:108EE000C06AFCEEC90AF1EE10FACDED030ABDF836
:108EF0000C803FF75EAD45F2A42303FB06FA41F672
:108F00008C3202FB0BAB83440BF5E8531C331A780D
:108F1000002A7FF44EAD08EE108A5FED2C8A1FED1B
:108F20002C1A5FED2C0AB8EEC89AA9EE281AC6EEE4
:108F3000018AB0EEE88AB4EEE08AF1EE10FA7FF72B
:108F40003AADBDEEE77AF5EEC04A17EE10BAF1EE93
:108F500010FA40F2E6384CBF4FF0020A4FF0010A17
:108F6000C34561EE859A30DCFDEEE96A2BEAEB73CE
:108F700016EE902A424530DD40F2E73842F65212B2
:108F8000BAF1010F02FB063B68D00BF50953083319
:108F900000EB430A1FED489ABAF804205FED478AB8
:108FA0004245B8BF424601EE102AF8EEC10A30EE43
:108FB000898A28EE287AB5EEC07AF1EE10FABFF66B
:108FC0000EAD00221FED507A0FE5FDEEE97A17EEA7
:108FD000902A424505DC40F2E73322EAE2789845E0
:108FE000CCD161EEA26AB0EE617ABDEEE69A19EEDE
:108FF000102AFAE445F2A42202FB06F241F68C3A6A
:109000000AFB0B288044B8F8C081CAE454D45FED51
:10901000624AABE408F5C3530A3300EB43085FED43
:10902000686AB8F804205FED697A9345A8BF934653
:1090300007EE10BAB8EEC79A79EE268A68EEA77ADC
:10904000F4EEC67AF1EE10FA3FF56BAD5FED759A6E
:10905000F7EE007A67E5F0EE617A64E50BF5C3534D
:109060000A3300EB430B5FED7A9ABBF804A05FED87
:109070007B7AC245A8BFC24607EE10AAF8EEC76ABF
:1090800036EEA99A29EE277AB4EEC67AF1EE10FAF6
:109090003FF5A5AC4FF6FF72B7EE007AA5E4FFEE00
:1090A000004A4FF0020806E50FD41FED898A36E525
:1090B000BFEE008AFFF715BBFFEE004A4FF0020B30
:1090C00056E405D41FED908A87E4BFEE008A26E5BA
:1090D000BFEE008A81E400BF2DE9F04700F533516F
:1090E000B0F848E3B0F84A73B0F84C53B0F84E43C8
:1090F0009FED410A0646103142F6D04CB6F8522395
:10910000B6F85433B0F85003B6F85693B6F858A3EF
:109110004FEA0E183F0126F80C804F80B6F85A73BC
:109120002D012401000112011B018D80CC80B6F8B5
:109130005C53B6F85E4308814A81B6F86003B6F81E
:1091400062238B813F01B6F864334F8206F53357B3
:109150004FEA091C4FEA0A1E2D01240100011201E9
:109160001B012E378D82CC8208834A83A1F80EC062
:10917000A1F810E08B833A462048FFF745F806F542
:10918000335106F5245506F525540E4601F13208F3
:10919000103518343C364FF001094FF0000A38F80A
:1091A000021F55F8042C287811410AF085FB207A1B
:1091B00078B1E268A2F164000028E06015DDB045F6
:1091C00005F1100504F1140407F10107E7D1BDE82A
:1091D000F0873B78002BF2D054F8041C84F80890F8
:1091E000E1602046F7F7D2FDE9E784F808A02046C1
:1091F000F7F7D6FDE3E700BF17B7D1386C14FF1FB0
:10920000F0B5DFED367AB4EEE70AF1EE10FA83B08E
:1092100005460E465DD5B5EEC00AF1EE10FA54DDF6
:109220009FED2F7A2F4F3049F6EE000AE0EE070A45
:109230004FF0640CBDEEE00A10EE104A87FB040309
:10924000E017C0EB63170CFB174381FB031ED91714
:10925000C1EBAE0101EB810CA3EB4C043037303491
:109260003031F8B2E3B2C9B2204C8DF8000022725E
:10927000012000224FF4807E22618DF80410E0620C
:10928000022101A84027C4F820E0E160A262227513
:109290006275A261E2618DF801208DF806208DF8DB
:1092A000053084E860006762F8F76AFEA5F10A03FA
:1092B0000F4884E848000E3DF8F762FE684684E8EF
:1092C0006000F8F75DFE03B0F0BD30231946184684
:1092D000CAE7392319461846C6E700BF23DB1F41FA
:1092E0000000C8421F85EB516766666664D50020A2
:1092F0004CAA01002DE9F04F0027804CDFF80CA2AA
:1093000085B08B4601F1BC060D464FF00409B84606
:10931000DBF8B830434500F0C880377895F97A3DDE
:109320007749002F14BF4FF0000E4FF0770E0868FA
:109330000390002B4FF0010240F3D1804FF02B0C33
:109340008DF80CC0002BB8BF5B42092B40F3D080D6
:109350008AFB0310D917C1EBA00030308DF80D0047
:1093600000928AFB0320C1EBA00202EB8201A3EB77
:10937000410303F130024FF480700021012384F88F
:1093800008E08DF80E204FF0400C29224FF0020E1D
:10939000206203A822600192C4F80490E362A162F3
:1093A000216121756175A161E161C4F824C0C4F82F
:1093B0000CE0F8F7E5FD009AEFB1524F019B3979C7
:1093C00011F0010F17D1504908680290029FC7F3AE
:1093D0000801B1F5807F0ED90092484A4FF0200C69
:1093E000136003A8EE23C2F8049013728DF80CC02A
:1093F000F8F7C6FD009A3078002A73D0002895F956
:109400007B7D0CBF002177213D4B632F1A680392AF
:1094100047DD31208DF80C008AFB073EFA17C2EBBE
:10942000AE008AFB003CC317C3EBAC0E0EEB8E0CF8
:10943000A0EB4C0030308DF80D008AFB0703C2EB27
:10944000A30202EB8200A7EB40033033012000228D
:1094500021724FF480778DF80E304021E0624FF09A
:10946000FF3303A8C4F80490A262E260226122756F
:109470006275A261E261276261622360F8F780FD94
:1094800008F1010805F5A545B8F1050F05F124051A
:1094900006F1010609F10D097FF43AAF05B0BDE808
:1094A000F08F092FB8DCFA17C7E79BED2B7AF2EEA5
:1094B0000E7A27EE270AFDEEC00A10EE900AC307C7
:1094C0007FF52BAF377895F97A3D6FB90C49002BB2
:1094D000086803903A464FF0770E3FF72FAF09D157
:1094E00019463DE70028CBD095F97B7D77218BE7A6
:1094F000D91735E72D208DF80C0023E764D500201F
:1095000088A801005C14FF1FEC44012067666666B2
:109510002DE9F047904D9EB00C4605F58046772228
:10952000A5F5807148784B1CFF2818BF4A70597800
:10953000FF2900D05A709F78D8781979FF2F18BF6B
:109540009A705F79FF2818BFDA709879FF2918BFE1
:109550001A71FF2FDF7918BF5A71FF2818BF9A714F
:10956000D91DFF2F18BFDA718D42DBD105F580754B
:10957000AE42D5D16022002106A80CF0DDFB774B6E
:1095800093E807000DF10C0888E80700C1460020A9
:1095900059F8047B3A780DF1180A82442AB910E090
:1095A0000AF8012B17F8012F5AB1232AF8D1D4F861
:1095B00098106131CAB20AF8012B17F8012F002A5E
:1095C000F3D120306028E3D1FF263D23FD22009611
:1095D0001B21A220624DF8F767F900224FF4807337
:1095E00003F5D55A03F5DD5903F5E55803F5ED5CB0
:1095F00003F5F55E03F5FD5703F5025603F5065036
:1096000003F50A510AF1010A09F1010908F10108FB
:109610000CF1010C0EF1010E013721362130213100
:1096200003F51063B3F5145F05F80A2005F8092067
:1096300005F8082005F80C2005F80E20EA55AA5573
:109640002A546A54CCD15E2200214648464F0CF081
:1096500073FB00223A704FF4807303F5D75A03F579
:10966000DF5703F5E75603F5EF5903F5F75803F510
:10967000FF5C03F5035E03F5075003F50B511E373E
:109680001E360AF11E0A09F11E0908F11E080CF126
:109690001E0C0EF13E0E3E303E3103F51063B3F565
:1096A000145F05F80A20EA55AA552D4F05F8092040
:1096B0004FF0000605F8082005F80C2005F80E20EC
:1096C0002A546A54C9D15E2231462848284D0CF0EC
:1096D00033FB43F6FD60FF233B5443F6FE5243F653
:1096E000FE6143F6FD50BB547B543E544FF48072F0
:1096F00001274023EF62AE62EE602E612E756E751B
:10970000AE61EE612E722A626B62AA4635274FF077
:10971000A3090DF1180808EB4610C5F800906F601A
:10972000F8F72EFCD4F8981001F5CF403A3054F8F1
:109730002020B24206F1010606D0032EA7F10C0745
:10974000E7D11EB0BDE8F0870A48CAF80090CAF811
:109750000470F8F715FCF0E7970301208CA80100CE
:1097600098020120391D0120961D01203941012058
:1097700064D5002050AA01002DE9F04FCC4E8A4656
:10978000A1B01D4606F580477721A6F58070447884
:10979000431CFF2C18BF41705878FF2800D0597027
:1097A0009C78D878FF2C1C7918BF9970FF285879BD
:1097B00018BFD970FF2C9C7918BF1971FF2818BFEA
:1097C0005971FF2CDC7918BF9971D81DFF2C18BF77
:1097D000D9718642DBD106F58076BE42D5D1002311
:1097E0000E930D930F931093002D00F0BB83DAF8C6
:1097F000F010022900F0D28320264FF02B0E6C27A8
:109800004FF06108672080228DF834E08DF83570C4
:109810008DF836808DF837008DF838608DF83A6015
:109820008DF839202D2461204FF06C0C4FF0670E1D
:109830008DF83D008DF83B408DF83CC08DF83EE042
:109840004FF0C4094FF03C0BC3223D20C5273B26F7
:109850004FF0FF0800242A231421CDF80080F8F7E8
:1098600023F85A4630462C2312210094F8F71CF8AE
:109870003A463046132312210094F8F715F848466B
:109880003A46DFF83C9200942C231221F8F70CF8AA
:109890003A4630462C232B2140270094F8F704F851
:1098A000C9F82470834F89F81580012380211F2275
:1098B0000DA84FF4807B022689E80600C9F82830FD
:1098C000C9F80C30C9F8103089F81440C9F81840AC
:1098D000C9F81C4089F80840C9F820B0C9F82C60C4
:1098E000F8F74EFB0FCF0DF1440CACE80F000FCF93
:1098F000ACE80F000FCFACE80F0097E807008CE84A
:10990000070055B140F2E7306B4D6C491395E722E3
:10991000159018901B901F911D92002301264FF463
:109920008077402511ACDFF89CB1C9F82C60049415
:10993000C9F82860C9F80030C9F80430C9F80C30FB
:10994000C9F8103089F81430C9F81830C9F81C303B
:109950000393C9F82070C9F82450CDF82CA00B99B6
:10996000039A91F8FC001041FF240026C30789F8F0
:10997000154089F8086010D591ED3B7AF3EE047A32
:1099800027EE270AFDEEC00A10EE908A18F00103B8
:1099900003D14B4F3C727B751C46049DA96809910D
:1099A00008460CF06DFA2A68D5F804C0059200EB61
:1099B000400002EB4003002B174603F1010A02F1BD
:1099C000FF320CF1FF360CF1090E7DDBFF2F7BDC43
:1099D0000CF10805472D77D8FF2BA8BFFF2327EAF6
:1099E000E7783F2DA8BF3F252CEAEC70434506954C
:1099F000079069DB01332F1A0137029303023F02FC
:109A00000893069D07998D424CDB08984FF48073AC
:109A100008EB0001A7F58075BB420BF80140C5F3C8
:109A2000022059443ED018B301281CD0022817D078
:109A3000032812D004280DD0052808D006281CBF02
:109A40004FF4007381F80041CC5403F58073CC547B
:109A500003F58073CC5403F58073CC5403F5807305
:109A6000CC5403F58073CC5403F58073BB4219D0FA
:109A700003F58070CC5403F500750C5403F5407069
:109A80004C550C5403F5806503F5A0604C550C54FF
:109A900003F5C06503F5E06003F50063BB424C5578
:109AA0000C54E5D1029908F101088845A9D10BE0D1
:109AB0009703012098A8010060AA010068AA01008C
:109AC00064D5002098020120FF2A5ED8BEF1490F1C
:109AD0005BD873463F2B26EAE674A8BF3F23A34218
:109AE00053DB5F1C3D1B02EB04282F024FF48073F5
:109AF000A7F580700021BB42C0F302240BF80810C8
:109B00000BEB080041D01CB3012C1CD0022C17D049
:109B1000032C12D0042C0DD0052C08D0062C1CBF11
:109B20004FF4007380F80011C15403F58073C154E1
:109B300003F58073C15403F58073C15403F580733A
:109B4000C15403F58073C15403F58073BB421CD02C
:109B500003F58078C15403F5007500F8081003F58B
:109B6000407403F580684155015503F5C06500F860
:109B7000081003F5A06403F5E06803F50063BB4239
:109B80000155415500F80810E2D1BAF1000FC0F2BA
:109B9000D681FF2A00F3B7803F2E00F2B4805746EB
:109BA000FF2FA8BFFF2722EAE273BB42069700F30C
:109BB000AA804FEA0C21A1F580700A9018445844FD
:109BC0004442C3F1010804F0030144463C44A1426D
:109BD00028BF2146062C98BF2146079321B30BEBE3
:109BE000062000250129C55403F1010700F0108269
:109BF0000229C55503F1020700F00A820329C55561
:109C000003F1030700F004820429C55503F104079A
:109C100000F0FE810529C55503F1050700F0F88124
:109C2000C5550633A1426ED0641A201F069D0294CA
:109C3000079C8708281B401A7D1C02282C46089583
:109C40004FEA85084FD907980A9D054429440BEB34
:109C500001000790002501204BF801500799A04210
:109C600007F0070701F1040180F096812FB3012F5F
:109C70001DD0022F17D0032F12D0042F0DD0052F87
:109C800008D0062F03D0079C04316560022041F8FC
:109C9000045B013041F8045B013041F8045B0130A2
:109CA00041F8045B013041F8045B089C013001304D
:109CB000A04241F8045B80F06F81029C0F4608309F
:109CC00047F8045B4D607D60089FCD60B8420D6130
:109CD0004D618D61CD6101F12001EFD302942546E4
:109CE000454543440FD0069C0BEB0628581C002129
:109CF000844208F8031006DB02339C4208F8001087
:109D000001DB08F80310BEF1000FC0F21881BAF1B0
:109D1000FF0F68DC3F2E66DC73463F2B26EAE676B3
:109D2000A8BF3F239E425EDC5D1CA91B0F020AEB0D
:109D300006264FF48073A7F580700021BB42C0F364
:109D400002240BEB06080BF806104CD04CB3012C88
:109D500021D0022C1BD0032C15D0042C0FD0052CA5
:109D600009D0062C1CBF4FF4007388F8001108F8C6
:109D7000031003F5807308F8031003F5807308F8E7
:109D8000031003F5807308F8031003F5807308F8D7
:109D9000031003F5807308F8031003F58073BB42CA
:109DA00021D003F5807603F5007503F5407008F8BF
:109DB000031003F5A06408F8061008F8051003F571
:109DC000806608F8001003F5C06503F5E06003F550
:109DD0000063BB4208F8061008F8041008F80510E4
:109DE00008F80010DDD1FF2A00F3A980BEF13F0F73
:109DF00000F3A5805546FF2D22EAE272A8BFFF2599
:109E0000AA4200F39C804FEA0C2A0AF5106A0AEB7A
:109E10000207C2F101015F4408467B4203F00308D8
:109E20002844804528BF8046062894BF0146414605
:109E3000002900F0AF800BEB0E2400260129A65468
:109E400002F1010314D00229E65402F102030FD0FB
:109E50000329E65402F103030AD00429E65402F16F
:109E6000040305D0E654531D05291CBFE654931D79
:109E7000814264D0401A071FAC1ABE08671A06F167
:109E80000108022F4FEA88044AD95244114400279E
:109E90000BEB010A4BF801700121884506F007061B
:109EA0000AF1040239D91EB3012E1CD0022E17D09C
:109EB000032E12D0042E0DD0052E08D0062E03D06E
:109EC000CAF804700432022142F8047B013142F8DE
:109ED000047B013142F8047B013142F8047B0131FB
:109EE00042F8047B01310131884542F8047B14D9E2
:109EF000924608314AF8047B88455760CAF80470D6
:109F000002F1200242F8147C42F8107C42F80C7CEA
:109F100042F8087C42F8047CEAD8844223440ED0FC
:109F20000BEB0E2E5E1C0027AE420EF8037006DC13
:109F30000233AB420EF8067001DC0EF80370039A90
:109F40000499059B0998013214460C31039289E863
:109F500008100491F8F714F8052C7FF400AD21B037
:109F6000BDE8F08F92B3DAF8F040DAF8F43041341B
:109F700041334FF0800C8DF834408DF836308DF839
:109F800035C04FF09A094FF0660B992267209B2746
:109F900065265DE413466DE7029DA1E620232D278B
:109FA0006C264FF061094FF0670B80218DF83470FB
:109FB0008DF835608DF836908DF837B08DF83830E3
:109FC0008DF83A308DF839102B242CE4DAF8F4307F
:109FD0006C274FF06509722020224FF0630841334F
:109FE00061248DF835708DF836908DF838008DF835
:109FF00039208DF83A308DF834808DF837404FF0A5
:10A00000B1094FF04F0BB0225020B2274E261FE46B
:10A010003B4607E62DE9F04F2DED0A8B89B009EE9E
:10A02000101A1D9E1C9AD6F894409A4609EE900A82
:10A03000002C40F0A9820221012307940591069388
:10A0400005AF214657F8049B9FEDE3AADFEDE38AB5
:10A05000CDF80CA045F2A420894500FB02F81E9D16
:10A0600000F04881EC78002C00F0398141F68C300A
:10A0700000FB0983F21802F5E07492F879ED039879
:10A0800019EE102A801A08EE100ABEF1000F00F037
:10A0900008833344B8EEC88AF8EEC9AAF8EEE9BAE4
:10A0A00003F5196C4FF0BB0B208807EE100AB7EED2
:10A0B00000BAB8EEC71AF0EE4B6AE1EE686A0CF12E
:10A0C000FF3A4FF00009F0EE6A0AE6EE880AB0EEB9
:10A0D0006B0A37E040F2E733994539D09AF801002E
:10A0E00009F1010900285AD140F2E731894556D0DB
:10A0F0009AF8022009F1010C002A77D140F2E733E7
:10A100009C4573D09AF8031009F1020C002940F025
:10A11000958040F2E732944500F090809AF8040070
:10A1200009F103010AF1040A002840F0B18040F26D
:10A13000E73C614500F0AC8009F10409B9F57A7F8C
:10A1400000F0CD809AF801100AF1010A0029C1D06F
:10A1500034F8192004EE902AB8EEE4CAF0EE4B7AF7
:10A160000CEE909AECEE687A584609F10109F8EE87
:10A17000EC1AB0EE6BCAF0EE6ACAA1EE8ACAE8EE3B
:10A1800027CAB0EE4C1AF0EE6C1AF7F785FC9AF875
:10A190000100F0EE6C0AB0EE4C0A0028A4D034F8AE
:10A1A00019E002EE10EAF8EEC22AB0EE4B5A03EEC6
:10A1B000109AA2EEE85A5846F8EEC33AB0EE6BCACF
:10A1C000F0EE6ACAA3EE8ACAE8EE05CAB0EE4C1AEF
:10A1D000F0EE6C1AF7F760FC9AF80220F0EE6C0AC9
:10A1E000B0EE4C0A09F1010C002A87D034F81C00AB
:10A1F00007EE100AB8EEC71AF0EE4B4A06EE90CA08
:10A20000E1EE684A5846F8EEE65AB0EE6BCAF0EE58
:10A210006ACAA5EE8ACAE8EE24CAB0EE4C1AF0EE7D
:10A220006C1AF7F739FC9AF80310F0EE6C0AB0EEEE
:10A230004C0A09F1020C00293FF46BAF34F81C30D2
:10A2400007EE903AB8EEE76AB0EE4B3A02EE10CA6B
:10A25000A6EE683A58460AF1040AF8EEC22AB0EEB1
:10A260006BCAF0EE6ACAA2EE8ACAE8EE03CAB0EE82
:10A270004C1AF0EE6C1AF7F70FFC9AF80000F0EEAB
:10A280006C0AB0EE4C0A09F1030100283FF44FAF0D
:10A2900034F811E005EE10EAB8EEC54AF0EE4B6A6C
:10A2A00007EE101AE4EE686A584609F10409B8EEA0
:10A2B000C71AB0EE6BCAF0EE6ACAE8EE26CAA1EE83
:10A2C0000ACAF0EE6C1AB0EE4C1AF7F7E5FBB9F5D6
:10A2D0007A7FF0EE6C0AB0EE4C0A7FF433AF08AC34
:10A2E000BC4200F04C81D6F8941057F8049B894585
:10A2F0007FF4B8AE41F68C3202FB0183039895F8E7
:10A3000000E019EE102A03F5D87BF418801AB34444
:10A3100004F5E07408EE100ABEF1000F00F0D281DF
:10A320006978002940F03A81B8EEC88AF8EEC9AAE7
:10A33000B8EEE97A41F68C3202FB098EB6449BED09
:10A34000010ADEF8B401F8EEC07AF0EE470A86445E
:10A35000E7EE8A0A9EF89019B0EE601A002900F024
:10A3600077819DED03BAB8EECBCAF6EE005A71EED6
:10A37000254A7CEE25BA3AEEA50AFDEEE4CAFDEECA
:10A38000EB7AFDEEC00A4FF0660C1CEE902A1CEE34
:10A39000900A17EE903A10EE901ACDF800C0F7F739
:10A3A00083FA41F68C3B0BFB0983F21892F8790D86
:10A3B000002840F06E8141F68C3E0EFB0989B144C5
:10A3C00009F5E851DFF818E01C310023B6EE001A59
:10A3D000F7EE006ABCE000BF7F6A3C3E8000803739
:10A3E0009802012013EE902AFF2A1AD834F813C0DD
:10A3F00005EE10CAB8EEC54AF0EE665AE4EE685AA9
:10A40000B0EE6ABAA5EE88BA7BEE01CAFDEEECBAF0
:10A410001BEE90BABBF13F0F9CBF0EEB0B2B0BF862
:10A420000200013300EE103AF8EEC07AF0EE470A6F
:10A43000E7EE8A0A0A7830EE816A002A40F0F68058
:10A44000FDEEC62A12EE902AFF2A1AD834F813A07D
:10A4500003EE10AAF8EEC33AB0EE665AA3EEE85A3D
:10A46000F0EE6A5AE5EE085A35EE81BABDEECBCA77
:10A470001CEE109AB9F13F0F03D80EEB092C0CF823
:10A48000020003F1010B0CEE90BAF8EEECBAB0EE5C
:10A49000470AABEE8A0A0A7870EE010A002A40F0F9
:10A4A000BC80BDEEE06A16EE102AFF2A1AD834F8F6
:10A4B0001BA002EE10AAF8EEC22AB0EE663AA2EE97
:10A4C000E83AB0EE6A5AA3EE085A75EE015AFDEE6C
:10A4D000E54A14EE909AB9F13F0F03D80EEB092C20
:10A4E0000CF8020003F1020B0BEE10BAB8EECBCA67
:10A4F000F0EE47CAECEE0ACA0A783CEE810A002A5E
:10A5000040F09D80FDEEC00A10EE902AFF2A1AD876
:10A5100034F81BA001EE90AAB8EEE16AB0EE662A0C
:10A52000A6EE682AB0EE6A3AA2EE083A33EE015A75
:10A53000BDEEC54A14EE109AB9F13F0F03D80EEBE9
:10A54000092C0CF802000333B3F57A7F3FF4C7AE51
:10A5500001EE903AB8EEE16AB0EE472AA6EE0A2A7A
:10A560000A7832EE013AFDEEC33A002A3FF43AAFE0
:10A5700013EE902A12F0010F7FF453AF34E709B0C5
:10A58000BDEC0A8BBDE8F08F022C00F09580002313
:10A590000221012005930691079051E59BED020AE7
:10A5A000DBED017AF8EEC00AF7EE006AE0EEE86A49
:10A5B00088230093F8EEC9AAB8EEE97AB8EEC88A03
:10A5C000B8EEE71AB0EE6A6AF0EE471AA6EE886AAD
:10A5D000E1EE0A1AB6EE002A76EE022A31EE823A4F
:10A5E000F0EE003A32EEA35A32EEE34A73EE235A0B
:10A5F00073EE634ABDEEC5BABDEEC4CAFDEEE5CA50
:10A60000FDEEE4BA1BEE103A1CEE101A1CEE902A76
:10A610001BEE900AF7F748F98CE6FDEEE01A11EE12
:10A62000902A12F0010F7FF45DAF3EE7BDEEC62A1F
:10A6300012EE102A12F0010F7FF423AF04E7FDEEB3
:10A64000C07A17EE902A12F0010F7FF47CAF5DE71D
:10A650009DED036AB8EEC62AF6EE006A71EE261A80
:10A6600032EE263A7AEEA63AFDEEE12ABDEEC35A64
:10A67000BDEEE34A4FF0660A12EE902A12EE900AFF
:10A6800015EE103A14EE101ACDF800A0F7F788F97D
:10A6900087E6334403F5196CF0EE47BA4FF0000B30
:10A6A00002E58945B8EEE97AF8EEC9AAB8EEC88A9B
:10A6B00014BFBB2000207EE60025012707940595E6
:10A6C0000697BDE4F21892F8790D0028E9D03344DA
:10A6D00003F5196CF346B8EEC88AF8EEC9AAF8EE8D
:10A6E000E9BAE1E42DE9F04F2DED028BB74F9BB0B5
:10A6F00080460D463C4607F580764FF0FF3200233A
:10A70000E25003F5807103F5007B03F5407A03F511
:10A71000806903F5A06C03F5C06E03F5E06003F5F6
:10A720000063B3F5804F625044F80B2044F80A20D0
:10A7300044F8092044F80C2044F80E202250DFD1C0
:10A740000434B442DBD1AA7F002A40F0ED80E97FD7
:10A75000002940F0C58295F82000002840F033839E
:10A76000AB6A002B71D0994A4FF0FF310027D151CD
:10A7700007F5807B07F5007007F5407A07F5806CD8
:10A7800007F5A06E07F5C06907F5E06407F50067F7
:10A79000B7F5804F42F80B104FF0FF38115042F8D8
:10A7A0000A1042F80C1042F80E1042F8091011512C
:10A7B000DDD10432B242D9D1FF2600962C23C22229
:10A7C00013213D200026F7F76FF83C2210462D2379
:10A7D00012210096F7F768F812231946C3223C208D
:10A7E0000096F7F761F8C32210462D231221009638
:10A7F000F7F75AF82D23764C00961946C3223C20D1
:10A80000F7F752F87F27012340211A227148A661E9
:10A810004FF4807BE66184F815802672C4F820B07E
:10A8200061626260E3622375A362E3602361276073
:10A83000F7F7A6FBA86A276024256560F7F7A0FB59
:10A840001BB0BDEC028BBDE8F08F95F82120002AEB
:10A8500040F0C88005F5DF3090F88CB0BBF1000FF8
:10A8600040F0BB8490F8AE10002940F0BD8395F80D
:10A87000A740002C40F0FA8495F81401002800F05D
:10A880000881554AD5F8001113680593059C601A94
:10A89000B0F5FA7F40F2FD80504C126820790A92A0
:10A8A000F9F772FFD5F810E10A9C484A0028CBBF9F
:10A8B0000020FF20FF270027002360F3070360F339
:10A8C0000F2360F3174360F31F63002101F58075C8
:10A8D000535001F50078535101F5407B01F5806C30
:10A8E00001F5A06A01F5C06901F5E06501F50061B7
:10A8F000B1F5804F42F8083042F80B3042F80C3086
:10A9000042F80A3042F809305351DFD10432B242E2
:10A910002E4DD1D1CEEB0406C6F3053005EB002455
:10A92000C6F30712A7548BE7284A4FF0FF310027E0
:10A93000D15107F5807907F5007807F5407C07F5D8
:10A94000806E07F5A06B07F5C06A07F5E06507F5AF
:10A950000067B7F5804F42F809104FF0FF3442F816
:10A96000081042F80C1042F80E1042F80B1042F892
:10A970000A105151DCD10432B242D8D11648144BDE
:10A9800006680696069A5C754FF48075C2F3080750
:10A99000012100204024AF421D625C62D96219751A
:10A9A0009962D9601961186058609861D86118720D
:10A9B0007FF646AF7F211F22094883E80600F7F79C
:10A9C000DFFA1BB0BDEC028BBDE8F08F98020120CE
:10A9D00064D50020BCAA0100EC4401205C14FF1FD8
:10A9E0007CAA0100B44B4FF0FF314FF0000B43F84D
:10A9F0000B100BF5A0670BF580700BF5007A0BF5CB
:10AA0000407E0BF5806C0BF5C0650BF5E0640BF533
:10AA1000006BBBF5804F195043F80A1043F80E1035
:10AA200043F80C10D95159514FF0FF371951DED16D
:10AA30000433B342D9D1A14AA14E1368099396E8D1
:10AA40000F000DF1280989E80F00099D9D4CC5F301
:10AA5000C1110DF1680808EB81000023022267751F
:10AA600001254FF4807750F8400CE36040262361C5
:10AA700027626662E562A5622375A361E3612372C2
:10AA800022606260F7F77CFA1BB0BDEC028BBDE878
:10AA9000F08F95F89040002C00F02682012C40F0B9
:10AAA000E38095F8F860002E40F05E8295F8FA2079
:10AAB000002A40F0598295F8F9A0BAF1000F40F051
:10AAC0005382814E814B1A68D6F8983009928DE8EE
:10AAD000480009A8214696F8A19002903E2340F232
:10AAE00015422D208DF824408DF82590FFF792FA1D
:10AAF00029464046FEF7FEFBD6F898109FED740AF3
:10AB00006231524655F8214007EE904AF8EEE70AC6
:10AB1000042120EE800AFC20FEF772FBD5F8942079
:10AB200095ED671A95ED687A002A00F01382F7EE2A
:10AB3000001AB4EEE17AF1EE10FA00F1D4839FED41
:10AB4000650A77221121FC20FEF75AFBD5F8A421D3
:10AB5000002A4DDB0026632A0A9640F3B0835E4B41
:10AB6000D11783FB0204C1EB641030308DF828004C
:10AB7000594E5A4886FB024CC1EB6C1B642303FB05
:10AB80001B2680FB064AF417C4EBAA0030305FFA9C
:10AB900080FE524B4B4C8DF829E083FB0206C1EB43
:10ABA000A609D5F89C00D5F8941009EB890CA2EB06
:10ABB0004C030126814214BF7721002130334FF42A
:10ABC00080720220E66200268DF82A30217240232E
:10ABD000FC212262E0601E220AA82661636284E8EA
:10ABE0000600A66226756675A661E661F7F7C8F9E4
:10ABF00095ED6A3AF7EE003AB4EEE33AF1EE10FA68
:10AC000000F167839FED330AD5F89440002C14BF00
:10AC1000772200222B21FC20FEF7F2FAD5ED6B4AB9
:10AC2000B7EE005AF4EEC54AF1EE10FA00F1528187
:10AC30009FED280A00223821FC20FEF7E1FA95F862
:10AC4000FB307BB941F2FF4642F2FF1B42F6FF6A3E
:10AC500043F6FF31BB5507F80B3007F80A307B5439
:10AC600087F8FF3795F8904095F8F860002E40F08F
:10AC70002E8195F8FA00002840F0298195F8F930E6
:10AC800063B14FF00109002C00F058834B46324667
:10AC900029464046FEF770FD95F89040012C7FF460
:10ACA000CFAD95F8FB1000293FF4CAAD29464046C8
:10ACB000FEF72EFCC4E500BF98020120EC44012001
:10ACC000E4A8010064D500206C14FF1FF4A8010063
:10ACD0000DE81F396DE71F411F85EB5167666666FA
:10ACE000B64A4FF0FF310023D15003F5807503F5CC
:10ACF000007003F5407B03F5806A03F5A06E03F551
:10AD0000C06703F5E06403F50063B3F5804F51516C
:10AD100011504FF0FF3542F80B1042F80A1042F87C
:10AD20000E10D1511151DFD10432B242DBD1FF26D6
:10AD300000962C23C22213213D200027F6F7B4FDF4
:10AD40003C2210462D2312210097F6F7ADFD122369
:10AD50001946C3223C200097F6F7A6FDC3221046F1
:10AD60002D2312210097F6F79FFD2D231946C322AC
:10AD70003C200097F6F798FD914A924C1168079194
:10AD8000079827604FF48076C0F308030122402122
:10AD9000B3426760A761E7616575277226626162E9
:10ADA000E2622275A262E26022617FF649AD7F21F4
:10ADB0001F22854884E80600F7F7E2F81BB0BDECD7
:10ADC000028BBDE8F08F7D4A4FF0FF314FF0000B52
:10ADD00042F80B100BF580700BF5007A0BF54079FB
:10ADE0000BF5806C0BF5A06E0BF5C0680BF5E064FD
:10ADF0000BF5006BBBF5804F11504FF0FF3742F859
:10AE00000A1042F8091042F80C1042F80E1042F8ED
:10AE100008101151DCD10432B242D7D1FF2600967E
:10AE20002C23C22213213D20F6F73EFD00243C22B4
:10AE3000009410462D231221F6F736FD12230094BC
:10AE40001946C3223C20F6F72FFDC322009410467A
:10AE50002D231221F6F728FD2D235A4D0094194673
:10AE6000C3223C20F6F720FD7F26012340211B2230
:10AE70004FF4807A5548AC61EC616F752C72696251
:10AE80006A60EB622B75AB62EB602B612E60C5F8DC
:10AE900020A0F7F775F84E48494F2E600FC83C6860
:10AEA00008940DF1280989E80F00089E0DF1680C3F
:10AEB000C6F3C1110CEB8108232258F8400C6A60DC
:10AEC000F7F75EF81BB0BDEC028BBDE8F08F95F88C
:10AED000F990D8E6F5EEC04AF1EE10FA37DDDFED75
:10AEE0003D5A24EEA50AA5E626468DF82A408DF89F
:10AEF00029408DF828408DF82B400AAF06F10B034E
:10AF000031468DE8B00040F215422D20FFF782F85F
:10AF1000013429464046FEF7EDF9052C06F10D06F1
:10AF2000ECD19FED2D8A05F5C277042457F8042F44
:10AF300006EE102AF8EEC66A2146002226EE880A9E
:10AF4000FC200D34FEF75CF9452CEFD18AE69FED2D
:10AF5000230A6FE6B7EE002AB4EEC21AF1EE10FA39
:10AF60001CD49FED1C0AEDE51D4B1E490868D3F863
:10AF7000981009908DE80A0009AC93F8A16002943A
:10AF80004FF0000E3E2340F2154201212D208DF896
:10AF900025608DF824E0FFF73DF850E6B5EEC01AC5
:10AFA000F1EE10FA40F30D82DFED0A2A002A14BFF9
:10AFB0007722002221EE220AC4E500BF9802012078
:10AFC000EC44012064D5002098AA0100A8AA010041
:10AFD000D4A801006DE71F410DE81F3900000000F3
:10AFE0006C14FF1FF4A801004FF480725946C54845
:10AFF0000AF0A2FE4FF48072594620460AF09CFEE9
:10B000004FF480725946A0180AF096FE4FF48072F1
:10B01000594604F500700AF08FFE4FF480725946CD
:10B0200004F540700AF088FE4FF48072594604F52A
:10B0300080600AF081FE4FF48072594604F5A060EA
:10B040000AF07AFE4FF48072594604F5C0600AF0A7
:10B0500073FE59464FF4807204F5E0600AF06CFE0E
:10B0600004F5106A04F500634FF0FF3119604FF4E6
:10B070008072995002F5807602F5007002F5407EEC
:10B0800002F5806402F5A06902F5C06702F5E06888
:10B0900002F5006B02F51062B2F55C5F9951195030
:10B0A0004FF0FF3643F80E10195143F80910D951EB
:10B0B00043F8081043F80B10DBD104335345D5D1C6
:10B0C000914C92482672002601234FF002094FF45A
:10B0D00080714FF0400B6660E6602661FF27E362F7
:10B0E000A362216267752675A661E661C4F824B083
:10B0F000C4F80090F6F744FF5A4631460AA8DFF834
:10B100001C82DFF834A226720AF016FE95F8AA0017
:10B110007F4F804ABB79B04214BF414651460091EF
:10B120000AA83F210AF056FE0A220AA8C4F8009095
:10B130006260F6F725FF95F8AA6097F807C0764A8F
:10B14000012E14BF4346534600930AA8ACF1640392
:10B150003F210AF03FFE0AA81321C4F80090616065
:10B16000F6F70EFF7B7995F8AAB0DFF8CC916B4E1D
:10B170006B4A052B96BF6B486B4B50F82330BBF1E5
:10B18000020F14BF3146494600910AA83F210AF038
:10B1900021FE4FF002082E220AA86260C4F8008047
:10B1A000F6F7EEFE3879F9F7EFFA95F8AA505F4A0C
:10B1B00080EAE077032D08BF4E46A7EBE0730096C8
:10B1C0003F210AA80AF006FE37230AA8C4F8008027
:10B1D0006360F6F7D5FEFFF733BB4A4B4FF0FF3104
:10B1E0004FF0000843F8081008F5807E08F5007A53
:10B1F00008F5407C08F5806408F5A06B08F5C06987
:10B2000008F5E06508F50068B8F5804F43F80E10C2
:10B210004FF0FF3243F80A1043F80C10195143F86D
:10B220000B1043F809105951DCD10433B342D7D184
:10B23000354B4FF480715A751962002201218C3010
:10B24000402702267F251F245F62DE621D605C604E
:10B250001A759A61DA611A729962D9601961F6F702
:10B260008FFE1BB0BDEC028BBDE8F08F254B4FF07D
:10B27000FF314FF0000C43F80C100CF580750CF505
:10B2800000700CF5407E0CF580670CF5A0680CF59D
:10B29000C06B0CF5E0640CF5006CBCF5804F5951A7
:10B2A000195043F80E10D95143F8081043F80B1009
:10B2B0001951E0D10433B342DBD1FFF7C1BA4FF0EB
:10B2C000200E092A8DF828E04FEAE2717FF761AC81
:10B2D0004EE4B5EEC03AF1EE10FA0CDD9FED144AE3
:10B2E00023EE040A90E4B5EEC07AF1EE10FA05DD23
:10B2F000B0EE471A58E69FED0F0A85E49FED0D0A60
:10B3000077221FE49802012064D50020CCAA010016
:10B310005C14FF1FDCAA0100F4AA010064B901005B
:10B3200010AB010034AA010074AA010024AB010093
:10B330006DE71F410000000070AA01004FF4807209
:10B34000FF2122480AF0F8FC4FF48072FF212048C8
:10B350000AF0F2FC4FF48072FF211E480AF0ECFC68
:10B360004FF48072FF211C480AF0E6FC4FF4807213
:10B37000FF211A480AF0E0FC4FF48072FF211848C0
:10B380000AF0DAFC4FF48072FF2116480AF0D4FC70
:10B390004FF48072FF2114480AF0CEFC4FF4807203
:10B3A000FF2112480AF0C8FC4FF48072FF211048B8
:10B3B0000AF0C2FC4FF48072FF210E480AF0BCFC78
:10B3C00064E49FED0D0AFFF7BDBB00BF9837012075
:10B3D0009838012098390120983A0120983B0120A3
:10B3E000983C0120983D0120983E0120983F012083
:10B3F00098400120984101200000000001380B46D0
:10B400003A2800F25C82DFE810F053024C02450259
:10B410003E0237023002290222021B02AE01A701BE
:10B42000A001990192018B0184017D0176016F01D8
:10B43000680161015A0153014C0145013E01370188
:10B440003001290122011B0113010B010301FB0043
:10B45000F300EB00E300DB00D300CB00C300BB0034
:10B46000B300AB00A3009B0093008B0083007B0024
:10B4700073006B0063005B0053004B0043003B0014
:10B48000BC48BD49C0F8EC201A463B2008F036B84D
:10B49000B848BA49C0F8E8201A463A2008F02EB851
:10B4A000B448B749C0F8E4201A46392008F026B855
:10B4B000B048B449C0F8E0201A46382008F01EB859
:10B4C000AC48B149C0F8DC201A46372008F016B85D
:10B4D000A848AE49C0F8D8201A46362008F00EB861
:10B4E000A448AB49C0F8D4201A46352008F006B865
:10B4F000A048A849C0F8D0201A46342007F0FEBF63
:10B500009C48A549C0F8CC201A46332007F0F6BF66
:10B510009848A249C0F8C8201A46322007F0EEBF6A
:10B5200094489F49C0F8C4201A46312007F0E6BF6E
:10B5300090489C49C0F8C0201A46302007F0DEBF72
:10B540008C489949C0F8BC201A462F2007F0D6BF76
:10B5500088489649C0F8B8201A462E2007F0CEBF7A
:10B5600084489349C0F8B4201A462D2007F0C6BF7E
:10B5700080489049C0F8B0201A462C2007F0BEBF82
:10B580007C488D49C0F8AC201A462B2007F0B6BF86
:10B5900078488A49C0F8A8201A462A2007F0AEBF8A
:10B5A00074488749C0F8A4201A46292007F0A6BF8E
:10B5B00070488449C0F8A0201A46282007F09EBF92
:10B5C0006C488149C0F89C201A46272007F096BF96
:10B5D00068487E49C0F898201A46262007F08EBF9A
:10B5E00064487B49C0F894201A46252007F086BF9E
:10B5F00060487849C0F890201A46242007F07EBFA2
:10B600005C487549C0F88C201A46232007F076BFA5
:10B6100058487249C0F888201A46222007F06EBFA9
:10B6200054486F49C0F884201A46212007F066BFAD
:10B6300050486C49C0F880201A46202007F05EBFB1
:10B640004C486949C2671A461F2007F057BF49484E
:10B65000664982671A461E2007F050BF4548644974
:10B6600042671A461D2007F049BF424861490267F8
:10B670001A461C2007F042BF3E485F49C2661A4680
:10B680001B2007F03BBF3B485C4982661A461A20E4
:10B6900007F034BF37485A4942661A46192007F066
:10B6A0002DBF3448574902661A46182007F026BFB6
:10B6B00030485549C2651A46172007F01FBF2D486C
:10B6C000524982651A46162007F018BF294850498A
:10B6D00042651A46152007F011BF26484D490265FC
:10B6E0001A46142007F00ABF22484B49C2641A4682
:10B6F000132007F003BF1F48484982641A461220EE
:10B7000007F0FCBE1B48464942641A46112007F068
:10B71000F5BE1848434902641A46102007F0EEBEF1
:10B7200014484149C2631A460F2007F0E7BE11488A
:10B730003E4982631A460E2007F0E0BE0D483C49A0
:10B7400042631A460D2007F0D9BE0A483949026300
:10B750001A460C2007F0D2BE06483749C2621A4684
:10B760000B2007F0CBBE0348344982621A460A20F8
:10B7700007F0C4BEA4430120F5080000E108000062
:10B78000CD080000B9080000A508000091080000DD
:10B790007D0800006908000055080000410800000D
:10B7A0002D0800001908000005080000F10700003E
:10B7B000DD070000C9070000B5070000A107000071
:10B7C0008D070000790700006507000051070000A1
:10B7D0003D070000290700001507000001070000D1
:10B7E000ED060000D9060000C5060000B106000005
:10B7F0009D06000089060000750600006106000035
:10B800004D06000039060000250600001106000064
:10B81000FD050000E9050000D5050000C105000098
:10B82000AD050000990500008505000071050000C8
:10B830005D050000490500003505000021050000F8
:10B840001F48204942621A46092007F057BE1C488B
:10B850001D4902621A46082007F050BE18481B49CD
:10B86000C2611A46072007F049BE1548184982618F
:10B870001A46062007F042BE1148164942611A4690
:10B88000052007F03BBE0E48134902611A4604200A
:10B8900007F034BE0A481149C2601A46032007F077
:10B8A0002DBE07480E4982601A46022007F026BEC8
:10B8B00003480C4942601A46012007F01FBE70473A
:10B8C000A44301200D050000F9040000E504000078
:10B8D000D1040000BD040000A9040000950400008C
:10B8E000810400006D04000008B5134640680A4654
:10B8F0001946FFF783FD08BD2DE9F04141688A68CC
:10B9000084B042F21074D3789B0609D5D578AF067F
:10B9100006D5D678B50603D5D778BB0600F17A816F
:10B92000B02490F85E3094708A6842F21075D67830
:10B93000B60608D4D778BC0605D492F803805FEA2F
:10B94000886440F1E480D578AF0622D592F802C031
:10B950004CF0300494708A6842F21075D678B706BD
:10B9600008D4D778BE0605D492F803805FEA8864CD
:10B9700040F1AE815B0043F00105ECB214718B68BD
:10B9800042F21072DE78B50703D4DF78BC0740F1CD
:10B99000DD814368597B012900F060819C6D5E6DFB
:10B9A000B442C0F0D1800023016E80F85C308A6818
:10B9B00042F21074D578AE060BD5D678B50608D508
:10B9C000D778BE0605D592F803C05FEA8C6500F112
:10B9D000C580B02490F8BA3094708A6842F210752D
:10B9E000D778BC0607D4D678B70604D492F803C03B
:10B9F0005FEA8C6671D5D578AE0622D592F80280C2
:10BA000048F0300494708A6842F21075D778BE0608
:10BA100008D4D678B40605D492F803C05FEA8C66E1
:10BA200040F173815B0043F00105ECB214718B6847
:10BA300042F21072DF78BF0703D4DE78B60740F118
:10BA4000A681036E597B012900F0AA809C6D5F6D71
:10BA5000BC427ED30023D0F89C4280F8B830002C42
:10BA60002ED0B84EB84F4FF0000801250EE06168A7
:10BA7000821A8A4208D3002B28D1A36825759342E5
:10BA80008CBF002201226275E468CCB12068026894
:10BA9000B24218D1A369217F93F8583038682269DF
:10BAA00003900B4103F001030398002ADFD1002B20
:10BAB000EAD13868029002992161E468002CE5D14E
:10BAC00004B0BDE8F08120469047DDE7C4F810805F
:10BAD00084F8148084F81580D6E792F803805FEA32
:10BAE000886488D4D478A70685D4D778BE0682D453
:10BAF000D678B4063FF57FAF92F803C05FEA8C6753
:10BB00003FF579AF083D7FF46BAF95703CE092F85C
:10BB100003C05FEA8C673FF516AFD478A6063FF501
:10BB200012AFD678B4063FF50EAFD778BF063FF513
:10BB30000AAF92F803805FEA88663FF504AF083DDC
:10BB40007FF4F5AE95707DE0671C1C449F65237DF6
:10BB50002AE7661C1C449E65237D7CE792F80380DF
:10BB60005FEA88637FF535AFD3789F067FF531AF05
:10BB7000D578AE067FF52DAFD678B5067FF529AF1F
:10BB8000083C7FF417AF947000BF8B6880229A70D6
:10BB900000BF036E01250D73597B01297FF456AF59
:10BBA0004FF000088DF806809DF806209A6842F252
:10BBB0001074D5782D0600F1758192F803C05FEA04
:10BBC0000C6100F16F81D1780E0600F16B81D7789E
:10BBD0003D0600F16781D678310600F16381D578A2
:10BBE0002F0600F15F8192F803805FEA086600F19A
:10BBF000598192F803C05FEA0C6500F15381083C5B
:10BC0000D7D1947000BF9A688021917000BF012441
:10BC10001C731FE792F803805FEA88677FF580AEA8
:10BC200092F803C05FEA8C667FF57AAED3789D0602
:10BC30007FF576AED578AB067FF572AE083C7FF423
:10BC400062AE947000BF8B6880229A7000BF436818
:10BC500001250D73597B01297FF4A0AE4FF0000C34
:10BC60008DF807C09DF807209A6842F21074D578C5
:10BC7000290600F1AD8092F803805FEA086700F1C1
:10BC8000A780D178090600F1A380D678370600F1A5
:10BC90009F80D7783E0600F19B80D5782D0600F175
:10BCA000978092F803C05FEA0C6100F1918092F8EE
:10BCB00003805FEA086700F18B80083CD7D194705D
:10BCC00000BF9A688021917000BF01241C736AE64E
:10BCD00092F803C05FEA8C673FF54CAED478A606B5
:10BCE0003FF548AED678B4063FF544AED778BF06E8
:10BCF0003FF540AE92F803805FEA88663FF53AAEC2
:10BD0000083D7FF42BAE95709CE792F803805FEAC4
:10BD100088643FF587AED478A7063FF583AED77821
:10BD2000BE063FF57FAED678B4063FF57BAE92F8FF
:10BD300003C05FEA8C673FF575AE083D7FF466AEE1
:10BD4000957021E7490B0000EC440120DD78AE0737
:10BD50003FF51FAE93F803C05FEA8C753FF519AE4F
:10BD600093F803805FEA88743FF513AEDC78A70789
:10BD70003FF50FAEDE78B6073FF50BAEDF78BD07B7
:10BD80003FF507AE083A7FF4FDAD9A705AE7DD78CB
:10BD9000AC073FF556AE93F803805FEA88773FF52E
:10BDA00050AE93F803C05FEA8C763FF54AAEDC787C
:10BDB000A5073FF546AEDF78BC073FF542AEDE781B
:10BDC000B7073FF53EAE083A7FF434AE9A70DBE633
:10BDD000947804F0E70191709A681679F7B28DF8BB
:10BDE0000770957845F0080494709A680221D17024
:10BDF0009A6842F21074D678B6071BD4D778BD077C
:10BE000018D4D578AE0715D492F803C05FEA8C75C4
:10BE100010D492F803805FEA88710BD4D1788F0731
:10BE200008D4D678B60705D4D778BD0702D4083C25
:10BE3000E1D144E7947804F0C7059570996842F21F
:10BE40001072CE78B40640F19680CF78BF0640F1EC
:10BE5000928091F803C05FEA8C6440F18C8091F885
:10BE600003805FEA886740F18680CC78A60640F1BF
:10BE70008280CD78AD067ED5CE78B4067BD5CF78DE
:10BE8000BF0678D5083ADCD18A7000BF9968802453
:10BE90008C7000BF01259E681D73022713463279FE
:10BEA000F77081E5947804F0E70191709A6817794A
:10BEB000FEB28DF80660957845F0080494709A6893
:10BEC0000221D1709A6842F21074D778BF071BD450
:10BED000D678B60718D4D578A90715D492F8038078
:10BEE0005FEA887710D492F803C05FEA8C760BD4AF
:10BEF000D1788D0708D4D778B90705D4D678B70795
:10BF000002D4083CE1D17CE6947804F0C705957032
:10BF1000996842F21072CF78BD0628D5CE78B40663
:10BF200025D591F803805FEA886520D591F803C094
:10BF30005FEA8C641BD5CC78A70618D5CD78AE0601
:10BF400015D5CF78BD0612D5CE78B4060FD5083AF0
:10BF5000E1D18A7000BF996880248C7000BF0125F0
:10BF60009F681D73022613463A79FE7073E502221C
:10BF70000B79CA706FE502220B79CA7014E500BF15
:10BF80002DE9F04705460E4645F8041BDFF8B89347
:10BF9000DFF8B88305610021044681608161466055
:10BFA000C0F80C90C0F8148040221C3009F0C4FE88
:10BFB000392384F85E30B268907800F0BF01917048
:10BFC000A0680127777358B10668DD4973688B4212
:10BFD00004F10C0240F0828440680221FFF70EFA5F
:10BFE000276894F85C2084F85D20002104F1600645
:10BFF000616661674022C4F86890C4F87080E666A4
:10C00000276604F1780009F097FE3A2084F8BA0018
:10C01000B96891F802A00AF0BF038B70606E01222C
:10C020007A7358B10768C6497B688B4204F168028D
:10C0300040F0598440680221FFF7E0F9002305220F
:10C040004FF4FA70BF49C4F8C0204FF0060E04F157
:10C05000BC0904F1DC084FF0070C04F1FC07C4F83C
:10C06000E02084F8F820C4F80021C4F82021C4F8A6
:10C07000C400C4F8E400C4F80401C4F82401C4F8FE
:10C08000BC10C4F8DC10C4F8FC1084F8D8E0C4F884
:10C09000E890C4F8088184F818C1C4F82871C4F87D
:10C0A000D460C4F8F460C4F81461C4F8C830C4F8AB
:10C0B000CC3084F8D03084F8D130C4F8EC3084F837
:10C0C000F03084F8F130C4F80C3184F8103184F881
:10C0D0001131C4F82C3184F8303184F8313194F9BD
:10C0E0005DA084F838E14AF07F074FF0010C04F5B9
:10C0F0008E7904F59E7E04F5AE7804F5BE7AC4F818
:10C100001C11C4F84021C4F84401C4F83C1184F85F
:10C110005821C4F86021C4F86401C4F85C11C4F863
:10C120008021C4F88401C4F87C11C4F8A021C4F8AB
:10C130003451C4F85451C4F87451C4F89451C4F83B
:10C140004891C4F868E1C4F888814FF0020E04F504
:10C15000CE7884F898C104F5DE79C4F84C3184F8BF
:10C16000503184F85131C4F86C3184F8703184F85E
:10C17000713184F87831C4F88C3184F8903184F8C6
:10C180009131C4F8A40184F85D70C4F8B451032758
:10C19000C4F8D451C4F8F451C4F8A8A1042504F596
:10C1A000EE7AC4F89C11C4F8C021C4F8C401C4F8E4
:10C1B000BC11C4F8E021C4F8E401C4F8DC11C4F8EF
:10C1C0000022C4F8040284F8B8E1C4F8C88184F8F5
:10C1D000D871C4F8E891C4F8AC3184F8B03184F86F
:10C1E000B131C4F8CC3184F8D03184F8D131C4F8FD
:10C1F000EC3184F8F03184F8F131C4F80C3284F871
:10C20000103284F8113204F5FE7984F8F851C4F83C
:10C2100008A204F50778C4F8FC1184F838C284F841
:10C2200058E204F50F7C04F5177EC4F82022C4F808
:10C230002402C4F81C12C4F84022C4F84402C4F812
:10C240003C12C4F86022C4F86402C4F85C1284F89A
:10C250007872C4F88022C4F88402FF2284F818326D
:10C26000C4F82C3284F8303284F83132C4F84C32BD
:10C2700084F8503284F85132C4F86C3284F8703249
:10C2800084F87132C4F81462C4F83462C4F8546299
:10C29000C4F87462C4F82892C4F84882C4F868C22A
:10C2A000C4F888E2C4F88C32606884F8985284F844
:10C2B000B92004F51F778268C4F87C1284F89032A4
:10C2C00084F89132C4F89462C4F89C7242F21071FE
:10C2D000D678B60609D5D3789D0606D5D578AD06AD
:10C2E00003D5D778BB0600F17381B02194F85E3096
:10C2F0009170826842F21075D778B90608D4D67862
:10C30000B70605D492F803C05FEA8C6140F1418121
:10C31000D578AF062BD5967846F0300191708268BB
:10C3200042F21075D778BE0612D4D678B1060FD473
:10C3300092F803C05FEA8C6140F16C8108E000BFB5
:10C34000E9B8000060A8010054A801009D090000A0
:10C350005B00DDB21571836842F21072DE78B707B8
:10C3600005D493F803C05FEA8C7640F1918161684F
:10C370008B6842F21070DF783D0627D4DD782A06FC
:10C3800024D493F803C05FEA0C621FD493F803A08F
:10C390005FEA0A671AD493F803905FEA096615D436
:10C3A00093F803805FEA086510D4DA7812060DD49A
:10C3B000DE7837060AD40838DDD1987000BF8F6860
:10C3C0008020B87000BF01250D7327E0022794F884
:10C3D0005D00DF708D68AB7843F01002AA708E6844
:10C3E00030718A6842F21070D778BF0708D4D578C8
:10C3F000AE0705D492F803C05FEA8C7640F129813C
:10C40000D7780220FDB2D07015F0100240F07C8287
:10C41000ED0700F16D8289680226CE7061688A6836
:10C4200092F802C00CF0C70393708B6842F2107050
:10C43000DE78B20600F1AC81216E8A6842F210709B
:10C44000D578AE0612D5D678B5060FD592F803C0CA
:10C450005FEA8C660AD592F803A05FEA8A6505D583
:10C4600092F803905FEA896300F1EE81B02094F8BE
:10C47000BA3090708A6842F21075D678B00612D43D
:10C48000D778BF060FD492F803C05FEA8C660AD44F
:10C4900092F803A05FEA8A6005D492F803905FEAFD
:10C4A000896740F10882D578AE062BD5977847F09A
:10C4B000300090708A6842F21075D678B6060DD4B6
:10C4C000D778B8060AD492F803C05FEA8C6605D420
:10C4D00092F803A05FEA8A6040F19D815B00DDB2C3
:10C4E00015718B6842F21072DF78BF070AD493F897
:10C4F00003C05FEA8C7605D493F803A05FEA8A70E4
:10C5000040F1BC81216E8B6842F21070DE783506F6
:10C5100000F1E180DD782A0600F1DD8093F803C0A8
:10C520005FEA0C6600F1D78093F803A05FEA0A6522
:10C5300000F1D18093F803905FEA096200F1CB80AB
:10C5400093F803805FEA086700F1C580DA78160681
:10C5500000F1C180DF783D0600F1BD800838D5D1FB
:10C56000987000BF8E688020B07000BF01250D73E9
:10C57000216E8A6892F802C00CF0C70393708B6832
:10C5800042F21070DF78BD0600F1D2802046BDE88F
:10C59000F08792F803A05FEA8A673FF5B9AE92F898
:10C5A00003905FEA89663FF5B3AE92F803805FEAD5
:10C5B00088613FF5ADAED1788F063FF5A9AED7784B
:10C5C000BE063FF5A5AE083D7FF496AE957019E026
:10C5D000D678B7067FF589AE92F803A05FEA8A663F
:10C5E0007FF583AE92F803905FEA89657FF57DAEB3
:10C5F00092F803805FEA88637FF577AE08397FF4AD
:10C6000067AE917000BF836880229A7000BF0126D8
:10C610000673ACE692F803A05FEA8A673FF598AE2E
:10C6200092F803905FEA89663FF592AE92F8038034
:10C630005FEA88613FF58CAED1788F063FF588AE12
:10C64000D778BE063FF584AE083D7FF46BAE95709B
:10C65000D8E792F803A05FEA8A753FF5D1AE92F869
:10C6600003905FEA89733FF5CBAE92F803805FEAEF
:10C6700088773FF5C5AED3789E073FF5C1AED67833
:10C68000B5073FF5BDAE08387FF4AEAE907095E6C5
:10C6900093F803A05FEA8A763FF569AE93F80390BA
:10C6A0005FEA89753FF563AE93F803805FEA8871AE
:10C6B0003FF55DAED9788F073FF559AEDF78BE07FD
:10C6C0003FF555AEDD78AD073FF551AE083A7FF442
:10C6D00045AE9A7096E7022694F8B900DE708D6830
:10C6E000AB7843F01002AA708F6838718A6842F202
:10C6F0001070D678B3070CD4D578AF0709D492F868
:10C7000003C05FEA8C7304D492F803A05FEA8A77CF
:10C710006CD5D6780220F5B2D07015F0100240F03A
:10C72000FB80EE0700F1068189680227CF701FE7C2
:10C73000DE78B2067FF52AAFDD78AD067FF526AF4D
:10C7400093F803A05FEA8A627FF520AF93F8039025
:10C750005FEA89677FF51AAF93F803805FEA88661E
:10C760007FF514AFDA7895067FF510AFDF78BA065B
:10C770007FF50CAF08387FF405AF987000BF8B6869
:10C780008020987000BF01260E732046BDE8F08718
:10C79000DF78BF067FF550AEDD78AA067FF54CAE98
:10C7A00093F803A05FEA8A677FF546AE93F803909B
:10C7B0005FEA89667FF540AE93F803805FEA88659B
:10C7C0007FF53AAEDA7892067FF536AEDE78B706B8
:10C7D0007FF532AE08387FF42BAE987000BF8B68BF
:10C7E0008020987000BF01270F7325E692F8039010
:10C7F0005FEA89768DD492F803805FEA887588D4E1
:10C80000D3789B0785D4D778BF0782D408387FF4C4
:10C8100070AF9070A5E692F803905FEA89673FF5E4
:10C820005DAE92F803805FEA88663FF557AED07838
:10C8300080063FF553AED678B7063FF54FAE083DBC
:10C840007FF43BAE957011E092F803805FEA886751
:10C850007FF50CAED3789E067FF508AED778BD067F
:10C860007FF504AE08387FF4EBAD907000BF8B68A5
:10C8700080229A7000BF01270F7343E693F803905C
:10C880005FEA89773FF53EAE93F803805FEA8876EA
:10C890003FF538AED87885073FF534AEDE78B0077F
:10C8A0003FF530AEDD78AF073FF52CAE083A7FF4A8
:10C8B0001BAE9A70DAE792F803805FEA88663FF56C
:10C8C000F2ADD07880063FF5EEADD678B7063FF5ED
:10C8D000EAAD083D7FF4D1AD9570C7E7114602225D
:10C8E0009847FFF77DBB114602229847FFF7A6BB8A
:10C8F0008B680126DE7000BF8F680873BA7000BFB6
:10C900008B6880229A7086E588681025C57000BF04
:10C9100003208F680022F0E788681025C57000BFEB
:10C920008E68032000220873B27000BF8B688022DB
:10C930009A70F9E68B680127DF7000BF8E68F2E716
:10C9400010B4036841681A7890F809C00C78037A2B
:10C9500014EA0C0F02EA03021DD0847A04F00301EA
:10C960000AB141F0040141F008039A1003F1FF3CC1
:10C970008272BCF10D0F0BD8DFE80CF021071B070A
:10C980000A152121150A071B0721C268531EC3601F
:10C990005DF8044B7047817A01F00303002AE4D06C
:10C9A00043F00403E1E7C3689C1EC4605DF8044BD8
:10C9B0007047C1685DF8044B0231C1607047C468BC
:10C9C0000134C4605DF8044B704700BF08B5034BE9
:10C9D000D3F8EC00FFF7B4FF08BD00BF9C42012074
:10C9E00008B5034BD3F8E800FFF7AAFF08BD00BF66
:10C9F0009C42012008B5034BD3F8E400FFF7A0FFE9
:10CA000008BD00BF9C42012008B5034BD3F8E000ED
:10CA1000FFF796FF08BD00BF9C42012008B5034BFD
:10CA2000D3F8DC00FFF78CFF08BD00BF9C4201205B
:10CA300008B5034BD3F8D800FFF782FF08BD00BF4D
:10CA40009C42012008B5034BD3F8D400FFF778FFD0
:10CA500008BD00BF9C42012008B5034BD3F8D000AD
:10CA6000FFF76EFF08BD00BF9C42012008B5034BD5
:10CA7000D3F8CC00FFF764FF08BD00BF9C42012043
:10CA800008B5034BD3F8C800FFF75AFF08BD00BF35
:10CA90009C42012008B5034BD3F8C400FFF750FFB8
:10CAA00008BD00BF9C42012008B5034BD3F8C0006D
:10CAB000FFF746FF08BD00BF9C42012008B5034BAD
:10CAC000D3F8BC00FFF73CFF08BD00BF9C4201202B
:10CAD00008B5034BD3F8B800FFF732FF08BD00BF1D
:10CAE0009C42012008B5034BD3F8B400FFF728FFA0
:10CAF00008BD00BF9C42012008B5034BD3F8B0002D
:10CB0000FFF71EFF08BD00BF9C42012008B5034B84
:10CB1000D3F8AC00FFF714FF08BD00BF9C42012012
:10CB200008B5034BD3F8A800FFF70AFF08BD00BF04
:10CB30009C42012008B5034BD3F8A400FFF700FF87
:10CB400008BD00BF9C42012008B5034BD3F8A000EC
:10CB5000FFF7F6FE08BD00BF9C42012008B5034B5D
:10CB6000D3F89C00FFF7ECFE08BD00BF9C420120FB
:10CB700008B5034BD3F89800FFF7E2FE08BD00BFED
:10CB80009C42012008B5034BD3F89400FFF7D8FE70
:10CB900008BD00BF9C42012008B5034BD3F89000AC
:10CBA000FFF7CEFE08BD00BF9C42012008B5034B35
:10CBB000D3F88C00FFF7C4FE08BD00BF9C420120E3
:10CBC00008B5034BD3F88800FFF7BAFE08BD00BFD5
:10CBD0009C42012008B5034BD3F88400FFF7B0FE58
:10CBE00008BD00BF9C42012008B5034BD3F880006C
:10CBF000FFF7A6FE08BD00BF9C42012008B5024B0E
:10CC0000D86FFFF79DFE08BD9C42012008B5024B7E
:10CC1000986FFFF795FE08BD9C42012008B5024BB6
:10CC2000586FFFF78DFE08BD9C42012008B5024BEE
:10CC3000186FFFF785FE08BD9C42012008B5024B26
:10CC4000D86EFFF77DFE08BD9C42012008B5024B5F
:10CC5000986EFFF775FE08BD9C42012008B5024B97
:10CC6000586EFFF76DFE08BD9C42012008B5024BCF
:10CC7000186EFFF765FE08BD9C42012008B5024B07
:10CC8000D86DFFF75DFE08BD9C42012008B5024B40
:10CC9000986DFFF755FE08BD9C42012008B5024B78
:10CCA000586DFFF74DFE08BD9C42012008B5024BB0
:10CCB000186DFFF745FE08BD9C42012008B5024BE8
:10CCC000D86CFFF73DFE08BD9C42012008B5024B21
:10CCD000986CFFF735FE08BD9C42012008B5024B59
:10CCE000586CFFF72DFE08BD9C42012008B5024B91
:10CCF000186CFFF725FE08BD9C42012008B5024BC9
:10CD0000D86BFFF71DFE08BD9C42012008B5024B01
:10CD1000986BFFF715FE08BD9C42012008B5024B39
:10CD2000586BFFF70DFE08BD9C42012008B5024B71
:10CD3000186BFFF705FE08BD9C42012008B5024BA9
:10CD4000D86AFFF7FDFD08BD9C42012008B5024BE3
:10CD5000986AFFF7F5FD08BD9C42012008B5024B1B
:10CD6000586AFFF7EDFD08BD9C42012008B5024B53
:10CD7000186AFFF7E5FD08BD9C42012008B5024B8B
:10CD8000D869FFF7DDFD08BD9C42012008B5024BC4
:10CD90009869FFF7D5FD08BD9C42012008B5024BFC
:10CDA0005869FFF7CDFD08BD9C42012008B5024B34
:10CDB0001869FFF7C5FD08BD9C42012001380B46EC
:10CDC0003A2800F25C82DFE810F053024C02450280
:10CDD0003E0237023002290222021B02AE01A701E5
:10CDE000A001990192018B0184017D0176016F01FF
:10CDF000680161015A0153014C0145013E013701AF
:10CE00003001290122011B0113010B010301FB0069
:10CE1000F300EB00E300DB00D300CB00C300BB005A
:10CE2000B300AB00A3009B0093008B0083007B004A
:10CE300073006B0063005B0053004B0043003B003A
:10CE4000BC4ABD49C2F8EC303B20042206F056BB78
:10CE5000B848BA49C0F8E83004223A2006F04EBB80
:10CE6000B44AB749C2F8E4303920042206F046BB80
:10CE7000B048B449C0F8E0300422382006F03EBB88
:10CE8000AC4AB149C2F8DC303720042206F036BB88
:10CE9000A848AE49C0F8D8300422362006F02EBB90
:10CEA000A44AAB49C2F8D4303520042206F026BB90
:10CEB000A048A849C0F8D0300422342006F01EBB98
:10CEC0009C4AA549C2F8CC303320042206F016BB98
:10CED0009848A249C0F8C8300422322006F00EBBA0
:10CEE000944A9F49C2F8C4303120042206F006BBA0
:10CEF00090489C49C0F8C0300422302006F0FEBAA9
:10CF00008C4A9949C2F8BC302F20042206F0F6BAA8
:10CF100088489649C0F8B83004222E2006F0EEBAB0
:10CF2000844A9349C2F8B4302D20042206F0E6BAB0
:10CF300080489049C0F8B03004222C2006F0DEBAB8
:10CF40007C4A8D49C2F8AC302B20042206F0D6BAB8
:10CF500078488A49C0F8A83004222A2006F0CEBAC0
:10CF6000744A8749C2F8A4302920042206F0C6BAC0
:10CF700070488449C0F8A0300422282006F0BEBAC8
:10CF80006C4A8149C2F89C302720042206F0B6BAC8
:10CF900068487E49C0F898300422262006F0AEBAD0
:10CFA000644A7B49C2F894302520042206F0A6BAD0
:10CFB00060487849C0F890300422242006F09EBAD8
:10CFC0005C4A7549C2F88C302320042206F096BAD8
:10CFD00058487249C0F888300422222006F08EBAE0
:10CFE000544A6F49C2F884302120042206F086BAE0
:10CFF00050486C49C0F880300422202006F07EBAE8
:10D000004C4A6949D3671F20042206F077BA494881
:10D010006649836704221E2006F070BA454A6449B7
:10D0200053671D20042206F069BA4248614903672C
:10D0300004221C2006F062BA3E4A5F49D3661B20D8
:10D04000042206F05BBA3B485C49836604221A203E
:10D0500006F054BA374A5A4953661920042206F09A
:10D060004DBA3448574903660422182006F046BAE0
:10D07000304A5549D3651720042206F03FBA2D489F
:10D08000524983650422162006F038BA294A5049CD
:10D0900053651520042206F031BA26484D49036530
:10D0A0000422142006F02ABA224A4B49D3641320E2
:10D0B000042206F023BA1F48484983640422122040
:10D0C00006F01CBA1B4A464953641120042206F09C
:10D0D00015BA1848434903640422102006F00EBA1A
:10D0E000144A4149D3630F20042206F007BA1148BD
:10D0F0003E49836304220E2006F000BA0D4A3C49E3
:10D1000053630D20042206F0F9B90A483949036334
:10D1100004220C2006F0F2B9064A3749D3620B20EC
:10D12000042206F0EBB903483449836204220A2042
:10D1300006F0E4B99C420120CDC90000E1C900001D
:10D14000F5C9000009CA00001DCA000031CA00006C
:10D1500045CA000059CA00006DCA000081CA00001B
:10D1600095CA0000A9CA0000BDCA0000D1CA0000CB
:10D17000E5CA0000F9CA00000DCB000021CB000079
:10D1800035CB000049CB00005DCB000071CB000027
:10D1900085CB000099CB0000ADCB0000C1CB0000D7
:10D1A000D5CB0000E9CB0000FDCB00000DCC00008A
:10D1B0001DCC00002DCC00003DCC00004DCC00006B
:10D1C0005DCC00006DCC00007DCC00008DCC00005B
:10D1D0009DCC0000ADCC0000BDCC0000CDCC00004B
:10D1E000DDCC0000EDCC0000FDCC00000DCD00003A
:10D1F0001DCD00002DCD00003DCD00004DCD000027
:10D200001F4A204953620920042206F077B91C48BE
:10D210001D4903620422082006F070B9184A1B4910
:10D22000D3610720042206F069B9154818498361C3
:10D230000422062006F062B9114A164953610520FE
:10D24000042206F05BB90E4813490361042210461C
:10D2500006F054B90A4A1149D3600320042206F0AB
:10D260004DB907480E4983600422022006F046B9F2
:10D27000034A0C4953600120042206F03FB970476D
:10D280009C4201205DCD00006DCD00007DCD0000F1
:10D290008DCD00009DCD0000ADCD00001518000023
:10D2A00081170000ED16000038B504464068A64D11
:10D2B00003689A68AA4240F05083F3F771FD206832
:10D2C00002684FF00041FD23D1625363D06A002809
:10D2D000FCDA6068936B02689368AB4240F03A8373
:10D2E000F3F754FD21680A684FF000401223D06222
:10D2F0005363D16A0029FCDA6068936B0268936813
:10D30000AB4240F02483F3F74BFD206802684FF0F6
:10D310000041AE23D1625363D06A0028FCDA606812
:10D32000936B02689368AB4240F00E83F3F738FDCD
:10D3300021680A684FF00040B323D0625363D16A7A
:10D340000029FCDA6068936B02689368AB4240F096
:10D35000F882F3F71BFD206802684FF0004191232B
:10D36000D1625363D06A0028FCDA6068936B02686C
:10D370009368AB4240F0E282F3F712FD21680A683D
:10D380004FF00040CA23D0625363D16A0029FCDA0F
:10D390006068936B02689368AB4240F0CC82F3F70D
:10D3A000F5FC206802684FF000413F23D1625363CF
:10D3B000D06A0028FCDA6068936B02689368AB421D
:10D3C00040F0B682F3F7ECFC21680A684FF00040A9
:10D3D000A223D0625363D16A0029FCDA6068936BA0
:10D3E00002689368AB4240F0A082F3F7CFFC20685C
:10D3F00002684FF000410023D1625363D06A0028D5
:10D40000FCDA6068936B02689368AB4240F08A82F2
:10D41000F3F7C6FC21680A684FF00040A123D062F0
:10D420005363D16A0029FCDA6068936B02689368E1
:10D43000AB4240F07482F3F7A9FC206802684FF019
:10D4400000410023D1625363D06A0028FCDA60688F
:10D45000936B02689368AB4240F05E82F3F7A0FCE6
:10D4600021680A684FF00040A023D0625363D16A5C
:10D470000029FCDA6068936B02689368AB4240F065
:10D480004882F3F783FC206802684FF000411423C0
:10D49000D1625363D06A0028FCDA6068936B02683B
:10D4A0009368AB4240F03282F3F770FC21680A685F
:10D4B0004FF000401123D0625363D16A0029FCDA97
:10D4C0006068936B02689368AB4240F01C82F3F78C
:10D4D00067FC206802684FF00041B523D1625363B6
:10D4E000D06A0028FCDA6068936B02689368AB42EC
:10D4F00040F00682F3F74AFC21680A684FF00040CA
:10D500000023D0625363D16A0029FCDA6068936B10
:10D5100002689368AB4240F0F081F3F741FC206869
:10D5200002684FF00041AB23D1625363D06A0028F8
:10D53000FCDA6068936B02689368AB4240F0DA8172
:10D54000F3F724FC02E000BF310C000021680A68F8
:10D550004FF000400123D0625363D16A0029FCDA06
:10D560006068936B02689368AB4240F0C081F3F748
:10D5700017FC206802684FF00041B423D162536366
:10D58000D06A0028FCDA6068936B02689368AB424B
:10D5900040F0AA81F3F7FAFB21680A684FF00040D7
:10D5A000A023D0625363D16A0029FCDA6068936BD0
:10D5B00002689368AB4240F09481F3F7E7FB206880
:10D5C00002684FF00041FD23D1625363D06A002806
:10D5D000FCDA6068936B02689368AB4240F07E812E
:10D5E000F3F7DEFB21680A684FF00040C123D062E8
:10D5F0005363D16A0029FCDA6068936B0268936810
:10D60000AB4240F06881F3F7C1FB206802684FF03D
:10D610000041FF23D1625363D06A0028FCDA6068BE
:10D62000936B02689368AB4240F05281F3F7B8FB0A
:10D6300021680A684FF00040C723D0625363D16A63
:10D640000029FCDA6068936B02689368AB4240F093
:10D650003C81F3F79BFB206802684FF000410F23E9
:10D66000D1625363D06A0028FCDA6068936B026869
:10D670009368AB4240F02681F3F792FB21680A6879
:10D680004FF00040B923D0625363D16A0029FCDA1D
:10D690006068936B02689368AB4240F01081F3F7C7
:10D6A0007FFB206802684FF00041B123D1625363D1
:10D6B000D06A0028FCDA6068936B02689368AB421A
:10D6C00040F0FA80F3F762FB21680A684FF00040EF
:10D6D000E223D0625363D16A0029FCDA6068936B5D
:10D6E00002689368AB4240F0E480F3F759FB20688E
:10D6F00002684FF00041D123D1625363D06A002801
:10D70000FCDA6068936B02689368AB4240F0CE80AD
:10D71000F3F73CFB21680A684FF00040A223D06277
:10D720005363D16A0029FCDA6068936B02689368DE
:10D73000AB4240F0B880F3F729FB206802684FF055
:10D7400000412023D1625363D06A0028FCDA60686C
:10D75000936B02689368AB4240F0A280F3F720FB22
:10D7600021680A684FF00040BB23D0625363D16A3E
:10D770000029FCDA6068936B02689368AB4240F062
:10D780008C80F3F703FB206802684FF000411F23F1
:10D79000D1625363D06A0028FCDA6068936B026838
:10D7A0009368AB4276D1F3F7FBFA21680A684FF031
:10D7B0000040B623D0625363D16A0029FCDA606866
:10D7C000936B02689368AB4261D1F3F7DFFA20688C
:10D7D00002684FF000410823D1625363D06A0028E9
:10D7E000FCDA6068936B02689368AB424CD1F3F744
:10D7F000D7FA21680A684FF00040BE23D062536315
:10D80000D16A0029FCDA6068936B02689368AB42C6
:10D8100037D1F3F7BBFA206802684FF000410723C5
:10D82000D1625363D06A0028FCDA6068936B0268A7
:10D830009368AB4222D1F3F7B3FA21680A684FF03C
:10D840000040A923D0625363D16A0029FCDA6068E2
:10D85000936B02689368AB420DD1F3F7A1FA246889
:10D8600025684FF00040AF21E8626963EA6A002A48
:10D87000FCDAAB6B38BD00219847F0E700219847F0
:10D88000DBE701219847C6E700219847B1E701216E
:10D8900098479CE70021984787E70121984772E75E
:10D8A000002198475CE70121984746E70121984706
:10D8B00030E7002198471AE70121984704E7002143
:10D8C0009847EEE600219847D8E601219847C2E63E
:10D8D00000219847ACE60121984796E60021984739
:10D8E00080E6012198476AE60121984754E6002125
:10D8F00098473EE60121984728E6002198470EE622
:10D9000001219847F8E500219847E2E50121984771
:10D91000CCE501219847B6E500219847A0E5012113
:10D9200098478AE50021984774E5012198475EE50C
:10D930000021984748E50121984732E500219847A2
:10D940001CE50121984706E500219847F0E40021F5
:10D950009847DAE401219847C4E400219047AEE4F7
:10D96000F8B58A7A90F89C600D460446D0F8981075
:10D97000002A00F0E48190F89E00012800F0E48184
:10D98000012391F85970B34027EA030C204681F82F
:10D9900059C050F8A01FAD4E0B68E97AB34240F071
:10D9A000FD81D4F8A40094F8A870002940F04281C9
:10D9B00094F8A910012900F04281012390F859E060
:10D9C000BB402EEA030180F859102046297B50F80D
:10D9D000AC3F1A68B24240F0E581D4F8B00094F848
:10D9E000B470002900F0CF8194F8B610012900F03E
:10D9F000CF81012390F859C003FA07F22CEA0207FD
:10DA000080F859702046697B50F8B82F1368B342EC
:10DA100040F0C681D4F8BC0094F8C070002900F032
:10DA2000A78194F8C210012900F0A781012390F882
:10DA300059E003FA07F22EEA020780F859702046EF
:10DA4000A97B50F8C42F1368B34240F0AD81D4F8DD
:10DA5000C80094F8CC60002900F07E8194F8CE10C4
:10DA6000012900F07E81012790F859C007FA06F2DB
:10DA70002CEA020E80F859E0E06EA97C0668B768CF
:10DA8000B847E87B616F94F87860002800F04C811B
:10DA900094F87A30012B00F04C81012791F859C09D
:10DAA00007FA06F22CEA020081F859002B7CD4F820
:10DAB000801094F88460002B00F02A8194F886008E
:10DAC000012800F02A81012791F859E007FA06F2AF
:10DAD0002EEA020C81F859C06E7CD4F88C1094F8B0
:10DAE0009050002E00F0088194F89200012800F078
:10DAF0000881012791F859E007FA05F22EEA020C95
:10DB000081F859C061688A6842F21070D678B6060A
:10DB100010D5D578AD060DD5D778BD060AD592F8C3
:10DB200003E05FEA8E6305D592F803C05FEA8C6775
:10DB300000F16A81B02094F85E3090708A6842F2F9
:10DB40001075D778B80610D4D678B7060DD492F8E9
:10DB500003E05FEA8E6008D492F803C05FEA8C6746
:10DB600003D4D078860640F18481D578A8062AD5DA
:10DB700092F802C04CF0300090708A6842F2107542
:10DB8000D778BE060DD4D678B0060AD492F803E052
:10DB90005FEA8E6005D492F803C05FEA8C6740F1BB
:10DBA0001C815B00DDB215718B6842F2107293F834
:10DBB00003C05FEA8C7706D4D878860703D4DF7871
:10DBC000BE0740F1398161688B6842F21070DE78DF
:10DBD00035063DD4DD782A063AD493F803E05FEAAF
:10DBE0000E6235D493F803C05FEA0C6730D4DA785C
:10DBF00016062DD4DF783D062AD4DE78320627D4E7
:10DC0000DD782F0624D40838E1D1987000BF8F68E2
:10DC10008020B87000BF01230B7361688C68A67800
:10DC200006F0C702A2708B6842F21070DD78AD0674
:10DC30003ED4F8BD94F8AA1001297FF4BEAE90F846
:10DC4000592001FA07F71743F9B2BCE6B50B0000FB
:10DC5000022294F85D00DA708F68BB7843F01006FA
:10DC6000BE708D6828718A6842F21070D778BB0741
:10DC70000DD492F803E05FEA8E7708D492F803C0DF
:10DC80005FEA8C7603D4D3789D0740F18F8092F8B9
:10DC900003C002205FFA8CF3D07013F0100240F042
:10DCA000FB80DE0700F1068189680225CD70B4E7AC
:10DCB000DF78BC06BDD5DC78A706BAD5DE78B60617
:10DCC000B7D593F803E05FEA8E65B2D593F803C049
:10DCD0005FEA8C64ADD5DA789206AAD5DD78AF0616
:10DCE000A7D50838A2D1987000BF8B6880209870A3
:10DCF00000BF01270F73F8BD94F8910001287FF44D
:10DD0000F8AE91F85930A84018435FFA80FCF7E666
:10DD100094F8850001287FF4D6AE91F85930B040D0
:10DD200018435FFA80FCD5E694F87930012B7FF434
:10DD3000B4AE91F85970B3403B43D8B2B4E690F812
:10DD40009D0001287FF41CAE91F8592000FA06F6D8
:10DD500016435FFA86FC19E694F8CD1001297FF48A
:10DD600082AE90F85930B14019435FFA81FE81E6E6
:10DD700094F8C11001297FF459AE90F85930B94098
:10DD80001943CFB259E694F8B51001297FF431AEAA
:10DD900090F85930B9401943CFB231E6984714E6AC
:10DDA00098474CE690472DE6984765E6D678B30746
:10DDB0003FF56DAFD578AF073FF569AFD778BE07B0
:10DDC0003FF565AF92F803E05FEA8E753FF55FAF10
:10DDD00008387FF44BAF907018E7D07886063FF58F
:10DDE000E0AED778B8063FF5DCAED678B7063FF59B
:10DDF000D8AE92F803E05FEA8E663FF5D2AE083DFA
:10DE00007FF4BEAE95700FE0D3789E067FF592AE9C
:10DE1000D678B5067FF58EAED578AB067FF58AAE9F
:10DE200008387FF473AE907000BF8B6880229A70C0
:10DE300000BF01270F73C6E6DE78B5073FF5C3AE16
:10DE4000DD78A8073FF5BFAE93F803E05FEA8E7771
:10DE50003FF5B9AE93F803C05FEA8C763FF5B3AEF9
:10DE6000D87885073FF5AFAE083A7FF4A0AE9A7038
:10DE7000DAE7D778B8063FF578AED678B7063FF53B
:10DE800074AE92F803E05FEA8E663FF56EAE083D31
:10DE90007FF457AE9570C7E788681023C37000BF42
:10DEA0008F68032000220873BA7000BF8E6880223A
:10DEB000B270F9E68E680125F57000BF8F68F2E751
:10DEC0004FF47A72704B02FB01F19942F0B400F208
:10DED000AF806E4CA14200F2AF806D4DA94200F2BE
:10DEE000AD806C4EB14200F2AE806B4FB94200F291
:10DEF000AE806A4B994200F2B080694CA14200F2B8
:10DF0000AE80684DA94200F28A804AF6A836B14236
:10DF100088BF4FF4807200F28380634F4FF4004655
:10DF20004FF48072B94280F08B8053005F4FB7FB93
:10DF3000F3FC614580F089801344B7FBF3F5A942F7
:10DF400080F087801344B7FBF3F4A14280F0838014
:10DF50001344B7FBF3FC614580F083801344B7FBA7
:10DF6000F3F5A9427FD21344B7FBF3F4A1427CD26C
:10DF70001344B7FBF3FC614579D21344B7FBF3F5C7
:10DF8000A94276D21344B7FBF3F7B94273D21344D4
:10DF9000464CB4FBF3FC61456FD21344B4FBF3F57C
:10DFA000A9426CD21344B4FBF3F7B9423ED21344F6
:10DFB000B4FBF3FC614564D21344B4FBF3F5A9420E
:10DFC00029D21344B4FBF3F2914228BF102223D28A
:10DFD000F024374D3549374A4FF47A7707FB03F37E
:10DFE000B1FBF3F34360286820F008072F6029682D
:10DFF00021F47F2C2CF47F6343F4602030432043D2
:10E00000286016683307FCD5294C256845F00802BE
:10E010002260F0BC70470F22511E0C01D9E780220C
:10E020005308224CB4FBF2F71E027BE70D22F3E704
:10E030001E4F0026012275E70222F1E70422EFE7D6
:10E0400013460024C5E70822EAE70222E4E710228B
:10E05000E6E70322E0E70422DEE72022E0E74022B1
:10E06000DEE70522D8E70622D6E70722D4E7082212
:10E07000D2E70922D0E70A22CEE70B22CCE70C2216
:10E08000CAE70E22C8E700BF4FA9AB00A7D45500CE
:10E0900053EA2A002975150094BA0A00495D050063
:10E0A000A4AE02005157010095BA0A000095BA0AC1
:10E0B0002C100B4024100B402DE9F04107468846F8
:10E0C00005F046FF194C1A4E054604E005F040FFE6
:10E0D000431BB34226D82368DB07F7D4154A1648FA
:10E0E000C2F80080076005F033FF144C104F06465D
:10E0F00004E005F02DFF851BBD4213D82568104BA9
:10E100000E492B40002BF4D00E480A6802600A60CA
:10E1100006680B4C3440A4F10104B4FA84F7780982
:10E12000BDE8F0810020BDE8F08100BF24100B4065
:10E1300040420F0008100B400C100B4030100B40F9
:10E1400001000F00D04401202DE9F04F85B03F4F72
:10E1500001900291039205F0FBFEDFF82CA13C4EEA
:10E16000BB468146DAF800803A4D05F0F1FE0446E0
:10E1700004E005F0EDFE011BA94225D83368D9075C
:10E18000F7D4354A3548C2F80080506005F0E0FE0B
:10E19000304C054604E005F0DBFE401BA04213D8DE
:10E1A00039682F4B0B40002BF5D02E4CDBF80000CC
:10E1B0002060CBF800002268294B1340012B03D1CB
:10E1C000294D2968CA050FD405F0C2FE214BC9EBC1
:10E1D00000049C42C6D9019840F23312292105B0AF
:10E1E000BDE8F04F04F018BF204D214F2B701A48A6
:10E1F000039B2049029E002222603B601E4A1F4B67
:10E2000006600A601E481F49B863196005F0A0FE49
:10E21000104E074604E005F09BFEC21BB2420BD82D
:10E220002B78002BF7D12468154D2540022D03D102
:10E23000012005B0BDE8F08F019840F23D12232186
:10E2400005B0BDE8F04F04F0E7BE00BF30100B4052
:10E2500024100B4040420F0008100B4000001A0D24
:10E2600001000F00D044012010100B40D4440120C5
:10E2700000100B4004100B40400001000C100B403C
:10E2800002007F1111003A06D84401202DE9F04F19
:10E2900093B0804605F05CFEA44CA54E054605E013
:10E2A00005F056FE411BB14200F2DC80236813F0FA
:10E2B0000100F5D19F49A04A0860106005F048FEB2
:10E2C0009E4C9B4D064605E005F042FE871BAF4283
:10E2D00000F2C88020689A4B984F0340002BF3D07F
:10E2E000DFF884A23968CAF800103960DAF8002033
:10E2F000934E1640012E40F0B5808C4EBB464FF039
:10E300000A0905F025FE8A4D044604E005F020FECA
:10E31000021BAA4225D83068C307F7D48549864D29
:10E32000884B834C4FF4D5720A602B6005F010FEC9
:10E33000054604E005F00CFE401BA04211D83868E9
:10E340007F4A0240002AF5D0DBF80030CAF80030DE
:10E35000CBF80030DAF80010794D0D40012D00F0B7
:10E36000DB81B9F10109CCD198F81110764B002965
:10E3700008BF4FF44013019305F0EAFD6F4F6B4C5B
:10E38000DFF8B0B10090B94605F0E2FD684E0546F1
:10E3900004E005F0DDFD431BB34258D8206810F0BF
:10E3A0000101F6D1644B694ACBF800101A6005F000
:10E3B000CFFD5F4D064604E005F0CAFD821BAA4270
:10E3C00045D838685E4901400029F5D0D9F80020C9
:10E3D000CAF80020C9F80020DAF80060584B334032
:10E3E000012B34D105F0B4FD514E054604E005F093
:10E3F000AFFD401BB0422AD82068C007F7D44E4B6F
:10E40000019A5349CBF80020196005F0A1FD484D51
:10E41000064604E005F09CFD811BA94217D8386828
:10E42000474901400029F5D0D9F80020CAF800205A
:10E43000C9F80020DAF80030414E1E40012E06D106
:10E4400005F086FD00993A4D401AA84215D940467C
:10E4500040F29112432104F0DFFD8346584613B089
:10E46000BDE8F08F40464FF4BF72202104F0D4FD88
:10E470008346584613B0BDE8F08F364B1A68002A21
:10E4800082DA354D196829601868284C410044BF6C
:10E490003248067005F05CFD254E074605E005F0A4
:10E4A00057FDC31BB34200F24181236813F00105FD
:10E4B000F5D12048204A2A490560116005F048FD41
:10E4C0001E4F1B4C064605E005F042FD851BA5428C
:10E4D00000F22C813D681A4B18482B40002BF3D0DA
:10E4E0000268CAF800200260DAF80010144E0E40EC
:10E4F000012E40F01B8105F02BFD0C4F0C4C054606
:10E5000005E005F025FD421BA24200F21F813B6899
:10E5100013F00106F5D10748074A12490660116059
:10E5200005F016FD054C024D074625E024100B4072
:10E5300040420F0008100B400C100B4030100B40F5
:10E5400001000F0000001A080000304000001A37D8
:10E550000000022910100B40C8440120C4440120CF
:10E560000000090200001A03D044012005F0F0FC6D
:10E57000C61BAE4200F2EA8026689D4B9D483340A0
:10E58000002BF3D00268CAF800200260DAF800100D
:10E59000974F0F40012F40F0D980974CDFF87892C9
:10E5A0002568964E964C2B0C1F04C9F8007005F098
:10E5B000CFFC054605E005F0CBFC401BB04200F265
:10E5C000CD802068C207F6D48E498F4C8F4A0F60E9
:10E5D000226005F0BDFC874D884C064605E005F03D
:10E5E000B7FC811BA14200F2B9802868804B814FA3
:10E5F0000340002BF3D03968CAF800103960DAF80C
:10E6000000207B4E1640012E40F0A8807A48DFF8AB
:10E610002CB204687E4EDBF80050009083683168AD
:10E6200088F83040220A200C88F82F2088F82C50D7
:10E63000220E88F82E002C0A280C2D0E4FEA132EDD
:10E6400088F8241088F8283088F82D2088F82B4086
:10E650000A0A1C0C090C1B0E88F82950002588F8A2
:10E660002A0088F8264088F8221088F827E088F8E1
:10E67000253088F8232088F83150D9F800106548F3
:10E68000654CFFF719FD002870D00098634B0268B5
:10E69000DBF800101B68306888F82150160A150C4A
:10E6A00088F81F6088F81E500E0A0D0C4FEA132CD4
:10E6B00088F8140088F8202088F81C1088F8183092
:10E6C000090E120E88F81B6088F81A501E0C050AF5
:10E6D0001B0E000C88F8191088F8120088F81D200D
:10E6E00088F817C088F8166088F8153088F8135035
:10E6F00021684B48FFF7E0FC00283FD021684948DB
:10E70000FFF7DAFC002841D1404640F2AB1240212D
:10E7100004F082FC8346ACE6374F3C68B4F5D57F05
:10E720000CD1414E88F81150019625E6404640F242
:10E730009912212104F070FC83469AE640464FF47A
:10E74000C272252104F068FC834692E640464FF4ED
:10E75000CE72222104F060FC83468AE6404640F2F5
:10E76000A112262104F058FC834682E640464FF46D
:10E77000D272272104F050FC83467AE6404640F2EC
:10E78000A712242104F048FC834672E602212748A0
:10E79000FFF792FC83460028B6D0254A254E116823
:10E7A000174C21F006031360156845F00200106055
:10E7B0004FF01012326005F0CBFB8DE80101D9F863
:10E7C00000800E4E05F0C4FB054604E005F0C0FBDA
:10E7D000401BB0424FD82168CB07F7D40948164BED
:10E7E000C0F80080436005F0B3FB044D06462CE002
:10E7F00001000F0030100B4010100B4040420F0082
:10E8000024100B4008100B400C100B4000000909AD
:10E810001C100B400000090AD844012018100B40BE
:10E8200000001B0700001A370000304000001A06E5
:10E8300028100B4044100B4000001A0D14100B4020
:10E8400005F086FB811BA94215D83A68484911405A
:10E850000029F5D0474B474E1868CAF800003060D1
:10E86000DAF80050424A44492A40012A03D1434B76
:10E870001868C00537D405F06BFB009D404E421B65
:10E88000B2429CD9DDF8048040F23312292140467F
:10E8900004F0C2FB00284FD146F2A811DFF81CA1FA
:10E8A000DFF81C91374F384E384D394C0020CAF8EC
:10E8B0000000C9F8000038603060286020604046E1
:10E8C000FFF7FEFA40F243424FF488634FF0010C29
:10E8D000CAF80020C9F800203B6032602A6022603C
:10E8E00088F810C0C5E52B4C2B4F2C4D3A700026F4
:10E8F00002AB0E60DDF80480294923606FF07F448D
:10E900002C602848284A294D0D60294E2949066067
:10E91000116005F01DFB1A4D044604E005F018FBDC
:10E92000031BAB421CD838780028F7D1DAF8007006
:10E930001F4A3A40022A13D19DF81540A307ABD5D0
:10E9400002AA1D494046FFF7FFFB0028A4D09DF80E
:10E95000187007F00F03012B9ED14CF250319DE748
:10E9600040F23D122321404604F056FB92E700BFDF
:10E9700001000F0030100B40D044012010100B405C
:10E9800040420F0008D004400CD0044010D0044096
:10E9900014D0044000100B40D444012008100B4058
:10E9A00004100B4038100B400C100B4040000100CD
:10E9B00002007F1111003A06F1FFFF8000D00440F1
:10E9C00004D004402DE9F041437D012B8CB062D08E
:10E9D000046EC26D944208D300239C4601F1FF38B7
:10E9E00098450CD00CB0BDE8F081651C0444056668
:10E9F00094F81CC001F1FF3863469845F2D1457D7B
:10EA00008DF808C0012D00F0A781076EC36D9F42ED
:10EA1000C0F0DF8000228DF809209F4280F05B82E9
:10EA20007E1C074406663A7F37468DF80A209F42CF
:10EA300080F04A827E1C074406663B7F8DF80B30CF
:10EA400004290DF1080E20D00EEB08010DF10B0288
:10EA5000002502248027012609E008F101038044F3
:10EA6000036698F81C3002F8013F91420DD0437DB7
:10EA7000012B00F0B480D0F86080C36D9845ECD3D2
:10EA8000002302F8013F9142F1D141687046884766
:10EA90000CB0BDE8F08100268DF803609DF80330CE
:10EAA000036942F21074DF783D0625D493F80380A1
:10EAB0005FEA086220D493F803C05FEA0C651BD4B8
:10EAC000DA78120618D4DD782F0615D4DE783606EB
:10EAD00012D4DF783D060FD493F803805FEA086212
:10EAE0000AD4083CDFD19C7000BF036980229A7071
:10EAF00000BF012404756FE79C7804F0E7029A7068
:10EB000003691D79EEB28DF803609F7847F0080421
:10EB10009C7003690222DA70036942F21074DD7896
:10EB2000AF071BD4DE78B60718D4DF78BF0715D43B
:10EB300093F803C05FEA8C7610D493F803805FEA01
:10EB400088750BD4DA78920708D4DD78AF0705D43E
:10EB5000DE78B60702D4083CE1D1C4E79C7804F023
:10EB6000C7079F70026942F21073D578AD0640F175
:10EB7000AD81D678B40640F1A98192F803C05FEA6E
:10EB80008C6540F1A38192F803805FEA886440F1CC
:10EB90009D81D478A70640F19981D778BE0640F1CF
:10EBA0009581D578AD0640F19181D678B40640F1D3
:10EBB0008D81083BD9D1937000BF02698024947085
:10EBC00000BF01250669057502273579F7709C4657
:10EBD00004E77E1C074406663A7F37461BE78DF83C
:10EBE00007509DF80730036942F2107893F803C08C
:10EBF0001CF0800F2ED193F803C01CF0800F29D198
:10EC000093F803C01CF0800F24D193F803C01CF0CC
:10EC1000800F1FD193F803C01CF0800F1AD193F816
:10EC200003C01CF0800F15D193F803C01CF0800FB7
:10EC300010D193F803C01CF0800F0BD1B8F1080875
:10EC4000D4D183F8028000BF03699F7000BF002306
:10EC5000067516E793F8028008F0E70C83F802C007
:10EC6000036993F804805FFA88FC8DF807C093F875
:10EC7000028048F0080C83F802C00369DC70036965
:10EC800042F2107893F803C01CF0020F23D193F8DE
:10EC900003C01CF0020F1ED193F803C01CF0020F3A
:10ECA00019D193F803C01CF0020F14D193F803C0DC
:10ECB0001CF0020F0FD193F803C01CF0020F0AD111
:10ECC00093F803C01CF0020F05D193F803C01CF0A9
:10ECD000020F00F0738193F8028008F0C70C83F8EC
:10ECE00002C0D0F8108042F2107C98F803309B06E6
:10ECF0002DD598F803309B0629D598F803309B064C
:10ED000025D598F803309B0621D598F803309B064B
:10ED10001DD598F803309B0619D598F803309B064B
:10ED200015D598F803309B0611D5BCF1080CDCD141
:10ED300088F802C000BF03699F7000BFD0F8108040
:10ED40000675634698F804C088F803408BE698F887
:10ED5000043088F8034086E600248DF806409DF8CC
:10ED60000630036942F21075DF783F0600F1B58086
:10ED7000DA78160600F1B180DE78340600F1AD8055
:10ED800093F803E05FEA0E6700F1A78093F803C0F1
:10ED90005FEA0C6600F1A180DC78240600F19D801A
:10EDA000DF783F0600F19980DA78160600F1958049
:10EDB000083DD9D19D7000BF036980249C7000BFBD
:10EDC0000127427D07750023012A8DF8093040F0A4
:10EDD000D48100258DF805509DF80530036942F275
:10EDE000107293F803C05FEA0C6700F11E8193F87C
:10EDF00003E05FEA0E6600F11881DC78270600F177
:10EE00001481DF783E0600F11081DE78340600F1CF
:10EE10000C81DD782F0600F1088193F803C05FEACA
:10EE20000C6600F1028193F803E05FEA0E6400F1E2
:10EE3000FC80083AD5D19A7000BF036980279F7083
:10EE400000BF0125447D05750023012C8DF80A3093
:10EE500040F0908100228DF804209DF80430036971
:10EE600042F2107593F803C05FEA0C6700F1AB80C3
:10EE700093F803E05FEA0E6600F1A580DC782706D0
:10EE800000F1A180DF783E0600F19D80DE78340637
:10EE900000F19980DA78170600F1958093F803C0A5
:10EEA0005FEA0C6600F18F8093F803E05FEA0E647E
:10EEB00000F18980083DD5D19D7000BF036980268F
:10EEC0009E7000BF012202750023B7E51379022767
:10EED0009C46D77082E50022A7E59D7805F0E706FD
:10EEE0009E70036993F804E05FFA8EFC8DF806C00B
:10EEF0009C7844F008079F7002690225D570036969
:10EF000042F21075DE78B4071DD493F803E05FEA8F
:10EF10008E7718D493F803C05FEA8C7413D4DC782E
:10EF2000A70710D4DF78BE070DD4DA7894070AD487
:10EF3000DE78B70707D493F803E05FEA8E7602D451
:10EF4000083DDFD136E79D7805F0C7049C70026963
:10EF500042F21073D778BE0640F10281D678B5062A
:10EF600040F1FE8092F803C05FEA8C6740F1F880C0
:10EF700092F803E05FEA8E6640F1F280D578AD0644
:10EF800040F1EE80D478A70640F1EA80D778BE063B
:10EF900040F1E680D678B50640F1E280083BD9D151
:10EFA000937000BF04698027A77000BF0126026923
:10EFB000067502251679D570427D05E7B8F1080877
:10EFC0007FF460AE3DE69D7805F0E7049C70036930
:10EFD0001F79FEB28DF804609A7842F008059D70A2
:10EFE00003690224DC70036942F21075DF78BC0704
:10EFF0004DD4DE78B7074AD4DA78970747D493F828
:10F0000003C05FEA8C7642D493F803E05FEA8E7423
:10F010003DD4DC78A7073AD4DF78BE0737D4DE7852
:10F02000B40734D4083DE1D146E79A7802F0E7040A
:10F030009C7003691F79FEB28DF805609D7845F0DC
:10F0400008029A7003690224DC70036942F21072AC
:10F05000DF78BC074DD4DE78B7074AD4DD78AF0738
:10F0600047D493F803C05FEA8C7642D493F803E068
:10F070005FEA8E743DD4DC78A7073AD4DF78BE0708
:10F0800037D4DE78B40734D4083AE1D1D3E69D789A
:10F0900005F0C7029A70046942F21073E778BE0661
:10F0A0005AD5E678B50657D594F803C05FEA8C6761
:10F0B00052D594F803E05FEA8E664DD5E578AD064B
:10F0C0004AD5E278970647D5E778BE0644D5E67874
:10F0D000B50641D5083BE1D1A37000BF0469802289
:10F0E000A27000BF01270469077502252679E57023
:10F0F000A4E49A7802F0C7059D70046942F2107387
:10F10000E778BE0631D5E678B5062ED5E2789706C3
:10F110002BD594F803C05FEA8C6626D594F803E0FB
:10F120005FEA8E6521D5E578AF061ED5E778BE0685
:10F130001BD5E678B50618D5083BE1D1A37000BF12
:10F1400007698025BD7000BF01260269067502248B
:10F150001679D470447D78E602252379E5706DE454
:10F1600002251379D570427D2EE602222379E270C2
:10F17000447D6AE6076EC36D59E4076EC36D4CE4C7
:10F1800008B5044B1A681AB101461046FFF71AFC7D
:10F1900008BD00BF984201202DE9F04F2DED028BF4
:10F1A0009FB00746482200210CA806F0C5FD07F5D0
:10F1B0001F5318460024FF2207F2A27501211430C4
:10F1C000DFF878B3DFEDDB8A9FEDDB8A01900395F2
:10F1D00007F51F5707940694089409940A940B9412
:10F1E00000948DF854208DF855208DF84E104FF076
:10F1F0000048D2480CA9F7F721F8D048DBF898600E
:10F20000009B0A930B9390F89040002E00F09A8395
:10F210009BF84890CA4A8DF82290D2ED007A27EEEA
:10F22000A80AB4EEC80AF1EE10FA40F14383B5EE35
:10F23000C00AF1EE10FA40F3CA83FCEEC00ACDED2D
:10F24000020A9DF808A0BF498DF818A091ED001A98
:10F2500061EE281AF4EEC81AF1EE10FA40F11F839D
:10F26000F5EEC01AF1EE10FA40F3A583BCEEE12AE8
:10F270008DED022A9DF808508DF81D50012E00F0EA
:10F2800014839BF849C0B04B8DF823C0D3ED002AFE
:10F2900022EEA83AB4EEC83AF1EE10FA40F1FD823F
:10F2A000B5EEC03AF1EE10FA40F38783FCEEC33AB4
:10F2B000CDED023A9DF80820A4488DF8192090ED74
:10F2C000004A64EE284AF4EEC84AF1EE10FA40F122
:10F2D000F682F5EEC04AF1EE10FA40F36983BCEE17
:10F2E000E45A8DED025A9DF808E08DF81EE0022EDA
:10F2F00000F0EC829BF84A9095498DF82490D1ED6E
:10F30000005A25EEA86AB4EEC86AF1EE10FA40F190
:10F31000D482B5EEC06AF1EE10FA40F35B83FCEEE6
:10F32000C66ACDED026A9DF808508A4B8DF81A50D6
:10F3300093ED007A67EE287AF4EEC87AF1EE10FACF
:10F3400040F1A082F5EEC07AF1EE10FA40F32B8383
:10F35000BCEEE70A8DED020A9DF808208DF81F200B
:10F36000032E00F095829BF84BA07B488DF825A0DA
:10F37000D0ED000A20EEA81AB4EEC81AF1EE10FA89
:10F3800040F1D882B5EEC01AF1EE10FA40F31983BD
:10F39000FCEEC11ACDED021A9DF808C06F498DF838
:10F3A0001BC091ED002A62EE282AF4EEC82AF1EE85
:10F3B00010FA40F1B482F5EEC02AF1EE10FA40F3F3
:10F3C000FE82BCEEE23A8DED023A9DF808508DF8CF
:10F3D0002050042E00F0A9829BF84C60604B8DF801
:10F3E0002660D3ED003A23EEA84AB4EEC84AF1EE07
:10F3F00010FA40F19182B5EEC04AF1EE10FA40F3F6
:10F40000E382FCEEC44ACDED024A9DF808E055497E
:10F410008DF81CE091ED005A65EE285AF4EEC85ABA
:10F42000F1EE10FA40F16682F5EEC05AF1EE10FAF4
:10F4300040F3BB82BCEEE56A8DED026A9DF8089050
:10F440008DF82190012C00F05C820024DBED2C6A09
:10F450008DF82740F5EEC06AF1EE10FA0DDDB2EE40
:10F460000E7A66EE877ABDEEE70A10EE100A00F01B
:10F47000010585F001068DF82860DBED2D0AF5EE1B
:10F48000C00AF1EE10FA0DDDB2EE0E1A60EE811A2E
:10F49000BDEEE12A12EE10AA0AF0010C8CF0010375
:10F4A0008DF82730304A30481478002C40F0D58150
:10F4B0002E4E224A2E4C92F8783D31782D4E2578EA
:10F4C0002D4A19433378147829432C4D19432C4B7A
:10F4D0002E781A782B4B21432B4C314325782B4E19
:10F4E0002B4C114329431D7832782A4B26782A4C1D
:10F4F00029431143294A1D78294B31431678294A5B
:10F500002943314325781E7814680C4B0594294310
:10F5100093F86A20059D31430170C5F30800002A65
:10F5200000F02182054E96F86B50002D00F0058208
:10F530003AE000BF00807F4300007F436C14FF1F50
:10F5400038D500204CD500203CD5002050D50020D7
:10F5500040D5002054D5002044D5002058D50020A7
:10F5600048D500205CD500201BD30020703DFF1F34
:10F57000FC58FF1F8874FF1F1490FF1FA0ABFF1FD4
:10F580002CC7FF1F44FEFF1FB8E2FF1FD019002049
:10F590005C350020E850002000880020746C0020BA
:10F5A0008CA30020EC440120002940F0D581AE4618
:10F5B0008DF82A5075469BF8A0409BF8A990009BB7
:10F5C0008DF82D908BF8A93034B1C3494FF0010C60
:10F5D00081F8A0308DF82CC09BF8A8208DF82F5012
:10F5E00042B1BD4E9DF8000086F8A80085F00105E7
:10F5F0008DF82F509BF8A74001988DF82E4006A952
:10F60000FEF7AEF94FF480420021B448DFF8E092F3
:10F6100006F092FBB049B248FBF764F8DDF80CA0A5
:10F62000D9F80460D9F808C0D9F80C50D9F81040BE
:10F63000D9F81400310C330A01F4706223F47F61AD
:10F6400042EA010E06F0F0064EEA060ED9F818104E
:10F65000D9F81C2059F8203FAAF802E04FEA1C46CE
:10F660004FEA1C2E06F470662EF47F6E46EA0E0EEC
:10F670000CF0F00C4EEA0C06AAF804604FEA154EA6
:10F680002E0A0EF4706C26F47F6E4CEA0E0605F01E
:10F69000F0053543AAF80650260C250A06F47066D4
:10F6A00025F47F65354304F0F0042C43060CAAF8DA
:10F6B0000840040A06F4706524F47F662E430C0AA1
:10F6C0000D0C00F0F000304305F4706624F47F6503
:10F6D0003543140A160C01F0F001294306F4706555
:10F6E00024F47F662E431C0A1D0C02F0F002324304
:10F6F000AAF80A0005F470667A48AAF80C1024F4F7
:10F700007F65354303F0F0032B438145AAF80E20B3
:10F710002AF8103F84D17868734A01688E6896424F
:10F7200040F03881F1F73CFB3C6825681523C5F8AB
:10F730002C806B63E86A0028FCDA78686A4A016802
:10F74000AB6B8E68964240F01D81F1F71FFB3C6861
:10F7500025681C23C5F82C806B63E86A0028FCDA56
:10F760007868614A0168AB6B8E68964240F0078109
:10F77000F1F70CFB3C6825685B23C5F82C806B63B4
:10F78000E86A0028FCDA7868574A0168AB6B8E6833
:10F79000964240F0F180F1F703FB3C682568752341
:10F7A000C5F82C806B63E86A0028FCDA78684E4A5A
:10F7B0000168AB6B8E68964240F0DB80F1F7E6FAA9
:10F7C0003C68009B2568C5F82C806B63E86A0028BC
:10F7D000FCDA7868444A0168AB6B8E68964240F068
:10F7E000C580F1F7D3FA3C6825683F23C5F82C8023
:10F7F0006B63E86A0028FCDA78683B4A0168AB6B07
:10F800008E68964240F0CC80F1F7CAFA3C682568D1
:10F810005C23C5F82C806B63E86A0028FCDA786802
:10F82000314A0168AB6B8C68FE68944240F0B58049
:10F83000F1F7ACFA3D6806F5FF502C681F3006F171
:10F84000FF3919F8013FC4F82C806363E16A00298D
:10F85000FCDA8145A36BF4D1CBE4244D1E4B2E681A
:10F860000596059A93F86A40C2F30800002C6ED101
:10F87000B0F5807F94BF002101219BF86B508DF87B
:10F880002A1098E6FF22032E8DF81F207FF46BAD1F
:10F89000012C7FF468ADA24667E5FF220CE5FF2549
:10F8A000012E8DF81D507FF4ECAC012C7FF4E9ACF7
:10F8B000A446E8E44FF0FF0AC5E4FF2535E54FF024
:10F8C000FF0E022E8DF81EE07FF414AD012C7FF4A4
:10F8D00011ADA14610E500BF6C14FF1F9802012076
:10F8E0009402012094420120310C0000EC440120DC
:10F8F000940201204FF0FF09012C8DF821907FF434
:10F90000A4ADDBF89420002A3FD18DF8294014469D
:10F91000012C7FF49AAD99E54FF0FF0E77E5FF25B6
:10F92000042E8DF820507FF457AD012C7FF454AD98
:10F93000264653E54FF0FF0C30E59DF800008DF8AA
:10F940002A0038E6012C7FF463ACA14662E4234927
:10F9500091F86B50002DF0D0B0F5807FAE468CBF93
:10F960000025012524E6002987D081E70121B04741
:10F9700039E70121B04723E70021B0470DE7012116
:10F98000B047F7E60121B047E1E6022A24D18DF81D
:10F9900028405AE50021B047C6E60121A04749E7C3
:10F9A0000021B04732E70022D8E44FF0000947E5D4
:10F9B0004FF0000E99E400255EE400227CE400256F
:10F9C00005E54FF0000CE9E44FF0000E1FE54FF0A5
:10F9D000000A38E40025A8E4144699E76C14FF1FD8
:10F9E0002DE9F04F2DED028BA1B0074648220021F2
:10F9F0000EA806F0A1F942F6F413002106ACFB585C
:10FA0000DB4A0991FF2508910A910B910C910D9108
:10FA1000069107910091204608218DF85C508DF8E1
:10FA20005D5006F0D7F907F51F5007F2A2721430A7
:10FA3000DFF848B3DFEDCF8A9FEDCF8A18940190AD
:10FA4000039207F51F574FF000480EA9CB48CB4C47
:10FA5000F6F7F4FBDBF89860009B0C930D9394F899
:10FA60009050002E00F09B839BF84890C4498DF87D
:10FA70002A90D1ED007A27EEA80AB4EEC80AF1EE7A
:10FA800010FA40F15683B5EEC00AF1EE10FA40F3D9
:10FA9000CB83FCEEC00ACDED020A9DF80820B948E0
:10FAA0008DF8202090ED001A61EE281AF4EEC81AA5
:10FAB000F1EE10FA40F13283F5EEC01AF1EE10FAD1
:10FAC00040F3A683BCEEE12A8DED022A9DF80830B2
:10FAD0008DF82530012E00F027839BF849A0AA4C11
:10FAE0008DF82BA0D4ED002A22EEA83AB4EEC83A45
:10FAF000F1EE10FA40F10083B5EEC03AF1EE10FAE3
:10FB000040F38883FCEEC33ACDED023A9DF808C07D
:10FB10009E498DF821C091ED004A64EE284AF4EE2A
:10FB2000C84AF1EE10FA40F10883F5EEC04AF1EE52
:10FB300010FA40F36B83BCEEE45A8DED025A9DF847
:10FB400008208DF82620022E00F0FD829BF84AE066
:10FB50008F488DF82CE0D0ED005A25EEA86AB4EE5F
:10FB6000C86AF1EE10FA40F1E682B5EEC06AF1EE35
:10FB700010FA40F35B83FCEEC66ACDED026A9DF895
:10FB80000830844C8DF8223094ED007A67EE287AA4
:10FB9000F4EEC87AF1EE10FA40F1A282F5EEC07AE6
:10FBA000F1EE10FA40F32C83BCEEE70A8DED020A69
:10FBB0009DF808908DF82790032E00F098829BF80E
:10FBC0004BA075498DF82DA0D1ED000A20EEA81AA2
:10FBD000B4EEC81AF1EE10FA40F1DA82B5EEC01AAE
:10FBE000F1EE10FA40F31B83FCEEC11ACDED021AC0
:10FBF0009DF8082069488DF8232090ED002A62EED8
:10FC0000282AF4EEC82AF1EE10FA40F1B682F5EE99
:10FC1000C02AF1EE10FA40F30083BCEEE23A8DED1B
:10FC2000023A9DF808308DF82830042E00F0AB829F
:10FC30009BF84C605A4C8DF82E60D4ED003A23EEC0
:10FC4000A84AB4EEC84AF1EE10FA40F19382B5EE3C
:10FC5000C04AF1EE10FA40F3E482FCEEC44ACDED66
:10FC6000024A9DF808C04F498DF824C091ED005A12
:10FC700065EE285AF4EEC85AF1EE10FA40F16882A7
:10FC8000F5EEC05AF1EE10FA40F3BD82BCEEE56A23
:10FC90008DED026A9DF808E08DF829E0012D00F055
:10FCA0005E820025DBED2C6A8DF82F50F5EEC06AE0
:10FCB000F1EE10FA0DDDB2EE0E7A66EE877ABDEE49
:10FCC000E70A10EE100A00F0010989F0010A8DF828
:10FCD00030A0DBED2D0AF5EEC00AF1EE10FA0DDDD5
:10FCE000B2EE0E1A60EE811ABDEEE12A12EE103A63
:10FCF00003F0010686F001048DF82F402A4A2A48B5
:10FD00001578002D40F0D781284E1C4C284A94F8D5
:10FD1000785D3178274B16781C782943264D31437E
:10FD2000264E2A7833782143254C1143254A2578DD
:10FD30001678254C1943254B2278254C29431D78EC
:10FD40003143244E294333782578234C1143234AE9
:10FD500019431678224B234A294331431D782678CC
:10FD60001368064C0593294394F86A203CE000BFD1
:10FD700038AB010000807F4300007F436C14FF1FFD
:10FD800038D500204CD500203CD5002050D500208F
:10FD900040D5002054D5002044D5002058D500205F
:10FDA00048D500205CD500201BD30020703DFF1FEC
:10FDB000FC58FF1F8874FF1F1490FF1FA0ABFF1F8C
:10FDC0002CC7FF1FB8E2FF1FD019002044FEFF1F01
:10FDD000E85000205C3500208CA30020746C0020CB
:10FDE00000880020EC440120059D31430170C5F3DB
:10FDF0000800002A00F0E481C14E96F86B30002B19
:10FE000000F0C881002940F0D4819C468DF8323042
:10FE100063469BF8A0509BF8A9E0009C8DF835E064
:10FE20008BF8A94035B1B6494FF0010A81F8A040DE
:10FE30008DF834A09BF8A8208DF8373042B1B04E31
:10FE40009DF8000086F8A80083F001038DF8373094
:10FE50009BF8A75001988DF8365008A9FDF780FD52
:10FE60004FF480420021A748DFF8AC9205F064FF10
:10FE7000A349A548FAF736FCDDF80CA0D9F80460D0
:10FE8000D9F808C0D9F80C50D9F81040D9F81400A6
:10FE9000320A310C01F4706122F47F6E41EA0E0ED9
:10FEA00006F0F0064EEA060ED9F81810D9F81C2014
:10FEB00059F8203FAAF802E04FEA1C464FEA1C2EF0
:10FEC00006F470662EF47F6E46EA0E0E0CF0F00C0F
:10FED0004EEA0C06AAF804604FEA154E2E0A0EF4FC
:10FEE000706C26F47F6E4CEA0E0605F0F005354383
:10FEF000AAF80650260C250A06F4706625F47F65DC
:10FF0000354304F0F0042C43060CAAF80840040A18
:10FF100006F4706524F47F662E430C0A0D0C00F085
:10FF2000F000304305F4706624F47F653543140A0D
:10FF3000160C01F0F001294306F4706524F47F6685
:10FF40002E431C0A1D0C02F0F0023243AAF80A00EC
:10FF500005F470666D48AAF80C1024F47F653543EB
:10FF600003F0F0032B438145AAF80E202AF8103F36
:10FF700084D17868664A01688E68964240F037817D
:10FF8000F0F70EFF3C6825681523C5F82C806B63DD
:10FF9000E86A0028FCDA78685D4A0168AB6B8E6815
:10FFA000964240F01C81F0F7F1FE3C6825681C2366
:10FFB000C5F82C806B63E86A0028FCDA7868544A3C
:10FFC0000168AB6B8E68964240F00681F0F7DEFE6A
:10FFD0003C6825685B23C5F82C806B63E86A0028C1
:10FFE000FCDA78684A4A0168AB6B8E68964240F04A
:10FFF000F080F0F7D5FE3C6825687523C5F82C80A5
:020000021000EC
:100000006B63E86A0028FCDA7868414A0168AB6BE8
:100010008E68964240F0DA80F0F7B8FE3C68009BAC
:100020002568C5F82C806B63E86A0028FCDA7868DC
:10003000374A0168AB6B8E68964240F0C480F0F797
:10004000A5FE3C6825683F23C5F82C806B63E86AF1
:100050000028FCDA78682E4A0168AB6B8E689642FD
:1000600040F0CB80F0F79CFE3C6825685C23C5F827
:100070002C806B63E86A0028FCDA7868244A0168FF
:10008000AB6B8C68FE68944240F0B480F0F77EFE63
:100090003D6806F5FF502C681F3006F1FF3919F84E
:1000A000013FC4F82C806363E16A0029FCDA8145D2
:1000B000A36BF4D1C9E4174B114A1E680596059C41
:1000C00092F86A50C4F30800002D6DD1B0F5807F1E
:1000D00094BF002101219BF86B308DF8321098E617
:1000E0004FF0FF09032E8DF827907FF468AD012DA6
:1000F0007FF465ADAA4664E54FF0FF0C08E500BF4C
:100100006C14FF1F980201209402012094420120E8
:10011000310C0000EC44012094020120FF23012E49
:100120008DF825307FF4D9AC012D7FF4D6ACAA46EA
:10013000D5E4FF22B3E4FF2323E5FF22022E8DF84E
:1001400026207FF403AD012D7FF400ADAE46FFE421
:100150004FF0FF0E012D8DF829E07FF4A2ADDBF802
:100160009420002A3ED18DF831501546012D7FF4A0
:1001700098AD97E54FF0FF0C75E5FF23042E8DF841
:1001800028307FF455AD012D7FF452AD2E4651E558
:10019000FF222FE59DF800008DF8320039E6012D91
:1001A0007FF462ACA94661E4224991F86B30002BE0
:1001B000F0D0B0F5807F9C468CBF0023012325E65C
:1001C000002988D082E70121B0473AE70121B047F2
:1001D00024E70021B0470EE70121B047F8E60121EE
:1001E000B047E2E6022A23D18DF8305059E50021CC
:1001F000B047C7E60121A0474AE70021B04733E7EF
:100200004FF00009D6E44FF0000E45E5002298E4D7
:1002100000235DE44FF0000C7AE4002303E50022A4
:10022000E8E44FF0000C1EE5002238E40023A8E4C7
:1002300015469BE76C14FF1F2DE9F04FADF51D7DB2
:1002400005460190482200210AA805F075FD00240A
:10025000FF2301220AA9CE488DF84C308DF84D308D
:100260008DF8482004940594069407940894099402
:10027000F5F7E4FF04A9C648C64EF7F76BFD05F590
:100280001F5004A91430FDF76BFB21464FF4804248
:10029000C14805F051FDBE49C048FAF723FA05F2FE
:1002A000A27A06F5804BD6F804E0B768F5683469A1
:1002B00006F114084FEA1E494FEA1E2C98E8070081
:1002C00009F470682CF47F694FEA174C48EA090872
:1002D0000CF470694FEA172C2CF47F6C0EF0F00EC2
:1002E00049EA0C0948EA0E0E4FEA154C4FEA152868
:1002F0000CF4706C07F0F00728F47F684CEA0808EB
:1003000049EA07074FEA144C4FEA14290CF4706CC1
:1003100005F0F00529F47F694CEA090948EA05056A
:100320004FEA104C4FEA10280CF4706C04F0F00403
:1003300028F47F684CEA080849EA04044FEA114CA3
:100340004FEA11290CF4706C00F0F00029F47F6979
:1003500056F8203FAAF802E04CEA090948EA0000F2
:100360004FEA124C4FEA12280CF4706C01F0F001C5
:1003700028F47F684CEA080849EA01014FEA134C67
:100380004FEA13290CF4706C29F47F6902F0F00233
:100390004CEA090C03F0F00348EA0208B3454CEAC2
:1003A0000302AAF80470AAF80650AAF80840AAF8AE
:1003B0000A00AAF80C10AAF80E802AF8102F7FF471
:1003C00072AF019E764F06F51F5ADAF804000568F1
:1003D000AC68BC4240F0F681F0F7E2FCDAF80000CD
:1003E00002684FF000411523D1625363D66A002E94
:1003F000FCDADAF80400936B0568AC68BC4240F0A4
:10040000DE81F0F7C3FCDAF8000002684FF000412B
:100410001C23D1625363D66A002EFCDADAF804009A
:10042000936B0568AC68BC4240F0C681F0F7AEFC47
:10043000DAF8000002684FF000415B23D162536399
:10044000D66A002EFCDADAF80400936B0568AC6813
:10045000BC4240F0AE81F0F7A3FCDAF8000002687D
:100460004FF000417523D1625363D66A002EFCDA47
:10047000DAF80400936B0568AC68BC4240F09681E2
:10048000F0F784FCDAF8000002684FF00041002326
:10049000D1625363D66A002EFCDADAF80400936B5B
:1004A0000568AC68BC4240F07E81F0F76FFCDAF87A
:1004B000000002684FF000413F23D1625363D66AC7
:1004C000002EFCDADAF80400936B0568AC68BC42D5
:1004D00040F06681F0F764FCDAF8000002684FF043
:1004E00000415C23D1625363D66A002EFCDADAF84D
:1004F0000400936B0568DAF80C40AA68BA4240F031
:100500004C81F0F743FCDAF8007004F5FF503E68C8
:100510001F3004F1FF3B4FF000411BF8013FF16237
:100520007363F56A002DFCDA5845B36BF5D1019E73
:100530001C4A1D491D4FDFF878A006F527594C4687
:100540002C3442F6EC18039446F80820B34606F51E
:10055000285042F6F813039E0022042442F23E552E
:100560007460B560CC464BF803200BF5265302931C
:100570004FF0FF0E69248CF83E208CF83CE08CF89C
:100580003F4002600298CCF84410DFF828B013E036
:100590006C14FF1F94020120980201209402012094
:1005A000310C00004B45454EE7CBA39230100B4079
:1005B000D8440120D0440120844E00F1380102913A
:1005C000B946DAF80080824D03F0C2FC044604E02C
:1005D00003F0BEFC031BAB42F3D83268D307F7D459
:1005E0007C487D4BC0F80080436003F0B1FC784C40
:1005F000054604E003F0ACFC411BA142E1D8396898
:10060000764A0A40002AF5D0D9F80030CBF80030FD
:10061000C9F80030DBF80000704D714C0540012D29
:10062000CFD170490A68D005CBD5DFF8DC916E4E8A
:10063000684889F800500023039D6C496C4F236083
:100640006C4A35604FF4813403606B4B74603B60DF
:100650000A6003F07DFC5E4E054605E003F078FC81
:10066000431BB34200F2908099F800000028F5D1B6
:10067000DBF8007060493940022940F085801CA8F1
:100680004FF40072002100245C4F504E05F054FBE3
:100690000194019A01320192DAF800804C4D03F086
:1006A00057FC044604E003F053FC001BA842F3D8B7
:1006B0003068C107F7D4474B4749C3F800805960F9
:1006C00003F046FC424C054604E003F041FC421BAB
:1006D000A242E1D83A68414810400028F5D0474985
:1006E000464D0B68CBF800302B60DBF800403B48F0
:1006F0003B4920400128CFD13A4A1368DA05CBD5CF
:1007000000240C603E49384D0A7889F800001CA886
:10071000286052BB019B5D022E483A4C344A05606A
:100720004FF48131344B334D21601360A56003F0E9
:100730000FFC274D044604E003F00AFC031BAB4208
:1007400015D899F80020002AF6D1DBF800002A49D4
:10075000014002290BD1019C42F24735AC4298D1AD
:1007600000200DF51D7DBDE8F08F019DD4E74FF40D
:1007700002723321029802F04FFC0028EBD10620D0
:100780000DF51D7DBDE8F08F4FF402723321029804
:1007900002F042FC0028F2D071E701219047B2E656
:1007A0000021A04798E60121A04780E60121A0474B
:1007B00068E60021A04750E60121A04738E6012164
:1007C000A04720E60021A04708E600BF24100B4008
:1007D00040420F0008100B4000001A0D01000F00EE
:1007E000D044012010100B4000100B400C100B40A7
:1007F00038100B4027003A1902007F1130100B40CF
:10080000C444012004100B40D44401202DE9F04FD2
:10081000044689B072B6D0F8443662B6754FD0F847
:100820005826396805910598D4F85C569E08821AB6
:10083000711BD4F8603618BFC4F85806012AB8BF37
:1008400001228802C4F85C6690FBF2F513B1002D1A
:1008500040F08F8403EB4302531948BF03339D10CC
:1008600094F86806C4F86056002DB8BF6D420028A1
:1008700000F09283604EA5F1020B86FB0B0CACEBF3
:10088000EB700130D4F8643604F53155303500FB97
:100890000131C4F86416E96272B6D4F8786662B6BB
:1008A0003A6806920698D4F88C26D4F89016B308C5
:1008B000591AA0EB0206C4F89036D4F8943618BF43
:1008C000C4F88C06012EB8BF0126880290FBF6F210
:1008D00013B1002A40F0438403EB4303981848BF48
:1008E0000330861094F89C26C4F89466002EB8BF96
:1008F0007642002A00F01F843F4BA6F1020883FBDA
:100900000802A2EBE8760136D4F89806DFF8E88012
:1009100006FB010104F53256C4F898162036296307
:10092000204604F5827E4FF0000C15E082EAE27961
:10093000A9EBE27AAAF1020388FB0392A2EBE3712E
:100940000131D0F8CC3601FB0B32C0F8CC26343064
:10095000704546F8042F51D072B6D0F8AC3662B666
:100960003A680792DDF81C90D0F8C026D0F8C4167B
:100970009B08B3EB010BC2EB0902C0F8C436D0F8F8
:10098000C83618BFC0F8C096012AB8BF01224FEA86
:100990008B2A9AFBF2F223B1002A02D024DD002B2D
:1009A00024DD03EB43018B1848BF033390F8D016C6
:1009B0009A10C0F8C8260029B8D182EAE273A3EBE6
:1009C000E279A9F10201012912DD4FEAA10AAAF197
:1009D0000B0222EAE273AAF104010029A8BF5B1806
:1009E0000AF101029918ACE7002BDADDC0F8C8C69D
:1009F0000121A6E7EC440120ABAAAA2A04F56670FF
:100A0000FAF77AFF94F8E80494F8C81494F8E92403
:100A100094F8C93494F8687494F86964287594F863
:100A20008804A97594F889146A7594F8A824EB755C
:100A300094F8A9346B772F766E76A876E9762A77C4
:100A400042F6704794F8A86594F8C805E6556870B2
:100A500094F8E815A97094F80826EA7094F82836F6
:100A60002B7194F8A9756F7194F8C965AE7194F8FB
:100A7000E905E87194F80916297294F829266A7232
:100A800094F80835AB7294F82875EF7294F84865BD
:100A90002E7394F86805687394F88815A97394F810
:100AA0000925EA7394F829352B7494F849756F7405
:100AB00004F52F5B94F86965AE74DBF8A80094F830
:100AC000892585F825004FF0FF33DBF8AC10EA7478
:100AD00004F53258CBF8A83085F824109BF8A5709F
:100AE0009BF8A460CBF8AC30294685F8237085F8D4
:100AF0002260DF4808F1380A42F6CD45F5F79EFB43
:100B0000DB485146F7F726F9675DDA4804F51F58C8
:100B1000002F40F05882019042F6CF4742F66546DA
:100B2000E15DA15542F6B84504F51F505146143019
:100B3000FCF716FF605DD04A9AF8161040F2145385
:100B400003FB00F082FB005CC7178444C7EBEC1B7F
:100B500004F522590BF5FA66A9F830609AF80150AD
:100B600003FB05F582FB057CAC44E817C0EBEC17F2
:100B700042F6B20B07F5FA6624F80B609AF80250B9
:100B800003FB05F582FB057CAC44E817C0EBEC17D2
:100B900042F6B40B07F5FA6624F80B609AF8035096
:100BA00003FB05F582FB057CAC44E817C0EBEC17B2
:100BB00042F6B60B07F5FA6624F80B609AF8045073
:100BC00003FB05F582FB057CAC44E817C0EBEC1792
:100BD00042F6B80B07F5FA6624F80B609AF8055050
:100BE00003FB05F582FB057CAC44E817C0EBEC1772
:100BF00007F5FA66A9F83A609AF8060003FB00F0D8
:100C000082FB00698144C517C5EBE91B42F6BC07AE
:100C10000BF5FA66E6539AF8070003FB00F082FB37
:100C2000006C8444C517C5EBEC1942F6BE0709F504
:100C3000FA66E6539AF8080003FB00F082FB006BAB
:100C4000C5178344C5EBEB1C04F523590CF5FA6773
:100C5000A9F800709AF8096003FB06F382FB030A07
:100C60009A44DB17C3EBEA1042F6C20200F5FA65BC
:100C7000A55242F2D077002900F06F81E15D002992
:100C800000F0AF824FF4804200217C48DFF8F491FD
:100C900005F052F876497A48F9F724FD04F2A27A71
:100CA00009F5804BD9F80470D9F80860D9F80C50D0
:100CB000D9F8104009F1140E9EE807004FEA174CCE
:100CC0004FEA172E2EF47F6E0CF4706C4CEA0E0C6B
:100CD00007F0F0074FEA164E4CEA07074FEA162CCA
:100CE0000EF4706E2CF47F6C4EEA0C0C06F0F006DD
:100CF0004FEA154E4CEA06064FEA152C0EF4706EBC
:100D00002CF47F6C4EEA0C0C05F0F0054FEA144E03
:100D10004CEA05054FEA142C0EF4706E2CF47F6C2F
:100D20004EEA0C0C04F0F0044FEA104E4CEA0404B6
:100D30004FEA102C0EF4706E2CF47F6C4EEA0C0C03
:100D400000F0F0004FEA114E4CEA00004FEA112C7F
:100D50000EF4706E2CF47F6C4EEA0C0C01F0F00176
:100D60004FEA124E4CEA01014FEA122C59F8203F8B
:100D7000AAF802702CF47F6C0EF4706E4EEA0C0E22
:100D800002F0F0024FEA134C4EEA02024FEA132E31
:100D90002EF47F6E0CF4706C4CEA0E0C03F0F00332
:100DA0004CEA030ECB45AAF80460AAF80650AAF84C
:100DB0000840AAF80A00AAF80C10AAF80E202AF88F
:100DC00010EF7FF46FAFD8F80400019D0768BE688C
:100DD000AE4240F00082EFF7E3FFD8F8004022680F
:100DE0004FF000401521D0625163D36A002BFCDA2A
:100DF000D8F80400019D0768936BBE68AE4240F0CE
:100E0000E781EFF7C3FFD8F8004022684FF00040B9
:100E10001C21D0625163D36A002BFCDAD8F804009D
:100E2000019D0768936BBE68AE4240F0BE81EFF74C
:100E3000ADFFD8F8004022684FF000405B21D0623F
:100E40005163D36A002BFCDAD8F80400019D0768CF
:100E5000936BBE68AE4240F0A581EFF7A1FFD8F8D2
:100E6000004022684FF000407521D06251630BE0D2
:100E70006C14FF1F310C00008180808098020120DB
:100E80009402012094020120D36A002BFCDAD8F8E6
:100E90000400019D0768936BBE68AE4240F07F81FD
:100EA000EFF774FFD8F8004022684FF000400021AF
:100EB000D0625163D36A002BFCDAD8F80400019D9C
:100EC0000768936BBE68AE4240F06681EFF75EFF45
:100ED000D8F8004022684FF000403F21D0625163B3
:100EE000D36A002BFCDAD8F80400019D0768936BE5
:100EF000BE68AE4240F04D81EFF752FFD8F8004097
:100F000022684FF000405C21D0625163D36A002B0D
:100F1000FCDAD8F80400019C0768936BBD68D8F828
:100F20000C60A54240F03281EFF730FFD8F8002086
:100F300006F5FF5017681F3006F1FF384FF00041EB
:100F400018F8013FF9627B63FE6A002EFCDA8045E7
:100F5000BB6BF5D109B0BDE8F08FE65D002E3FF424
:100F600091AED8F80400019A03689D68954240F05C
:100F70006781EFF715FFD8F8001008684FF00047B9
:100F8000AF26C7624663C36A002BFCDA42F2D07513
:100F90000022836B625575E6AE1E012E40F3F08091
:100FA000B310A3F10B09A3F1040A29EAE972BAF11B
:100FB000000FA8BF524401331A44012A00F0E08018
:100FC000551E68005EE402460190D8F804000168EE
:100FD0008B68934240F0D780EFF7E2FED8F80060CC
:100FE00035684FF00040C122E8626A63E96A00296F
:100FF000FCDAD8F80400AB6B0368019D9E68AE4232
:1010000040F0EC80EFF7C2FED8F8000001684FF026
:101010000042CA624F63CB6A002BFCDAD8F80400A6
:101020008B6B0668019AB56817F0010140F0C0802B
:10103000954240F0F080EFF7B3FED8F80020136837
:101040004FF00040A721D8625963DE6A002EFCDA17
:1010500004F5265C9B6BDFF804927A4D8CF87C706B
:101060000CF1380B04F527532C3303932746764CA9
:10107000764E2268029202F06BFF044604E002F012
:1010800067FF001BB042F2D82868C107F7D4704E42
:101090000299704B3160736002F05AFF6B4C064648
:1010A00004E002F055FF821BA242E0D8D9F80020EC
:1010B000694810400028F4D0684B694E674C1968A5
:1010C000674A316021601068634B65490340012B1A
:1010D000CDD1644E3468E205C9D5634D634A2B70A7
:1010E0005B4800230B60039911604FF48136036065
:1010F0003C465F4B5F4F56605F48604A38601A60FD
:1011000002F026FF514F064604E002F021FF821B49
:10111000BA4209D829780029F7D1514D564B286891
:101120000340022B3FF4F8AC58464FF402723321CF
:1011300001F072FFF0E4B31E012B17DD9E10A6F143
:101140000B00331F20EAE072002BA8BFD218013633
:101150003244012A0AD0501E4600FFF7D5BB5CDDA1
:10116000002B3FF7B9AB0026C4F894660126FFF7C1
:10117000CBBB59DD002B3FF76DAB0026C4F8606692
:101180000120FFF77FBB0021984727E70121A847EF
:10119000CCE60021B047B1E60121B04798E6012135
:1011A000B0477FE60021B04759E60121B04740E64D
:1011B000954242D1EFF7F4FDD8F8000003684FF0F4
:1011C0000041A626D9625E63DD6A002DFCDA3FE7A6
:1011D0000121B04717E60021B047FEE50121B047E5
:1011E00012E7D8F80400019B0768BE689E4222D12E
:1011F000EFF7D6FDD8F8001008684FF00045AE2292
:10120000C5624263C76A002FFCDA42F2D076012140
:10121000836BA15536E5A8470FE7002B7FF75CAB42
:101220000026C4F89466A1E7002B7FF713AB0026D5
:10123000C4F86066A4E7B047DCE70021A847BBE735
:10124000A84798E624100B40D844012040420F00E4
:1012500008100B4000001A0D01000F0030100B4069
:10126000D044012010100B40D444012000100B404A
:101270000C100B4038100B4002007F1127003A1968
:101280002DE9F04F2DED028B0446C84BC848C949E3
:10129000C94D6460002285B02060A160E26003F562
:1012A000A07EA3461F68D3F808905C68D3F818C0E6
:1012B0001E6A986A196B9A6B05EBC70805EBC9099A
:1012C0001F69D8F804A005EBC708CAF80040D9F890
:1012D00004A0DF68CAF80070D8F80440D3F814906E
:1012E000C4F8009005EBCC0C05EBC606DCF80470E6
:1012F000DC693C6076685F6A376005EBC00005EB2F
:10130000C1014468DE6A26604F68586B386005EB9F
:10131000C202D96B546840339E452160C2D1A74BAD
:10132000A64E5F6898683A683168A54BCBF81430D0
:10133000104300228BF818208BF820208BF82120F6
:10134000CBF82420CBF86820CBF86C203860CBF8A1
:101350001C100A70DBF81C70DFF870E27A70DBF8A2
:101360001C00984F8270DBF81C60FF21F170DBF8E5
:101370001C305A71DBF81C0050268671DBF81C10FB
:10138000CA71DBF81C005C4690F802B00BF07F03DA
:101390008370E669944604F114011222F270E1466A
:1013A000E04601914FF0FF304FF0010B864A0BFAF7
:1013B0000CF6002198E0CAF5C333A033834202D271
:1013C0001846E1468846538806FB03F3BEFBF3FA52
:1013D000BA4501F1010100F29D80CAF5C333A03383
:1013E000834202D21846E1468846938806FB03F3FF
:1013F000BEFBF3F3BB4201F1010A40F29780A3F573
:10140000C333A03B834205D2D046E146002B00F017
:10141000DF801846D38806FB03F3BEFBF3F3BB4221
:1014200001F1020A40F28C80A3F5C333A03B834252
:1014300005D2D046E146002B00F0CA801846138939
:1014400006FB03F3BEFBF3F3BB4201F1030A40F2D8
:101450008180A3F5C333A03B834205D2D046E14649
:10146000002B00F0B5801846538906FB03F3BEFB42
:10147000F3F3BB4201F1040A7ED9A3F5C333A03BC9
:10148000834205D2D046E146002B00F0A1801846E9
:10149000938906FB03F3BEFBF3F3BB4201F1050A9C
:1014A00061D9A3F5C333A03B834205D2D046E146C0
:1014B000002B00F08D801846D38906FB03F3BEFB9A
:1014C000F3F3BB4202F10E0201F1060A5DD9A3F566
:1014D000C333A03B834204D2D046E146002B77D0F1
:1014E0001846073140295BD0538806FB03F3BEFB47
:1014F000F3FABA4502F102027FF65DAFAAF5C333F3
:10150000A03B8342BFF45FAFE1468846002B5FD02B
:10151000184658E7AAF5C333A03B8342BFF465AF32
:10152000E1468846002B53D018465EE7C3F5C33327
:10153000A0338342BFF46EAFD0461846E14669E758
:10154000C3F5C333A0338342BFF479AFD046184606
:10155000E14674E7C3F5C333A033834284D2D04657
:101560001846E14680E7C3F5C333A0338342A3D2D4
:10157000D0461846E1469FE7C3F5C333A033834204
:1015800086D2D0461846E14682E7C3F5C333A0337E
:101590008342A6D207314029D0461846E146A3D15E
:1015A000BCF1020F14D00CF1010CFFE634B10100C4
:1015B00084A80100D9900000D8B6010010B3010042
:1015C00010A801009F8601006EB3010000879303FD
:1015D00008F03F02E069D14EDFF86C83D04942EA5F
:1015E000891A5FFA8AF34370E769CE4A787940F046
:1015F00020037B71E769787940F080037B71E769AC
:10160000B87840F08003BB7094F81890C64809EB96
:10161000490700EBC70B0127DBF80C00DFF82C9320
:1016200043099B0003F1604E0EF5614C00F01F0A68
:1016300007FA0AF0BD4BCCF8000001981860136857
:10164000A46743F4000010603068B94B20F002003A
:10165000306026464FF4803046F8741FC8F800000A
:101660008868DFF8EC8240F00200886041F2707018
:10167000086093E8030004F1800B0833C8F80060A9
:10168000C4F87C908BE8030093E8030004F1880E13
:101690008EE80300A74EA84BC4F89430002004F154
:1016A0007C0184F89000C4F80003C4F8040331609E
:1016B000166846F0006010609A6822F00C0199608C
:1016C0009E6846F0040098605A6A42F0040159622C
:1016D0005E6A26F0030058625A6A5A62D96841F07D
:1016E0000806DE60986840F003029A60996841F04D
:1016F00020069E60D86840F00402DA60196A8E48BD
:1017000011F040061EBF1E6A26F040061E62436AA4
:1017100043F0C00208BF37464262466A8649330634
:10172000FBD44B6A0B691FB10F6A47F04000086297
:10173000814F824ED7F84CC0B86C796C3A6CFB6B19
:10174000DFF810A2DFF81082604401440A44B86B4D
:10175000134403EB00090FCE4FEA590B4BF4004E34
:10176000C7F82CE004F54277C4F87CA00FC70FCE71
:101770000FC70FCE0FC796E80700002687E80700BF
:10178000474613214FF0100C11201222C4F8446375
:1017900047456B4EC4F87013C4F88C13C4F868C383
:1017A000C4F87CC3C4F86C03C4F88403C4F874237D
:1017B000C4F89423C4F87863C4F88063C4F88863D9
:1017C000C4F8906304F55E7A04F564794FF0010182
:1017D0000CD19AF8040002F07FFBD1450BD05AF8E7
:1017E000083F1F6847454FF00101F2D001215046E4
:1017F000B847D145F3D1019904F56670FAF7C0FBFB
:101800006FF000421C231B200021C4F84426C4F8BA
:10181000543684F84216C4F84C060221C4F84866CF
:10182000C4F8506602F058FB022194F8540602F006
:1018300053FBD5F8D800012700F50071C4F838161D
:1018400084F84076D5F8E02084F8417602F50073FC
:101850000220C4F83C3602F09FFBD4F8380694F816
:1018600040760178394205D094F8422642F0010BC7
:1018700084F842B6D4F83C0694F841E6037813EABB
:101880000E0F05D094F8427647F0020184F8421614
:1018900004F5C76A51461B20FBF790FA51461C20FD
:1018A000FBF78CFA0020274BC4F858066FF0004273
:1018B0000127C4F85C06C4F8600684F876061F2188
:1018C0001E20C4F86436C4F87826C4F88006C4F82C
:1018D0008816C4F87C660221C4F8846684F86876A9
:1018E00002F0FAFA022194F8880602F0F5FAD5F827
:1018F000F00084F8747600F50073C4F86C36D5F8FF
:10190000F82084F8757602F500710220C4F870168C
:1019100002F042FBD4F86C0620E000BF00700340E8
:10192000007103403C80044010B30100A444012036
:10193000F8A801009C43012000B0034008A9010061
:101940001CA801000100008004E100E034A80100AF
:10195000B444012044A80100610C000094F874C64E
:10196000037813EA0C0F04D094F876263A4384F8EF
:101970007626D4F8707694F875163878084205D033
:1019800094F8769649F0020B84F876B604F26C6A05
:1019900051461E20FBF712FA51461F20FBF70EFAA4
:1019A00000236FF0004201270820EA49C4F88C3672
:1019B000C4F89036C4F8943684F8AA360723C4F8DD
:1019C000AC26C4F8BC36C4F89816C4F8B406022194
:1019D000C4F8B066C4F8B86684F89C7602F07CFA65
:1019E000022194F8BC0602F077FA286C84F8A876F5
:1019F00000F50071C4F8A016AA6B84F8A97602F568
:101A000000730220C4F8A43602F0C6FAD4F8A00687
:101A100094F8A81690F800C01CEA010F04D094F8BE
:101A2000AA263A4384F8AA26D4F8A47694F8A9E61C
:101A30003B7813EA0E0F05D094F8AA0640F0020195
:101A400084F8AA1604F5D46949460820FBF7B6F9CC
:101A500049460720FBF7B2F900276FF0004209233F
:101A60000A20BC49C4F8E026C4F8F036C4F8C076B1
:101A7000C4F8C476C4F8C87684F8D07684F8DE76E4
:101A8000C4F8CC16C4F8E8060221C4F8E466C4F829
:101A9000EC6602F021FA022194F8F00602F01CFA3A
:101AA000286D012700F50071C4F8D41684F8DC769F
:101AB000AA6C84F8DD7602F500730220C4F8D836EB
:101AC00002F06AFAD4F8D40694F8DC760178394248
:101AD00005D094F8DE2642F0010B84F8DEB6D4F887
:101AE000D80694F8DDA6037813EA0A0F05D094F817
:101AF000DE7647F0020184F8DE1604F2D469494626
:101B00000A20FBF75BF949460920FBF757F9914F8B
:101B1000C4F8007700236FF000420C202021C4F8A5
:101B2000F436C4F8F836C4F8FC3684F8043784F880
:101B30001237C4F81427C4F81C07C4F82417C4F8D3
:101B400018670221C4F8206702F0C6F9022194F850
:101B5000240702F0C1F9286E012700F50073C4F8CC
:101B6000083784F81077D5F8002184F8117702F54A
:101B700000710220C4F80C1702F00EFAD4F808071E
:101B800094F8107703783B4205D094F8122742F07E
:101B9000010184F81217D4F80C0794F81177037830
:101BA0003B4205D094F8122742F0020184F8121744
:101BB00004F5E16B59460C20FBF700F9594620204B
:101BC000FBF7FCF800276FF0004218231920614949
:101BD000C4F84827C4F85837C4F82877C4F82C77D5
:101BE000C4F8307784F8387784F84677C4F8341727
:101BF000C4F850070221C4F84C67C4F8546702F0D7
:101C00006BF9022194F8580702F066F9D5F8C8007C
